:020000040002F8
:1060000020AF0020DD630200E5630200DD930200A3
:10601000E9630200EB630200ED6302000000000090
:10602000000000000000000000000000EF6302001C
:10603000F163020000000000F3630200F563020058
:10604000ADA10200F7630200B9CD020091B70200D2
:10605000A5B70200F76302008D92020071B0020042
:10606000F7630200F7630200F7630200F7630200C0
:10607000F7630200F7630200F7630200F7630200B0
:1060800005D1020015AB0200F7630200F7630200BE
:10609000F7630200F76302001DB80200F763020015
:1060A000F7630200F7630200F7630200F763020080
:1060B000A9A20200F7630200000000000000000037
:1060C000F7630200F7630200F7630200B9B702004A
:1060D0002DAB0200F7630200F7630200000000002E
:1060E00000000000000000000000000000000000B0
:1060F00000000000000000000000000000000000A0
:10610000000000000000000000000000000000008F
:10611000000000000000000000000000000000007F
:10612000000000000000000000000000000000006F
:10613000000000000000000000000000000000005F
:10614000000000000000000000000000000000004F
:10615000000000000000000000000000000000003F
:10616000000000000000000000000000000000002F
:10617000000000000000000000000000000000001F
:10618000000000000000000000000000000000000F
:1061900000000000000000000000000000000000FF
:1061A00000000000000000000000000000000000EF
:1061B00000000000000000000000000000000000DF
:1061C00000000000000000000000000000000000CF
:1061D00000000000000000000000000000000000BF
:1061E00000000000000000000000000000000000AF
:1061F000000000000000000000000000000000009F
:10620000DFF80CD000F0B8FC00480047EDE00300D8
:1062100020AF002000B583B002900091019244F2BB
:10622000010071466A460AF0E1FC03B000BD0000BF
:1062300030B450E8012F93B2C48923448489A34227
:1062400028BF1B1B0489A34202BFBFF32F8F00206E
:1062500007E0C3EA020340E80134002CE9D14FF023
:1062600001000A6030BC704750E8012FC2EA0242C8
:1062700040E801210029F7D1704730B450E8022FDF
:106280001FFAA2F3C488A34202BFBFF32F8F0020DE
:106290000DE0C48923448489A34228BF1B1BC2EAA2
:1062A000034340E80234002CE8D14FF001000A60BB
:1062B00030BC704750E8022FC2EA224240E8022177
:1062C0000029F7D17047034653E8022FD988B2EB73
:1062D000324F4FF0000017BF92B241EA014142EA4B
:1062E000014104E05A68B2EB324F08BF012043E895
:1062F0000212002AE8D1704730B4044654E8000F77
:106300000D4644E80053002BF8D1156030BC7047AF
:1063100030B4044654E8000F40EA010544E8005355
:10632000002BF7D1156030BC704730B4044654E8F8
:10633000000F00EA010544E80053002BF7D1156077
:1063400030BC704730B4044654E8000F80EA0105C1
:1063500044E80053002BF7D1156030BC704730B4CF
:10636000044654E8000F00EB010544E80053002BFD
:10637000F7D1156030BC704730B4044654E8000FC4
:10638000A0EB010544E80053002BF7D1156030BCA9
:10639000704770B404464FF0000054E8006F0D6879
:1063A000AE4207BF44E80023012044E800630E60CA
:1063B000002B1CBF0020F0E770BC704730B40446CF
:1063C00054E8000F88422CBF451A054644E80053A4
:1063D000002BF5D1156030BC70470000064880479F
:1063E00006480047FEE7FEE7FEE7FEE7FEE7FEE7BA
:1063F000FEE7FEE7FEE7FEE7F5C4020001620200E9
:106400002DE9F05F0546002092469B4688460646E9
:10641000814640241BE0284641464746224600F07C
:10642000A3FA53465A46C01A914110D31146184652
:10643000224600F016F82D1A67EB01084F46224657
:106440000120002100F00DF817EB00094E41201E3D
:10645000A4F10104DFDC484631462A464346BDE844
:10646000F09F202A04DB203A00FA02F10020704756
:106470009140C2F1200320FA03F319439040704782
:1064800040EA01039B0703D009E008C9121F08C0B6
:10649000042AFAD203E011F8013B00F8013B521E36
:1064A000F9D27047D2B201E000F8012B491EFBD2AD
:1064B00070470022F6E710B513460A46044619460F
:1064C000FFF7F0FF204610BD421C10F8011B002909
:1064D000FBD1801A704710B5002200E0521C835C8B
:1064E0008C5CA34201D1002BF8D1D8B2E1B2401AA2
:1064F00010BD30B504460020034600E05B1C93420B
:1065000003D2E05CCD5C401BF8D030BD034611F8EF
:10651000012B00F8012B002AF9D1184670472DE90C
:10652000FE4F804681EA0300C00F0C46009021F028
:10653000004123F00045B8EB0200A94105D24046D6
:10654000214690461C460B46024623F0004010436D
:1065500047D0270DC7F30A00C3F30A510290401A2F
:10656000019040286BDAC3F3130040F4801B0098BD
:10657000924620B10023D2EB030A63EB0B0B019888
:106580005946C0F140025046FFF76BFF06460D46E4
:1065900050465946019A00F0F7F910EB08006141A6
:1065A000002487EA115284EAE7731A4340D0009A24
:1065B00062B3019A012A4FEA075215DC001B61EB16
:1065C00002014FF0004202EA0752CDE90042001CEE
:1065D00041F5801132462B4600F02EFA03B0BDE89B
:1065E000F08F40462146F9E7001B61EB0201001CD9
:1065F00041F5801300185B412018A2F5001747EB06
:10660000030140EAD570B6196D4111E06D084FEAFB
:10661000360645EAC0754FEA0752001B61EB0201DE
:10662000001C41F5801149084FEA30000019514122
:1066300032462B4603B0BDE8F04F00F0EEB90098AB
:10664000012240000023D0EB020263EBE0730098CC
:1066500021464FEAE074B8EB000061EB0401E9E782
:1066600083F000435BE781F0004158E72DE9FE4FDE
:1066700081EA030404F0004421F0004100944FF04B
:10668000000B23F0004350EA01045ED052EA0304F9
:106690005BD0C3F30A54C1F30A552C44A4F2F3347B
:1066A0000194A0FB0254C1F3130141F48011C3F320
:1066B000130343F4801301FB024400FB034E840ADE
:1066C000970A44EA815447EA8357A4FB0768029576
:1066D0008D0A05FB07854FEA932C04FB0C54270514
:1066E000029D4FEA065847EA1637B5EB08056EEBF0
:1066F000070C870E920E47EA811742EA8312A7FB26
:106700000201B6EB0B0164EB00042B0D43EA0C33E2
:106710005E1844EB1C50DA465146E7FB0201C5F314
:1067200013044FEA0B3343EA14534FEA0432019C3B
:1067300043EA0603A4F10C040294009CCDE900B4E2
:1067400000F07AF903B0BDE8F08F00200146F9E7C8
:106750002DE9F04D81EA030404F0004B21F00045DF
:1067600014464FF0000A23F0004150EA050220D001
:1067700054EA01021DD0C5F30A570246C5F31303BC
:10678000C1F31300C1F30A5640F4801543F480139B
:10679000A7EB0608101BD64608F2FD3873EB050080
:1067A00002D308F1010801E092185B41B8F1000F33
:1067B00003DA00200146BDE8F08D00204FF480117F
:1067C000064684460EE0171B73EB050705D3121B24
:1067D00063EB050306434CEA010C49084FEA30001D
:1067E00092185B4150EA0107EDD152EA030012D042
:1067F00082EA040083EA0501084305D0101BAB417F
:1068000006D20122002306E000224FF0004302E0FE
:106810006FF0010253101AEB06004CEB085110EB1D
:106820000A0041EB0B01BDE8F04D00F0F6B80EB5E3
:10683000C10F80EAE0700844CA07002140F23343E8
:106840008DE80E000A460B4600F0F6F803B000BDD6
:106850000EB540F2334102910021CDE900110A4604
:106860000B4600F0E9F803B000BD70B5C1F30A5261
:1068700001F000450024C1F3130140F2FF3341F45D
:1068800080119A4201DA002070BD40F233439A42EF
:10689000A2F2334203DC524200F066F800E090407E
:1068A0002C43F1D0404270BDC1F30A5210B5C1F380
:1068B000130140F2FF3341F480119A4201DA0020C3
:1068C00010BD40F233439A42A2F2334203DC5242FB
:1068D00000F04AF810BD904010BD00F0004230F0CA
:1068E00000400AD0C10D01F56071C0F3160042EA04
:1068F0000151C2084007114370470020014670470C
:1069000030B5041E71F1000404DB4FF00044404236
:1069100064EB0101141E73F1000405DB1C464FF00B
:106920000043524263EB0403994208BF904230BDDA
:1069300001F0004330B421F0004150EA010206D0DA
:106940000A0DA2F56072C1F31301002A02DC30BC0B
:1069500000207047440F44EAC104C100E01830BC75
:1069600000EBC25000F022B8202A04DB203A21FAC2
:1069700002F00021704721FA02F3D040C2F1200258
:106980009140084319467047202A06DBCB17203A6E
:1069900041FA02F043EAE07306E041FA02F3D04024
:1069A000C2F1200291400843194670470029A8BF50
:1069B0007047401C490008BF20F00100704710B428
:1069C000B0FA80FC00FA0CF050EA010404BF10BCDD
:1069D000704749B1CCF1200421FA04F411FA0CF10A
:1069E00018BF012121430843A3EB0C01CB1D4FEA43
:1069F00000614FEA102042BF002010BC704700EB3E
:106A0000C35010440029A4BF10BC7047401C49006B
:106A100008BF20F0010010BC704710B5141E73F1C0
:106A2000000408DA401C41F1000192185B411A434E
:106A300001D120F0010010BD2DE9F04D92469B469A
:106A400011B1B1FA81F202E0B0FA80F22032904640
:106A5000FFF707FD04460F4640EA0A0041EA0B0132
:106A600053465A46084313D0114653EA010019D041
:106A7000C8F140025046FFF777FF05460E465046E4
:106A800059464246FFF7EDFC084305D0012004E0DB
:106A900020463946BDE8F08D0020054346EAE07601
:106AA0002C4337430A986305E40AA0EB0800002250
:106AB000FD0A44EA47540A3002D500200146E9E7BE
:106AC000010510196941DDE9084500196941BDE872
:106AD000F04DA2E72DE9F04D00231A461B1A8A411A
:106AE00003DB00200146BDE8F08DC1F30A52C1F37B
:106AF000130141F480154FF0000BD10702D10018AB
:106B00006D41521E0027044640F2FF11384601EB4A
:106B1000620A3E468046024600204FF48011FFF78D
:106B200023FFC2197141BB1846EB0100B4EB030C03
:106B300075EB000C04D3E41A65EB000517460E460E
:106B4000241908F101006D4180463428E3DDF9196C
:106B500046EB0600091BA84103D24FF0FF32134653
:106B600001E0002213461BEB070046EB0A51BDE88B
:106B7000F04DFFF752BF0000064C074D06E0E068FD
:106B800040F0010394E8070098471034AC42F6D374
:106B9000FFF73AFB308904005089040070B58C1867
:106BA00010F8015B15F0070301D110F8013B2A1121
:106BB00006D110F8012B03E010F8016B01F8016B0E
:106BC0005B1EF9D12B0705D40023521E0DD401F80A
:106BD000013BFAE710F8013BCB1A921C03E013F8D3
:106BE000015B01F8015B521EF9D5A142D8D3002008
:106BF00070BD00000023B3EB920F1FD093085B42DF
:106C000090ED000A0133B0EEC00A81ED000A90ED6C
:106C1000010AB0EEC00A81ED010A90ED020AB0EE61
:106C2000C00A81ED020A90ED030A00F11000B0EEF7
:106C3000C00A81ED030A01F11001E1D112F0030253
:106C400008BF7047524200BF90ED000A013200F1C8
:106C50000400B0EEC00A81ED000A01F10401F3D195
:106C60007047000010B51AF02BFE002001490860A3
:106C700010BD0000C440002010B500F00DF810BD9C
:106C800038B50446002000906946204600F0F8F828
:106C9000BDF9000038BD00002DE9F84F00265F481F
:106CA0000068009006208DF802006C465C4F04B925
:106CB0005C4C394620461AF017FD054600BF0DB161
:106CC0004FF0FF3600248FE0574850F83400FF287B
:106CD0007DD0554800EBC4004068FF28F8D0524AE8
:106CE00052F834000021002213461746944600BF94
:106CF0004FF0A049C84642EA430949EA810949EAF6
:106D0000072949EA0C4A08F5E06949F820A000BFC4
:106D100000BF0020444901EBC401496801EBC101F7
:106D2000424A5054404901EBC401496801EBC1019A
:106D3000114448703C4901EBC401496801EBC101B1
:106D400011448870384901EBC401496801EBC10165
:106D50001144C8700220344901EBC401496801EBB9
:106D6000C1011144087100202F4901EBC401496899
:106D700001EBC101114448712B4901EBC401496881
:106D800001EBC10111448871274800EBC400007970
:106D9000401C254901EBC401496801EBC1011144C4
:106DA000C8710020204901EBC401496801EBC10111
:106DB000114408721C4A02EBC402526802EBC20280
:106DC0001A4BD118184A02EBC402107900E00AE00D
:106DD0001AF0F2FB05460DB14FF0FF36144800687B
:106DE000401C13490860641C082CFFF66DAF104866
:106DF000006848B10E48008881B20E481AF07CFB4A
:106E000005460DB14FF0FF36701C20B90A4A0BA1A0
:106E1000002003F0D3FCBDE8F88F0000A48004003C
:106E2000ADF30200A080040080400020586D0020D7
:106E3000C4400020A06D0020453F03006273705FD6
:106E40006164635F696E69745F70726F63657373A9
:106E50000000000010B507211F2000F06BF804218E
:106E60001C2000F067F8FFF717FF034806F068FAE8
:106E7000024804F021FD10BD3355030029550300DD
:106E80002DE9FC4706460F464FF0030923A103C92D
:106E9000CDE900014FF00008002022490870224887
:106EA000006810B90520BDE8FC871AF0F1FC054622
:106EB0000DB10720F7E709E0B9F10000A9F10109D8
:106EC00002D019F0F1FB01E00620ECE7154800784C
:106ED0000028F1D000240DE004EBC400134908445D
:106EE000C07930B1E0B20DF8080008F1010000F0FF
:106EF000FF08641C082CEFDB002408E01DF80400E8
:106F0000B04203D10A4830F814003880641C0648A7
:106F100000688442F2D30020C5E70000FFFFFFFFB6
:106F2000FFFFFFFFC0400020C4400020586D00203C
:106F3000A06D002002460B4600211EE0114850F8CB
:106F40003100904201D1012070470E4800EBC10092
:106F50004068984201D10220F6E7FF2A0CD0094888
:106F600050F83100FF2807D1064840F8312000EBE7
:106F7000C10043600020E7E7491C0829DEDB03204D
:106F8000E2E70000804000202DE9F04106460F4670
:106F900014469846069DB0EE000A84ED000A95ED71
:106FA000020AB1EE400A84ED010A95ED010A84ED72
:106FB000020A95ED020A84ED030AB0EE000A84EDA0
:106FC000040A95ED000AB1EE400A84ED050A95ED3C
:106FD000010AB1EE400A84ED060A95ED000A84ED3F
:106FE000070AB0EE000A84ED080A4146204615F073
:106FF0004DFCB0EE000A84ED000A95ED020A84ED26
:10700000010A95ED010AB1EE400A84ED020A95ED00
:10701000020AB1EE400A84ED030AB0EE000A84EDE4
:10702000040A95ED000A84ED050A95ED010A84ED48
:10703000060A95ED000AB1EE400A84ED070AB0EEAB
:10704000000A84ED080A3A464146204617F0B9FC8A
:10705000242239462046FFF713FA3A4631462046A5
:1070600017F0AFFC242239463046FFF709FABDE895
:10707000F081000010B5054A05A1002003F09EFB39
:10708000074A08A1012003F099FB10BD0971020015
:10709000424C455F436C69656E745F527800000036
:1070A00009730200424C455F436C69656E745F541E
:1070B0007800000030B50346104A1068002900DC53
:1070C00030BD002214E00D4C2468601C0C4CA04222
:1070D00001D3A4F580600B4C2468A04206D09C5CD0
:1070E000064D2D682C70054C206000E002E0521C1B
:1070F0008A42E8DB00BF00BFE2E70000743F0020E7
:1071000098560020783F002070B565E0334800783D
:1071100010B101285BD12BE000F0BAFC032800D2AB
:1071200070BD002000F084FCAA2803D0012000F0EC
:107130008DFD1CE0022000F07BFC0446E043C4B25D
:10714000012000F075FC264908700846007884424A
:1071500009D108460078052805DB20480078401C46
:107160001E49087002E0012000F070FD00BF32E00F
:1071700000F08EFC1A490978884200D2D0E7002539
:10718000002406E0204600F053FC2844C5B2601CF1
:10719000C4B213480078401EA042F3DC10490978BD
:1071A000491E88B200F044FCA84208D10C4800787F
:1071B00003F08CFB0A48007800F048FD02E0012053
:1071C00000F044FD00200549087000BF03E00020E6
:1071D0000249087000BF00BF98E70000843F00200C
:1071E000853F002010B5024610480068112802D3E0
:1071F0004FF0FF3010BD0E480C4B1B6800EB031026
:10720000C1600B48094B1B6800EB03100270094872
:10721000074B064C246803EB0413586003480068CE
:10722000401C024B18600020E4E700007C3F002077
:1072300098560020A85700202DE9F047C0B080469E
:107240008946164600250024701D00F0FF0AFA2E1C
:1072500003DD601E40B0BDE8F087AA200DF80400F1
:107260002046611CCCB21DF800002844C5B20DF8C0
:1072700004A02046611CCCB21DF800002844C5B211
:107280006FEA0A00C0B20DF804002046611CCCB2BF
:107290001DF800002844C5B20DF804802046611C8A
:1072A000CCB21DF800002844C5B200270CE019F844
:1072B00007000DF804002046611CCCB21DF8000048
:1072C0002844C5B2781CC7B2B742F0DB2046611C27
:1072D000CCB20DF80050214668461EF0B3FDB9E768
:1072E00008490AE00A68824204D100234376136AFF
:1072F0000B6001E002F1200100BF0A68002AF1D111
:1073000070470000803F002070B5002600251E4811
:10731000046831E0E06800282BD005F03BFA1B49F7
:107320000968451A05F036FA1849086005B90125BB
:10733000E068A84203D3E068401BE06001E0002061
:10734000E060E068A8B9207A00280ADD207A401EB3
:1073500020726068E060227E207C6169FFF76CFF2C
:1073600007E02046FFF7BCFFE06910B12046E16965
:107370008847607E0643246A002CCBD13146AFF2A9
:10738000770003F0F7F970BD803F0020883F0020B0
:107390002DE9F0410446884615461E461348076805
:1073A000ECB184F81080656126766068E060207832
:1073B000002803DD2078401E207201E000202072AA
:1073C0000120607604E0A74201D1BDE8F0813F6A68
:1073D000002FF8D105480068206204480460324656
:1073E00029464046FFF728FF00BFEEE7803F002018
:1073F00010B5054A05A1002003F0E0F9064A07A1EF
:10740000012003F0DBF910BDB1740200424C455F6E
:10741000486F73745F527800C1760200424C455F3A
:10742000486F73745F5478002DE9F04104460D46AF
:107430001B480668052D01DABDE8F0816778A07861
:10744000C04300F0FF082078AA280CD147450AD194
:10745000AF4208D1E078052805DAE9B22046114AA2
:107460001268904719E0002014E00D4909684E1C8D
:107470000D498E4201D3A1F580660C4909688E4200
:1074800006D0215C064A1268117005490E6000E0C2
:1074900002E0401CA842E8DB00BF00BFCCE70000D0
:1074A0008C3F0020943F0020A85C0020903F0020EB
:1074B00070B565E03348007810B101285BD12BE04E
:1074C00000F0F6FA032800D270BD002000F0C0FAE8
:1074D000AA2803D0012000F0DDFB1CE0022000F010
:1074E000B7FA0446E043C4B2012000F0B1FA2649DD
:1074F000087008460078844209D1084600780528BB
:1075000005DB20480078401C1E49087002E001207D
:1075100000F0C0FB00BF32E000F0CAFA1A49097857
:10752000884200D2D0E70025002406E0204600F083
:107530008FFA2844C5B2601CC4B213480078401EBC
:10754000A042F3DC10490978491E88B200F080FAA5
:10755000A84208D10C48007803F0F8F90A480078EE
:1075600000F098FB02E0012000F094FB00200549A8
:10757000087000BF03E000200249087000BF00BF90
:1075800098E70000A03F0020A13F002010B5024670
:1075900010480068112802D34FF0FF3010BD0E488C
:1075A0000C4B1B6800EB0310C1600B48094B1B68B8
:1075B00000EB031002700948074B064C246803EBEC
:1075C0000413586003480068401C024B18600020F8
:1075D000E4E70000983F0020A85C0020B85D002090
:1075E000014602480160002070470000943F0020DF
:1075F0002DE9F047C0B08046894616460025002494
:10760000701D00F0FF0AFA2E02DD40B0BDE8F087E1
:10761000AA200DF804002046611CCCB21DF8000021
:107620002844C5B20DF804A02046611CCCB21DF858
:1076300000002844C5B26FEA0A00C0B20DF8040089
:107640002046611CCCB21DF800002844C5B20DF8DC
:1076500004802046611CCCB21DF800002844C5B24D
:1076600000270CE019F807000DF804002046611C03
:10767000CCB21DF800002844C5B2781CC7B2B7428E
:10768000F0DB2046611CCCB20DF800502146684664
:107690001EF0F2FB00BFB8E708490AE00A68824220
:1076A00004D100234376136A0B6001E002F120014C
:1076B00000BF0A68002AF1D1704700009C3F0020FB
:1076C00070B5002600251E48046831E0E0680028F7
:1076D0002BD005F05FF81B490968451A05F05AF8E8
:1076E0001849086005B90125E068A84203D3E0689D
:1076F000401BE06001E00020E060E068A8B9207A6B
:1077000000280ADD207A401E20726068E060227E38
:10771000207C6169FFF76CFF07E02046FFF7BCFFA4
:10772000E06910B12046E1698847607E0643246A1B
:10773000002CCBD13146AFF2770003F01BF870BDBF
:107740009C3F0020A43F00202DE9F04104468846DC
:1077500015461E4613480768ECB184F81080656131
:1077600026766068E0602078002803DD2078401EDF
:10777000207201E0002020720120607604E0A74220
:1077800001D1BDE8F0813F6A002FF8D105480068BB
:10779000206204480460324629464046FFF728FF2D
:1077A00000BFEEE79C3F002010B50446002116E024
:1077B0000F4850F82100A04202D14FF0FF3010BD19
:1077C0000B4850F8210048B90A480078401C094A83
:1077D0001070074840F821400020F0E7491C0329B9
:1077E000E6DB05A1002003F089FD6FF00100E6E76C
:1077F000987500208C470020626C655F6576745F29
:10780000526567697374202D3E20746F6F206D611F
:107810006E79210A0000000010B50446002116E030
:107820000F4850F82100A04202D14FF0FF3010BDA8
:107830000B4850F8210048B90A480078401C094A12
:107840001070074840F821400020F0E7491C10293B
:10785000E6DB05A1002003F051FD6FF00100E6E733
:107860000073002052410020626C655F6576745F92
:10787000526567697374202D3E20746F6F206D61AF
:107880006E79210A0000000030B52DED048B83B025
:10789000B0EE408AF0EE608A3148007800285CD073
:1078A00018EE900AFFF719F841EC190B9FED2D0B1C
:1078B00053EC102BFFF724F804D3F4EEC88AF1EE52
:1078C00010FA04D2032003B0BDEC048B30BDB1EE3E
:1078D0000E0AB4EEC08AF1EE10FA01D20320F2E7EC
:1078E0009FED220A28EE800ADFED210A80EE201AA1
:1078F000BCEEC10A10EE100A80B2ADF806009FED92
:107900001B0A28EE000ADFED1A0A80EE201ABCEEF0
:10791000C10A10EE100A80B2ADF804004FF4C8702E
:10792000ADF80A000020ADF808001249088901A945
:1079300075DF0446082C0ED0112C0CD05CB100BFB2
:1079400025463DB100BF0CA240F289212846FEF732
:1079500061FC00BF00BF2046B5E70120B3E700008F
:107960008247002000000000003B9F4000007A4456
:1079700000409C44807300202E2E5C2E2E5C2E2E08
:107980005C626C655F6366675C686F73742E63002E
:10799000F0B503460C4698B24FF4004700211DE0B5
:1079A000665C80EA062C1FFA8CF0082513E000EADA
:1079B000070CBCF1000F06D048F2050C8CEA400C15
:1079C0001FFA8CF003E04FF6FF7C0CEA4000A5F1B3
:1079D000010C0CF0FF05002DE9DC491C9142DFD3BE
:1079E00000BFF0BD9FED0E2AC0EE022A9FED0D2ACA
:1079F00022EE822AB0EE421A9FED0B2A21EE022AD5
:107A000022EE202ADFED092A82EE223AF0EE431A16
:107A100090ED002A32EE212A80ED002A7047000006
:107A200000803B45CDCC8C3F00007A44000061458E
:107A300002460548006881180448814201D3A1F537
:107A40008061087870470000783F00209856002039
:107A500002460548006881180448814201D3A1F517
:107A60008061087870470000903F0020A85C0020EB
:107A700002460548006881180448814201D3A1F5F7
:107A80008061087870470000E03F0020D863002044
:107A9000054B1A68054B19688A4201D3501A02E057
:107AA00002F58063581A7047743F0020783F002029
:107AB000054B1A68054B19688A4201D3501A02E037
:107AC00002F58063581A70478C3F0020903F0020D9
:107AD000054B1A68054B19688A4201D3501A02E017
:107AE00002F58063581A7047DC3F0020E03F002019
:107AF00070B52DED108B82B006460C469FED520AF4
:107B0000F0EE408A9FED500AB0EE409A00251AE050
:107B100018EE900AFEF7E1FE41EC1B0B06EBC500E8
:107B200090ED001BB0EE410AF0EE610A53EC102B11
:107B300051EC1B0BFEF7F3FC41EC1A0BFEF7F8FEC1
:107B400008EE900A6D1CA542E2D300EE104AB8EE92
:107B5000400A88EE808A002542E018EE100AFEF7FF
:107B6000BCFE41EC1E0B06EBC50090ED001BB0EE19
:107B7000410AF0EE610A53EC102B51EC1E0BFEF79C
:107B800072FD41EC1F0B18EE100AFEF7A6FE41EC49
:107B90001E0B06EBC50090ED001BB0EE410AF0EEA7
:107BA000610A53EC102B51EC1E0BFEF75CFD41EC0F
:107BB0001D0B53EC1F2BFEF759FD41EC1B0B19EE6F
:107BC000100AFEF78AFE41EC1C0B53EC1B2BFEF750
:107BD000A6FC41EC1A0BFEF7ABFE09EE100A6D1C79
:107BE000A542BAD39FED180A8DED010A9FED160A42
:107BF0008DED000A00EE904AF8EE600A89EE200A48
:107C0000B5EEC00AF1EE10FA05DBF1EEC00ACDEDDB
:107C1000010A002005E0DFED0C0ACDED010A4FF06E
:107C2000FF3050B99DED010AC0EE080ACDED010A02
:107C30000122694601A8FEF7DDFF9DED000A02B0B2
:107C4000BDEC108B70BD00000000000018E0411E6C
:107C500088B20D4909680D4A1268914200D17047F7
:107C600009490968491C0A4A914204D3A2F5806176
:107C7000054A116004E004490968491C024A116080
:107C80000028E4D100BFEAE7783F0020743F0020DD
:107C90009856002018E0411E88B20D4909680D4A27
:107CA0001268914200D1704709490968491C0A4A83
:107CB000914204D3A2F58061054A116004E00449B1
:107CC0000968491C024A11600028E4D100BFEAE7B4
:107CD000903F00208C3F0020A85C002018E0411E4F
:107CE00088B20D4909680D4A1268914200D1704767
:107CF00009490968491C0A4A914204D3A2F58061E6
:107D0000054A116004E004490968491C024A1160EF
:107D10000028E4D100BFEAE7E03F0020DC3F00207C
:107D2000D863002038B505466946284601F034FB83
:107D300004460CB1204638BD009801F0E9F9FAE795
:107D40000849095C01290CD1002206490A54891FFF
:107D5000098C31B10349891F098C491E014A921FC0
:107D6000118470471A4F0020014600200DE000EBFF
:107D70008002074B03EBC20292F8252022B900EBE8
:107D8000800203EBC2021162401C0228EFDB704745
:107D90009CFF002001460348405C012800D1704749
:107DA0000020FCE71A4F00200348008C002801DD6A
:107DB000012070470020FCE7144F002010B500217F
:107DC000064802F0D7FC012005490870322048809F
:107DD00001208880072001F0B1FF10BDE180020082
:107DE000144F002010B51A48408800282ED00121D9
:107DF000184802F0BFFC1648808868B9144800781B
:107E000018B901201249087002E0002010490870DA
:107E100001200F49888014E00D48007818B90E49F8
:107E2000072001F06FFF0A480078012804D14FF0C5
:107E30007F41072001F066FF05488088401E044905
:107E4000888003484088401E0149488010BD0000DA
:107E5000144F0020E180020000106FFF70B504464F
:107E6000241F26A1002003F049FA4FF40070B0EB64
:107E7000145F04D03149002003F040FA70BD08348B
:107E800001212F4880F84D1080F84C102022214607
:107E90002830FEF7F5FA2546A869C01E2C46A861D1
:107EA00028A100202A6803F029FA29A100206A6885
:107EB00003F024FA29A10020AA6803F01FFA2AA1DE
:107EC0000020EA6803F01AFA2AA100202A6903F0C8
:107ED00015FA2CA100206A6903F010FA2CA10020E9
:107EE000AA6903F00BFA2DA10020EA6903F006FA53
:107EF0002EA1002003F002FA00BFBFE70D0A2D2DCE
:107F00002D2D2D2D2D2D2D2D2D2D2D2D2D2D2D4589
:107F100052524F52202D2D2D2D2D2D2D2D2D2D2D0D
:107F20002D2D2D2D2D2D0D0A486172644661756C25
:107F3000745F48616E646C65720D0A000888040005
:107F40009CFF002052303A3078253038580D0A0016
:107F500052313A3078253038580D0A0052323A30D2
:107F600078253038580D0A0052333A3078253038A9
:107F7000580D0A005231323A3078253038580D0AFF
:107F8000000000004C523A3078253038580D0A0075
:107F900050433A3078253038580D0A007850535203
:107FA0003A3078253038580D0A0000007379737420
:107FB000656D2072657365742E2E2E0D0A0000000B
:107FC0000649095C012908D0012204490A54891F85
:107FD000098C491C014A921F118470471A4F0020D6
:107FE000F0B5BFB006460F46002400253846FEF720
:107FF0006BFA85B2F82D02D9601E3FB0F0BD114872
:10800000007930B100222046611CCCB20DF800206E
:1080100005E001222046611CCCB20DF8002020466C
:10802000611CCCB20DF800600DEB04002A46394605
:10803000FEF726FA6019C4B222466946AD20FFF762
:10804000FBF8DAE7085200200120024981F82500F8
:10805000704700009CFF002010B522210C48FEF75D
:1080600028FA01200A4908703220488001208880BF
:10807000084A09A1C82002F0A1FB0D4A0DA1642005
:1080800002F09CFB1549AD20FFF780FA10BD0000FF
:10809000144F0020E1800200457863657074696FB9
:1080A0006E5F4C65645F50726F63657373000000B0
:1080B00045810200457863657074696F6E5F556E27
:1080C0006B6F776E52657365745F496E666F5F5351
:1080D000656E645F50726F63657373005D5003007B
:1080E00000B589B0002012F035FD012810DB01AA8F
:1080F0000021084612F024FDBDF80400ADF81C0074
:10810000BDF80600ADF81E00BDF80800ADF820006F
:10811000BDF9200040F2DC51884206DB0748008CA4
:10812000002802DDFFF75EFE06E0BDF920000449ED
:10813000884201DCFFF742FE09B000BD144F002069
:1081400024FAFFFF30B5C7B00024EAE004EB840056
:10815000764901EBC00090F8250001286FD104EBAF
:10816000840001EBC00090F8240010B1012868D110
:1081700017E004EB84006D4901EBC0006CA1026ABA
:1081800007A805F0ABFC07A91020FFF729FF38B9B5
:10819000002004EB8401654A02EBC10181F825004F
:1081A00050E004EB8400614901EBC000C16904EBBD
:1081B00084005E4A02EBC0008069C01E04EB8402AA
:1081C0005A4B03EBC202526904EB8403574D05EB93
:1081D000C3031B69CDE90332CDE9050104EB84003B
:1081E000294601EBC000C06804EB84012A4602EB7B
:1081F000C101896804EB84022B4603EBC20252687A
:10820000CDE90021029004EB8400194651F830308A
:1082100004EB840001EBC00047A1026A07A805F047
:108220005DFC07A91020FFF7DBFE38B9002004EB46
:1082300084012A4602EBC10181F8250002E06FE0CB
:10824000FFE700BF00BF04EB8400384901EBC0002A
:1082500090F82400012859D104EB840051F8302013
:1082600042A1002003F04AF804EB84002F4901EBFF
:10827000C00041A14268002003F040F804EB8400F4
:108280002A4901EBC0003FA18268002003F036F8C4
:1082900004EB8400254901EBC0003DA1C268002029
:1082A00003F02CF804EB8400204901EBC0003BA153
:1082B0000269002003F022F804EB84001B4901EB63
:1082C000C0003AA14269002003F018F804EB8400D2
:1082D000164901EBC0008069C21E37A1002003F0DF
:1082E0000DF804EB8400114901EBC00035A1C2690F
:1082F000002003F003F804EB84000C4901EBC000FC
:108300000BA1026A002002F0F9FF09E004EB8400EF
:10831000064901EBC00006A1026A002002F0EEFF50
:10832000641C022CFFF612AF47B030BD9CFF00204A
:1083300069643A25640D0A0069643A25642C523A4E
:10834000307825782C307825782C307825782C30AA
:108350007825782C307825782C307825782C307852
:1083600025782C307825780D0A00000052303A30FC
:1083700078253038580D0A0052313A307825303897
:10838000580D0A0052323A3078253038580D0A001C
:1083900052333A3078253038580D0A005231323A8B
:1083A0003078253038580D0A000000004C523A3021
:1083B00078253038580D0A0050433A307825303847
:1083C000580D0A00785053523A3078253038580DFD
:1083D0000A0000007047000010B50248006805F070
:1083E00001F910BD483F002010B500210348C0F836
:1083F0002B100348006805F0F5F810BD0852002066
:108400004C3F002070B504461822214603480068FE
:1084100005F052F90546284670BD0000503F002087
:108420002DE9F043C5B00446782126A8FEF741F8AF
:10843000B0A10020449A02F061FF44A9B948006845
:1084400005F0FEF806461EB1304645B0BDE8F083A3
:10845000A8A10020449A02F051FF4498451E10E064
:10846000B04909684819012225A905F025F90646F1
:108470000EB13046E9E79DF89400A52800D102E04E
:108480006D1E002DECDA00BF002D19DA7821204690
:10849000FEF70FF8A4482060782020677822214654
:1084A0000020FFF775FA1FFA80F8A04848EA00009C
:1084B00060679FA10020626F02F020FF0020C4E7E8
:1084C0006D1C984909682944081F042243A905F036
:1084D000F3F806460EB13046B7E7924909682944D9
:1084E000A1F10800042242A905F0E6F806460EB103
:1084F0003046AAE70027E8194299884201D24298FB
:10850000471B8849096829443944429A881A042239
:1085100026A905F0D1F806460EB1304695E70EE0E3
:108520007F1C8049096829443944429A881A0422E8
:1085300026A905F0C1F806460EB1304685E77A490E
:1085400026988842ECD107F108004299814201D86F
:1085500004207AE77349096829443944429BC81AC0
:10856000A3F10801CA1B26A905F0A6F806460EB11C
:1085700030466AE707F108004299814245D843989E
:1085800083B2424676A1002002F0B8FE7821204650
:10859000FDF78FFF644820607820206701A8FFF76F
:1085A00031FF00200AE00DF10E010A5C04F13501F3
:1085B0000A5402A90A5C611D0A54401C0628F2DB19
:1085C0009DF8190084F82F00059921639DF8181073
:1085D00034200155782221460020FFF7D9F91FFAEF
:1085E00080F8524848EA000060674E48006804F08E
:1085F000F9FF06460EB1304627E700F0AFFB06460E
:108600000EB1304621E700201FE7782107A8FDF7CB
:1086100050FF0DF11C0942980838C21B26A9484694
:10862000FDF72EFF429848440838C01B429901606C
:1086300049460020429AFFF7ABF91FFA80F84398A9
:1086400080B2404515D138482690782042900020CD
:108650004390782226A9FFF79BF91FFA80F8334848
:1086600048EA00004390782226A92046FDF708FF3B
:108670003DE078212046FDF71CFF2B482060782044
:10868000206701A8FFF7BEFE00200AE00DF10E01F1
:108690000A5C04F135010A5402A90A5C611D0A54FE
:1086A000401C0628F2DB9DF8190084F82F0005997C
:1086B00021639DF8181034200155782221460020AE
:1086C000FFF766F91FFA80F8184848EA000060676B
:1086D0001448006804F086FF06460EB13046B4E642
:1086E00000F03CFB06460EB13046AEE600BF00206F
:1086F000ABE600005A6F6E655F476574427974653A
:1087000053697A6528696E666F5F7A6F6E652C2093
:10871000267A6F6E655F6279746573293A25640AFB
:1087200000000000483F0020AA5555AA000055A5AA
:1087300072656164207A6F6E6520616C6C20636C79
:108740006561722C70666C6173682D3E7461696C32
:108750005F63726331363A307825780D0A00000085
:10876000737472756374206368616E67652C7265DB
:10877000616420637263206661696C203A307825F9
:10878000782030782578200D0A0000000148006824
:10879000704700004C3F00202DE9F843002700F00F
:1087A0008FFCA349012004F0CDFE05462A46A1A175
:1087B000002002F0A3FDAD49022004F0C3FE0546EF
:1087C0002A46ABA1002002F099FDB749012004F030
:1087D000B9FE05462A46B5A1002002F08FFDC24829
:1087E000FFF710FE80464246C0A1002002F086FD41
:1087F000BD48807D05280EDBFFF7EEFDFFF7F4FD99
:108800000020B949887500F08DFAC0A1002002F05F
:1088100075FD05F0A1F9B448807D401CB24988750A
:1088200000F080FA82480468C2A10020226802F0A9
:1088300065FDC649206888427ED0C5A10020226817
:1088400002F05CFD7821CF48FDF733FEBF48CD49EB
:1088500008607820086794480668BC4930688842F8
:1088600054D1002500200CE09F49091D0A5CC54930
:10887000491D0A549C490A310A5CC24935310A54DF
:10888000401C0628F0DBC0A1002002F037FD0025C7
:1088900008E09548001D425DBFA1002002F02EFDBA
:1088A000681CC5B2062DF4DBBDA1002002F026FD38
:1088B000BCA1002002F022FD002508E08A480A3011
:1088C000425DB5A1002002F019FD681CC5B2062D5D
:1088D000F4DBB3A1002002F011FD83480169A9482F
:1088E00001638148017DA74880F834107E48407DAF
:1088F000A44981F82F007C48007D00907A480369E4
:10890000427DACA1002002F0F9FC05E01821764878
:10891000FDF7CFFD00F006FA00F020FAB3A1002029
:10892000226802F0EBFC8949206888420CD0B7A18C
:10893000002002F0E3FC00E019E0BAA10820FFF7F4
:108940004FFB0127BDE8F883BCA10020226802F09C
:10895000D5FC002507E04FF4FA7017F0EDF80FF0A2
:10896000C1FF681CC5B2062DF5DB05F0F5F847B967
:108970008448FFF755FD80464246B5A1002002F02D
:10898000BDFC8048D0F81B10D0F82300814204D2EF
:108990007C48D0F81B10C0F823107A48D0F82B2060
:1089A000B4A1002002F0AAFC7648D0F81F30D0F81D
:1089B0001B20B6A1002002F0A1FC724A3C32C1A1EA
:1089C000002002F09BFCC3A1002002F097FC0120D4
:1089D0006C4908710321102017F0B6FB642017F0D2
:1089E000ABF8102000BF4FF0A042114600BFD1F8F5
:1089F0001025C24002F0010262480271007901288C
:108A000004D10121102017F09FFB03E0002110206A
:108A100017F09AFB5B48007920B1B2A1002002F068
:108A20006DFC03E0B7A1002002F068FC00BF89E7FD
:108A3000483F00205A6F6E655F416C6C6F63612820
:108A4000464C4153485F414444525F494E464F5F54
:108A5000504147454E554D2C2026696E666F5F7A12
:108A60006F6E65293A25640A000000004C3F002023
:108A70005A6F6E655F416C6C6F636128464C415361
:108A8000485F414444525F535445505F504147450D
:108A90004E554D2C2026737465705F7A6F6E652974
:108AA0003A25640A00000000503F00205A6F6E65AE
:108AB0005F416C6C6F636128464C4153485F414491
:108AC00044525F4241434B55505F504147454E55DC
:108AD0004D2C20266261636B75705F7A6F6E65291D
:108AE0003A25640A0000000080520020466C617341
:108AF000685F4765744261636B75702028266D421C
:108B000061636B7570293A25640A00006D426163E8
:108B10006B75702E4572726F725374617274466C0D
:108B20006167203E3D203521212121212121212164
:108B300021210A00466C61736820686561642072B7
:108B40006561642825303458292E0A00AA5555AA93
:108B5000466C61736820666972737420696E69740B
:108B60002825303458292C777269746520696E661F
:108B70006F6D6174696F6E20746F20666C617368CD
:108B80002E0A0000085200204261636B206D616371
:108B9000416464725F4C3A00253032583A0000005C
:108BA0000D0A00004261636B206D61634164647271
:108BB0005F523A004261636B20446174613A6966B6
:108BC000636F6E6669673A25642C686172645665E6
:108BD000723A25642C6261636B75702E736F6674D4
:108BE00076657273696F6E3A25640A00466C61732C
:108BF000682068656164207365636F6E64207265C8
:108C000061642825303458292E0A0000466C6173AF
:108C1000682077726974652068656164206661699F
:108C20006C2E0A00466C6173682077726974652047
:108C300068656164206661696C0000005379737433
:108C4000656D2072657365742E2E2E0A000000007B
:108C5000466C6173685F476574496E666F6D6174D9
:108C6000696F6E28266D466C617368293A25642009
:108C70000A0000006D466C6173682E6D5374657058
:108C80002E6E756D3D25640A000000006D466C6116
:108C900073682E6D537465702E73746570437572AE
:108CA0005B305D3D25642C6D466C6173682E6D53A1
:108CB0007465702E737465704375725B315D3D250C
:108CC000640A000065727220636F6465203A257340
:108CD0000A000000466C61736820696E6974206F39
:108CE0006B2E0A003D3D3D3D3D3D3D204C6566748B
:108CF000202073686F6F65203D3D3D3D3D3D3D202B
:108D00000A0000003D3D3D3D3D3D3D205269676804
:108D1000742073686F6F65203D3D3D3D3D3D3D20B6
:108D20000A00000010B50A480A4908600A480068AD
:108D300004F058FC04460CB1204610BD1822054929
:108D40000548006804F0E6FC04462046F5E700000C
:108D5000AA5555AA80520020503F0020F0B5A1B07E
:108D6000782102A8FDF7A5FB20A95248006804F06D
:108D700067FC054615B1284621B0F0BD2098441E79
:108D800010E04C4909680819012201A904F094FC7B
:108D900005460DB12846EFE79DF80400A52800D14F
:108DA00002E0641E002CECDA00BF00204249486754
:108DB000782008674148086078220020FEF7E8FD27
:108DC00087B23F4838433C494867002C0FDA782285
:108DD0003848006804F09EFC05460DB12846CBE7F4
:108DE000354838A1426F002002F088FA5FE0641C29
:108DF000304909682144081F04221FA904F05CFCC3
:108E000005460DB12846B7E72A4909682144A1F172
:108E1000080004221EA904F04FFC05460DB12846A7
:108E2000AAE70026A0191E99884201D21E98061BA7
:108E300020490968214431441E9A881A042202A953
:108E400004F03AFC05460DB1284695E70EE0761C85
:108E500018490968214431441E9A881A042202A93B
:108E600004F02AFC05460DB1284685E7134902980F
:108E70008842ECD10F4909682144881978220E49AB
:108E800004F048FC05468DB10A48006804F0AAFBCE
:108E900005460DB128466FE7782207490548006866
:108EA00004F038FC05460DB1284665E700BF0020F8
:108EB00062E70000483F002008520020AA5555AA4A
:108EC000000055A57772697465207A6F6E65206120
:108ED0006C6C20636C6561722C6D466C6173682EDE
:108EE0007461696C5F63726331363A307825780D4E
:108EF0000A000000F8B506460F46144634212548FE
:108F0000FDF7D7FA012023493B3981F83B00012EB8
:108F10000CD06FF48050304478B1B0F5405F1CD075
:108F20006FF440510844002829D10DE032221AA1E3
:108F30001848401CFDF7A4FA28E032221CA115486D
:108F4000401CFDF79DFA21E0254620A11148401C58
:108F5000D5E9003204F0C2FD18E0254628680090EB
:108F600021A10C48401CD5E9013204F0B7FD094BA2
:108F70005B1C22A10020AA6802F0C0F906E03A4674
:108F800024A10448401C04F0A9FD00BF00BFFFF766
:108F9000E5FEF8BD4352002053443A204153534567
:108FA0005254494F4E204641494C45440D0A000059
:108FB00053443A20494E56414C4944204D454D4F6B
:108FC0005259204143434553530D0A0041535345E1
:108FD0005254494F4E204641494C45442025733A4E
:108FE00025750D0A000000006572726F723A2575D2
:108FF0002C25733A25750D0A000000003E3E3E3ECA
:109000003E65727220636F6465203A25642C257377
:1090100000000000554E4B4E4F574E204641554CD8
:1090200054203078253038580A000000F8B521481F
:10903000D0F82B0020490968884236D209F042F95D
:10904000064609F045F934184FF07F4000EA046005
:109050004FF47F0101EA042108434FF47F4101EA04
:109060001421084340EA146000901249D1F82B10F3
:10907000124A126802EB81000422694604F04AFB9E
:1090800005460DB12846F8BD0A48D0F82B00401C13
:109090000849C1F82B000846D0F81B10C0F823106F
:1090A000D0F81F10C0F8271001E00520EBE70020E2
:1090B000E9E7000008520020543F00204C3F002008
:1090C00070B50026094D00222946094816F079FEA0
:1090D000044604B1761E10F0F3FC701C20B9054A5A
:1090E00005A1002001F06AFB70BD0000C8840400E7
:1090F000004B0020753F03006273705F666C617304
:10910000685F696E69745F70726F63657373000086
:1091100070B5044604F0030000B90CB9032070BD1B
:10912000B4F5E82F0AD0B4F5EA2F07D0B4F5EC2F48
:1091300004D0B4F5EE2F01D0012000E0002008B1EA
:109140000120ECE7002301222146064816F003FE29
:1091500005460DB10920E2E702481EF0BEFA0020E4
:10916000DDE70000004B00202DE9F84F044688465B
:109170001546994604F0030000B914B90320BDE870
:10918000F88F05F0030000B90DB90420F7E7601966
:10919000B0F5F02F01D90220F1E7B9F1000F0DD0A1
:1091A0004FEA950B002607E054F826A00AF10100CB
:1091B00008B10520E3E7761C5E45F5D300202B4679
:1091C000424621460090064816F0DCFE07460FB1E5
:1091D0000820D4E702481EF080FA0020CFE7000004
:1091E000004B00202DE9F84304460F4690461E46EA
:1091F00004F0030000B914B90320BDE8F883A019F6
:10920000B0F5F02F01D90220F7E74FB933464246B7
:1092100021461D4816F014FE05467DB30720ECE7F5
:1092200006F0030000B90EB90420E6E7B4F5E82F14
:109230000AD0B4F5EA2F07D0B4F5EC2F04D0B4F57A
:10924000EE2F01D0012000E0002008B10120D4E77A
:109250000023012221460C4816F07DFD05460DB184
:109260000920CAE7002033464246214600900648BE
:1092700016F088FE054615B10820BEE702E0024858
:109280001EF02BFA0020B8E7004B00202DE9F84F24
:109290000026002000904FF480770125002410E084
:1092A000384617F003F940B100BF25480068284050
:1092B00018B1384617F0ECF82E436D00381D87B210
:1092C000641C082CECD34FF4BE7017F0EFF850B1CB
:1092D0004FF4BE7017F0DCF846F000466A460121F4
:1092E000002016F0C7FFF0B210B3012500241DE0E6
:1092F00005EA0600C0B100BF124850F82400C0F3D0
:109300000420814600BF0F4850F82400C0F30140FC
:10931000824620460CF05AF98046B8F1000F02D080
:1093200051464846C04700BF6D00641C082CDFD37F
:1093300006F0004010B168461AF078FBBDE8F88FDF
:1093400004630040106500400020084991ED000AC8
:10935000F6EE000A30EE200ABCEEC00A10EE101A3B
:10936000C8B2642800DD642070470000F83F002088
:10937000024602F0030000B90AB903207047B2F5B3
:10938000F02F02D8B2F5E82F01D20220F6E7C2F39F
:10939000890008600020F1E70246042A01D3062074
:1093A00070474FF4E82000EB023008600020F7E738
:1093B00002460023B2F5F02F02D8B2F5E82F01D211
:1093C00002207047A2F5E820C0F30F33042B01D32D
:1093D0000620F6E70B800020F3E7000000BFEFF364
:1093E0000880804600BFEFF3098000BF4046FEF7CB
:1093F00035FD0A2404B90DE000BF4FF47A7505B9B4
:1094000004E0134EAF013846B04700BF601E041E93
:10941000F3D100BF00BF00BF00BF00BF00BFBFF35C
:109420004F8F00BF00BF00BF0A48006800F4E06033
:1094300009490843001D0749086000BF00BF00BF7D
:10944000BFF34F8F00BF00BF00BF00BF00BFFDE7ED
:10945000917D04000CED00E00000FA0510B500213C
:109460000C2016F0C8FF012017F09AFD00210D20F6
:1094700016F0C1FF012017F093FD01210C2016F01A
:10948000BAFF012017F08CFD00210C2016F0B3FF6D
:1094900010BD1CB50020009003460122114601902A
:1094A0000C2016F0D1FD0C2016F0C6FE0C2016F094
:1094B0002AFF0020009003460122114601900D2052
:1094C00016F0C2FD0D2016F0B7FE0D2016F01BFFA2
:1094D0001CBD10B500210C2016F08DFF01210D20C0
:1094E00016F089FF012017F05BFD01210C2016F01A
:1094F00082FF012017F054FD00210C2016F07BFFA5
:1095000010BD2DE9F04107460E4615469846002449
:1095100000F084F8384600F057F800F0AFF810B9C2
:109520000020BDE8F081304600F04EF800F0A6F8CB
:1095300008B90020F5E700F071F8791CC8B200F016
:1095400043F800F09BF808B90020EAE7002406E0A1
:1095500000F012F82855FFF781FF601CC4B2A8F193
:109560000100A042F4DC00F007F82855FFF7B1FF36
:1095700000F06CF80120D4E770B5002501210D2022
:1095800016F039FF00BF17E06006040E00210C2022
:1095900016F031FF052017F003FD01210C2016F015
:1095A0002AFF052017F0FCFC0D2016F094FE08B1F0
:1095B00044F00104681CC5B2082DE5DB00210C2035
:1095C00016F019FF204670BD70B50446002500BF97
:1095D0001DE000210C2016F00EFF052017F0E0FC26
:1095E00004F0800020B101210D2016F004FF03E0FB
:1095F00000210D2016F0FFFE6006040E01210C2054
:1096000016F0F9FE052017F0CBFC681CC5B2082D3A
:10961000DFDB00210C2016F0EEFE70BD10B501213D
:109620000D2016F0E8FE01210C2016F0E4FE0520C6
:1096300017F0B6FC00210D2016F0DDFE052017F016
:10964000AFFC00210C2016F0D6FE10BD10B5002195
:109650000C2016F0D0FE00210D2016F0CCFE0520C7
:1096600017F09EFC01210C2016F0C5FE01210D20F3
:1096700016F0C1FE052017F093FC10BD10B50024B4
:1096800001210D2016F0B7FE012017F089FC012101
:109690000C2016F0B0FE0BE0601CC0B2044632286D
:1096A00003DBFFF7D3FF002010BD012017F078FC8B
:1096B0000D2016F010FE0028EED100210C2016F02F
:1096C0009AFE0120F0E72DE9F04180460D4616464E
:1096D0001F460024FFF7A2FF4046FFF775FFFFF784
:1096E000CDFF10B90020BDE8F0812846FFF76CFFE0
:1096F000FFF7C4FF08B90020F5E7002409E0305D5A
:10970000FFF762FFFFF7BAFF08B90020EBE7601C24
:10971000C4B2BC42F3DBFFF799FF0120E3E700008E
:1097200010B50548007828B1044B054A054906489C
:1097300000F0DCF810BD00009847002019C10300BC
:10974000AC4700209C4700202277002001200149DF
:109750000870704798470020002001490870704742
:10976000984700202DE9FC4704460D4616461F4643
:10977000DDE90AA8DDF830904348007868B1534627
:109780003A4631462846CDE900891AF0F5FC3F49B2
:10979000A1F1480010F052F90CE053463A46314628
:1097A0002846CDE900890CF06FFB3849A1F148004B
:1097B0000CF01CFB35484838B0F84A00401C3349CF
:1097C0004839A1F84A00002C40D02F48007818B141
:1097D0002F481AF057FE54E02E4890F848302B4896
:1097E000483890F848102B4A0CF028FB2A49A1F180
:1097F00048000CF00FFB28484838B0F84A00401CDD
:1098000025494839A1F84A00084690F84A1090F8CE
:109810004800401C204A483A11541046B0F84A000B
:109820000012114691F8481050541146B1F84A0000
:1098300000EBD0714910A0EB410111BB104690F82C
:109840004830042100201CF08BFB1AE00F484838F8
:1098500090F84A1090F84800401C0C4A483A1154BD
:109860001046B0F84A000012114691F848105054C2
:10987000104690F84800801CC3B2042100201CF060
:109880006FFBBDE8FC87000098470020D2760020DF
:109890009C4700203E7600201E77002070B50446CD
:1098A0000D46E07804281AD16278211D0C48FCF797
:1098B000E7FD6078C01F0A4981F848006078801E83
:1098C000215C6078C01E205C41EA00200449A1F8B8
:1098D0004A000448007810B103481AF0D3FD70BD67
:1098E0003E76002098470020AC4700202DE9F0414B
:1098F00004460E4615461F466548007810B10128FB
:109900000CD10CE06889002808DD0120604908704E
:1099100028461AF037FF30461AF034FFB5E008E069
:1099200004F14C0128461AF0EDFDB4F896005949AF
:109930000880688971898842F2DC6889002867DDBF
:1099400004F14C0128461AF0DDFD52480088401C05
:1099500050490880B4F896000988884259D000BF61
:109960004D480088401C4C4908804A480088401CEB
:1099700048490880214630461AF0C4FDB4F84A0030
:109980004449098888423BD1214630461AF0BAFD45
:1099900094F8943094F8481004F14C022046B847EB
:1099A0003E49A1F1480010F05BF83C484838B0F857
:1099B0004A00401C39494839A1F84A00084690F845
:1099C0004A1090F84800401C344A483A1154104656
:1099D000B0F84A000012114691F848105054114650
:1099E000B1F84A0000EBD0714910A0EB410131B948
:1099F000104690F84830042100201CF0B1FA07E02E
:109A00007089002803DC00202149087000E0A7E7E6
:109A10003AE0214630461AF075FD94F8943094F8F7
:109A2000481004F14C022046B8471C49A1F14800F7
:109A300010F016F819484838B0F84A00401C174989
:109A40004839A1F84A00084690F84A1090F84800B2
:109A5000401C124A483A11541046B0F84A0000120D
:109A6000114691F8481050541146B1F84A0000EBE5
:109A7000D0714910A0EB410131B9104690F848303F
:109A8000042100201CF06CFA00BF00BFBDE8F0818B
:109A9000BC470020BE470020083F00201E77002062
:109AA00070B505460C46002026490860264800216E
:109AB00001604160816025480160416081604FF430
:109AC000A2712348FCF7F5FC2248002101604160A7
:109AD00081602148016041608160204801604160EF
:109AE000816024211E48FCF7E4FC24211D48FCF77A
:109AF000E0FC6C211C48FCF7DCFC4FF4A2711B4815
:109B0000FCF7D7FC24211A48FCF7D3FC2421194880
:109B1000FCF7CFFC24211248FCF7CBFC2421114890
:109B2000FCF7C7FC144890ED000A2146114812F0DA
:109B300073F924220F491148FCF7A2FC00201049B8
:109B4000086070BD34490020F481002000820020AC
:109B5000287E00206C7F0020DC810020E88100202E
:109B6000787F00209C7F0020C07F00202C80002078
:109B700070810020948100202C490020B8810020B1
:109B80005849002010B500210E2016F0FAFB0020E5
:109B9000024908700249087010BD0000D13F002042
:109BA000D03F002010B5012001F03CFE174CE368C7
:109BB000A2686168206801F03BFE1548008801F04A
:109BC00047FE00F057FF00231A466021114800F0BD
:109BD00055FF114908600E2016F0CDFA01210E2024
:109BE00016F0CFFB112016F0C6FA0021112016F056
:109BF000C8FB0A4A0AA10A2000F0E0FD0B4801F068
:109C00005BFE0B4803F09CFB10BD0000B43F00203E
:109C1000C43F0020D85E0020CC3F0020359C0200CD
:109C20004C45445F50726F636573730029520300A3
:109C30003B52030010B500242C48007810B10128D5
:109C400051D10AE02A48007830B101202749087034
:109C500001210E2016F095FB45E0264800780828E3
:109C60003BDA25482349097810F8310001280FD143
:109C70002149204A127801EBC201486803F062FAD8
:109C80001E48042102681E48006801F0E7FD24E038
:109C90001848047816E0184810F8340001280FD14D
:109CA00014480470144901EBC401486803F04AFAEF
:109CB0001248042102681248006801F0CFFD03E059
:109CC000601EC4B2002CE6DC00BF34B900210E20B7
:109CD00016F057FB0020074908700020044908705F
:109CE0000249087000BF00BF10BD0000D23F002035
:109CF000D03F0020D13F0020985F0020C83F0020C7
:109D0000CC3F0020082800DB70470122084B03F8F5
:109D100030201A4602EBC0025160064A1278904287
:109D200004DB044A10700122034B1A7000BFEBE7FA
:109D3000985F0020D13F0020D03F0020082800DBA2
:109D400070470021084A02F830104FF07F4102EBC3
:109D5000C002516005490978884202DB0121044AAA
:109D6000117000BFECE70000985F0020D13F002099
:109D7000D03F002010B50021082016F051FB012033
:109D800017F01AF90021072016F04AFB012017F0FE
:109D900013F90121082016F043FB012017F00CF9FC
:109DA0000021082016F03CFB10BD1CB500200090DF
:109DB0000346012211460190082016F059F90820A7
:109DC00016F049FA082016F0A9FA00200090034680
:109DD000012211460190072016F04AF9072016F0DB
:109DE0003AFA072016F09AFA092016F0E8F901214C
:109DF000092016F015FB062016F0E1F91CBD10B580
:109E00000021082016F00CFB0121072016F008FBAA
:109E1000012017F0D1F80121082016F001FB0120E4
:109E200017F0CAF80021082016F0FAFA10BD2DE943
:109E3000F04107460E4615469846002400F084F887
:109E4000384600F057F800F0BDF810B90020BDE822
:109E5000F081304600F04EF800F0B4F808B9002068
:109E6000F5E700F071F8791CC8B200F043F800F093
:109E7000A9F808B90020EAE7002406E000F012F88B
:109E80002855FFF777FF601CC4B2A8F10100A0427B
:109E9000F4DC00F007F82855FFF7B1FF00F06CF88C
:109EA0000120D4E770B500250121072016F0B8FA8B
:109EB00000BF17E06006040E0021082016F0B0FA7B
:109EC000052017F079F80121082016F0A9FA0520DD
:109ED00017F072F8072016F00AFA08B144F00104EE
:109EE000681CC5B2082DE5DB0021082016F098FAA1
:109EF000204670BD70B50446002500BF1DE000215E
:109F0000082016F08DFA052017F056F804F08000AE
:109F100020B10121072016F083FA03E00021072079
:109F200016F07EFA6006040E0121082016F078FA79
:109F3000052017F041F8681CC5B2082DDFDB0021B1
:109F4000082016F06DFA70BD10B50121072016F03B
:109F500067FA0121082016F063FA052017F02CF8A3
:109F60000021072016F05CFA052017F025F80021E3
:109F7000082016F055FA10BD10B50021082016F083
:109F80004FFA0021072016F04BFA052017F014F8BD
:109F90000121082016F044FA0121072016F040FAAA
:109FA000052017F009F810BD10B5082016F0C0F80C
:109FB000072016F0BDF8092016F0BAF8062016F0B2
:109FC000B7F810BD10B500240121072016F028FABB
:109FD000012016F0F1FF0121082016F021FA0BE014
:109FE000601CC0B20446322803DBFFF7C5FF002027
:109FF00010BD012016F0E0FF072016F078F90028C8
:10A00000EED10021082016F00BFA0120F0E72DE92F
:10A01000F04180460D4616461F460024FFF794FF88
:10A020004046FFF767FFFFF7CDFF10B90020BDE8FE
:10A03000F0812846FFF75EFFFFF7C4FF08B9002054
:10A04000F5E7002409E0305DFFF754FFFFF7BAFFA2
:10A0500008B90020EBE7601CC4B2BC42F3DBFFF799
:10A060008BFF0120E3E700007CB5002511F04EFCDA
:10A070004042C6B20D48058800242A122146641CBD
:10A080000DF80120EAB22146641C0DF8012021469A
:10A09000641C0DF8016023466A4603210020FDF789
:10A0A00077F90020014908807CBD0000083F0020AE
:10A0B0002DE9F041022001210A46002423462546CD
:10A0C00000BF4FF0A0473E4641EA420747EA8407F7
:10A0D00047EA032747EA054C06F5E06747F820C042
:10A0E00000BF00BF002116F02FF9642000F01AF81D
:10A0F000064802F0B3FB064A06A1002000F05EFB12
:10A100000749A420FDF76EF8BDE8F08165A10200C3
:10A11000A9A102004D545F70726F636573730000F4
:10A12000554E030010B50446224608A1002001F058
:10A13000E5F84CB1094804600121022016F004F949
:10A140000121074800F016FB10BD00004D54204DC2
:10A15000545F52756E3A2564200A0000A83F002023
:10A16000A9A1020010B504460D480068B0B10C4822
:10A17000006828B10A480068401E0949086002E0EA
:10A180000020074908600648006838B9002102200D
:10A1900016F0DAF80021034800F0ECFA10BD0000D8
:10A1A000A83F0020A9A102007047000010B54FF49D
:10A1B000807015F09CFC80B14FF4807015F0A0FC0D
:10A1C000012015F0A7FC2048407930B901201E4934
:10A1D000487108460168002088474FF4827015F0E6
:10A1E00086FC50B14FF4827015F08AFC022015F005
:10A1F00091FC15480168012088474FF4887015F0DC
:10A2000076FC50B14FF4887015F07AFC102015F0F0
:10A2100081FC0D480168022088474FF4867015F0D4
:10A2200066FC80B10020094908604FF4867015F083
:10A2300067FC082015F06EFC002003498871084671
:10A2400001680320884710BD5C4A0020340C0040A0
:10A250002DE9F0411DF04CFA0EF044FB15210320CE
:10A26000002213461446154600BF0F073E4642EA39
:10A27000430747EA800747EA042747EA054C06F503
:10A28000E06747F821C000BF00BF00F017F8FFF7F4
:10A2900089FCFFF70DFFFEF77FFAFDF7DDFE1DF0ED
:10A2A00063F9BDE8F081000010B50249024812F0E0
:10A2B00021FC10BD6C4A002000C0014010B5034ACB
:10A2C00003A142F2107000F079FA10BDC5A302009C
:10A2D0005057525F50726F63657373002DE9F04100
:10A2E0001321084602F012FDFFF74CFC002108463E
:10A2F00010F0B0FE0021012010F0ACFE0021022081
:10A3000010F0A8FE0021032010F0A4FE002104207C
:10A3100010F0A0FE0DF046F80DF078FC02200021B0
:10A3200061B900BF00BF4FF0A0421346012505FAF6
:10A3300000F2C3F80C2500BF00BF0CE000BF00BF57
:10A340004FF0A0421346012505FA00F2C3F8082594
:10A3500000BF00BF00BF00BFC82015F005FC1920DA
:10A360000021022200231D461E4600BF4FF0A04CD4
:10A37000674643EA450C4CEA810C4CEA062C4CEA51
:10A38000024C07F5E06848F820C000BF00BF33DF8B
:10A390000446FEF7D9FF054623462A4602A10020BF
:10A3A00000F0ACFFBDE8F081706F776572206F66DA
:10A3B000662E2E2E4241543A25642C4552523A259F
:10A3C000640A000010B5FEF7BFFF002830D105F089
:10A3D00059FB01282CD1FEF7B7FF0446224615A1F0
:10A3E000002000F08BFF18A1002000F087FFFEF78F
:10A3F0001DFE18B118A10D20FDF7F2FDFEF7AEFC11
:10A4000018B119A10D20FDF7EBFD4FF47A70FFF79D
:10A4100089FE0EF067FA002406E005F029FD6420AD
:10A4200015F0A2FB601CC4B20A2CF6DBFFF756FF46
:10A4300010BD000042617474657279506572736575
:10A440006E743A25640A0000706F776572206F663B
:10A45000662E2E2E0A0000007361766520737465E7
:10A4600070206661696C00007361766520696E66B4
:10A470006F726D6174696F6E206661696C000000B7
:10A4800010B52DED048BF0EE408AB0EE608A9FEDA2
:10A49000860AB0EE409A9FED850AF0EE409A844815
:10A4A000007820B101281FD002281CD16DE0B3EE46
:10A4B000040AB4EEC08AF1EE10FA0ADD02207C49EB
:10A4C0000870B0EE680A0BF0BBF97A4880ED000A1C
:10A4D00009E0B0EE680A02F0BBFD764880ED000AA4
:10A4E000012073490870D7E0B3EE040AB4EEC08AC5
:10A4F000F1EE10FA20DD02206D4908709FED6A0A26
:10A500006D4880ED000A9FED6D0AF4EEC08AF1EE11
:10A5100010FA39D2674890ED000ADFED690AB4EE0F
:10A52000E00AF1EE10FA2FDDB0EE680A0BF088F9C0
:10A53000604880ED000A27E0B0EE680A02F088FD6E
:10A54000604880ED000A5B4890ED000A5D48D0ED60
:10A55000000AB4EEE00AF1EE10FA04DD90ED000A14
:10A56000544880ED000A0BF0C5F968B1514890EDF0
:10A57000000ADFED530AB4EEE00AF1EE10FA03DD53
:10A580009FED510A80ED000A86E0B3EE040AB4EEB6
:10A59000C08AF1EE10FA18D2012045490870B2EED7
:10A5A000040AC8EE800A4948C0ED000A414890ED0F
:10A5B000000ADFED470AB4EEE00AF1EE10FA6ADDB8
:10A5C0009FED410A80ED000A65E0F0EE690A394826
:10A5D00090ED000A13F07EFD3E4880ED000AF7EE94
:10A5E000000AB0EE480AFDF7FDF9F0EE690A3948B5
:10A5F00090ED000A02F020FDB0EE409AB0EE680A3D
:10A600000BF01EF92F4880ED000A9FED330AC8EECB
:10A61000000A2948C0ED000A90ED000AF7EE000A92
:10A62000B4EEE00AF1EE10FA03DDB7EE000A80EDB9
:10A63000000A214890ED000AF7EE000A30EEC00A49
:10A640002048D0ED000A20EE200A1B48D0ED000A79
:10A6500000EE890A1B4880ED000A164890ED000ABA
:10A660001848D0ED000AB4EEE00AF1EE10FA04D278
:10A6700090ED000A0F4880ED000A0E4890ED000AA8
:10A68000DFED110AB4EEE00AF1EE10FA03DD9FED02
:10A69000130A80ED000A00BF00BF064890ED000AD3
:10A6A000BDEC048B10BD0000000000000000AF43B3
:10A6B0000C400020004000201040002000007A459F
:10A6C0000000BE42044000200000C842F03F0020CD
:10A6D0003333C6420840002000007A44CDCCC74244
:10A6E00070B50025002400BF39E02046FDF73CFB93
:10A6F0001E4800EB0410007B00B92EE01B4800EB65
:10A700000410806810B3194800EB0410408828B981
:10A71000164901EB04118868804717E002F03AF807
:10A72000124901EB04114968401A104901EB041168
:10A73000498888420AD302F02DF80C4901EB041134
:10A7400048600A4901EB041188688047074800EB1C
:10A750000410007800B1012500BF601CC4B2044899
:10A7600000888442C1DB284670BD0000544B0020A5
:10A77000D63D002010B50246002014E00D4B03EB3F
:10A7800000139B6893420CD10A4B03EB00131B7818
:10A790008B4205D001F00103064C04EB001423703A
:10A7A00010BD431CD8B2044B1B889842E6DB00BFA7
:10A7B000F6E70000544B0020D63D00202DE9F04183
:10A7C00005460F461646002419E0234800EB041006
:10A7D0008068B04211D101201F4901EB04110873B8
:10A7E0001D4800EB0410458001F0D4FF1A4901EB2D
:10A7F000041148600120BDE8F081601CC4B2174814
:10A8000000888442E1DB154800883C2802DB4FF0D9
:10A81000FF30F0E710481149098800EB011086600D
:10A8200001210D480D4A128800EB021001730A48FD
:10A830000A49098800EB0110458001F0ABFF064989
:10A84000064A128801EB0211486004480088401C47
:10A85000024908800020CEE7544B0020D63D00205E
:10A86000014600200DE00A4A02EB001292688A427B
:10A8700005D10022064B03EB00131A737047421CEC
:10A88000D0B2044A12889042EDDB00BFF6E7000028
:10A89000544B0020D63D0020024600200CE0094B1E
:10A8A00003EB00139B68934204D1064B03EB0013A8
:10A8B00059807047431CD8B2034B1B889842EEDB8B
:10A8C00000BFF6E7544B0020D63D00202DE9F041B3
:10A8D00005460320FDF7ACF80746052D01DABDE873
:10A8E000F081002426E0174800EB04100078B842FD
:10A8F0001FD1144800EB0410C068D0B1002609E055
:10A90000311D88B2FDF794F80E4901EB0411496836
:10A910008855761C681FB042F2DC0A4901EB04112D
:10A920000872084A02EB041002EB0412D16888474F
:10A9300004E0641C044800688442D4D300BF00BF14
:10A94000CDE70000985600207C3F0020F0B5C1B054
:10A9500005460320FDF77CF80746052F12DA002490
:10A9600006E0211D88B2FDF773F801A90855641CA3
:10A97000681FA042F5DCC3B201AA39460020FCF7EB
:10A98000E3FE00BF052D01DA41B0F0BD002426E052
:10A99000164800EB04100078B8421FD1134800EBB2
:10A9A0000410C068D0B1002609E0311D88B2FDF75F
:10A9B0004FF80E4901EB041149688855761C681F51
:10A9C000B042F2DC094901EB04110872074A02EBBC
:10A9D000041002EB0412D168884704E0641C0448A8
:10A9E00000688442D4D300BF00BFCDE7A85C00203C
:10A9F000983F00202DE9F04105460320FDF738F887
:10AA00000746052D01DABDE8F081002426E017484D
:10AA100000EB04100078B8421FD1144800EB04107A
:10AA2000C068D0B1002609E0311D88B2FDF720F8DA
:10AA30000E4901EB041149688855761C681FB04225
:10AA4000F2DC0A4901EB04110872084A02EB041017
:10AA500002EB0412D168884704E0641C04480068D3
:10AA60008442D4D300BF00BFCDE70000D8630020EC
:10AA7000E43F002010B500F025F810BD2DE9F041AD
:10AA800007460C4615461E460848807A30B100201D
:10AA900000F0D8FE00F00EF8FFF7ECFF0448076066
:10AAA00084808560C660BDE8F08100006C400020B5
:10AAB000486D002010B5024816F00EFC10BD0000D5
:10AAC0006440002070B5002508480949026809481B
:10AAD00016F036FB044604B16D1E681C20B9064A08
:10AAE00006A10020FFF76AFE70BD0000784000203C
:10AAF0006C40002064400020A53F03006273705F3B
:10AB000070776D5F696E69745F70726F6365737380
:10AB10000000000010B5034A1068034A1168884716
:10AB200010BD0000E84A0020E44A002010B50422CD
:10AB30000021024811F082FF10BD000000400240D9
:10AB400070B506460C4615462B4622460021304677
:10AB5000FEF748FB70BD70B504460D461646B4F5C9
:10AB6000F02F02D8B4F5E82F01D2022070BD324692
:10AB700021462846FBF784FC0020F7E710B514486F
:10AB80000FF012F900201349087701F003FE114974
:10AB90008861002008700AF0E4FE4FF07F41062033
:10ABA000FFF7B0F80620FFF7C9F80121022010F0E6
:10ABB00051FA08480021816081810020064908700F
:10ABC000084604F041FF05A1002000F097FB10BDEE
:10ABD0002C3F0020E85100203C3F00206170705F56
:10ABE00073656C665F636865636B696E675F5072FF
:10ABF0006F6365737320636C6561725F616C6C5F1A
:10AC00006578636570740D0A000000002DE9F04757
:10AC10002DED068B86B005460E4617464FF0000810
:10AC2000C146C246002005E035F9101003AA42F8DB
:10AC30002010401C0328F7DB0598002801DB0146A3
:10AC400000E041428846002004E036F910104DF83B
:10AC50002010401C0328F8DB0298002801DB014685
:10AC600000E041428946EE48007803280CDBED48BD
:10AC70004068EC4908600846806848600220E8495E
:10AC800008700120E8490860E54801780078401C18
:10AC9000E34A1070E34840F82180E4480078032834
:10ACA0000CDBE3484068E249086008468068486079
:10ACB0000220DE4908700120DB490860DB4801788A
:10ACC0000078401CD94A1070D94840F82190D948E2
:10ACD000007803280CDBD8484088D749088008460C
:10ACE000808848800220D34908700120CE4908603E
:10ACF000B888404201B2CF4802780078401CCD4B62
:10AD00001870CD4820F81210C748006801287DD17E
:10AD1000C4488068C3494968401A12D4C7480088AB
:10AD200020B9C0488068C649086011E0BD48806805
:10AD3000C349096888420BDDBA488068C049086089
:10AD400006E0BE48008818B9B6488068BD4908606A
:10AD5000B7488068B6494968401A12D4BA48008892
:10AD600020B9B3488068B949086011E0B0488068EC
:10AD7000B649096888420BDDAD488068B349086070
:10AD800006E0B148008818B9A9488068B049086051
:10AD9000A4488068AB490968401A40F69801884287
:10ADA00012DD0120A54908809E488068A5490968F0
:10ADB000401AA8490968884206DD9A488068A14976
:10ADC0000968401AA349086099488068A049096841
:10ADD000401A40F69801884212DD01209A49088005
:10ADE000934880689A490968401A9B4909688842D3
:10ADF00006DD8F48806896490968401A96490860C0
:10AE0000884880688F490968401A00E0EEE040F207
:10AE1000DC51884228DD8F480068FBF708FD41ECD3
:10AE20001A0B9FED8E0B53EC102BFBF71FFC41EC24
:10AE3000180B7C498968824A1268501AFBF7F7FCA4
:10AE400041EC190B53EC182BFBF75AFD13D2754844
:10AE5000806874494968441A002C01DB204600E0F0
:10AE60006042B0F5C87F06DA00207449088040F6D9
:10AE70009800784908606E48806875490968401AEA
:10AE800040F2DC51884228DD73480068FBF7CFFCB4
:10AE900041EC1A0B9FED710B53EC102BFBF7E6FB0B
:10AEA00041EC180B62498968684A1268501AFBF72E
:10AEB000BEFC41EC190B53EC182BFBF721FD13D210
:10AEC0005B4880685A494968441A002C01DB2046D7
:10AED00000E06042B0F5C87F06DA00205A490880D9
:10AEE00040F698005C4908605648006810B9002098
:10AEF000524908805648006810B90020524908801D
:10AF00005848008838BB5848B0F90000B0F5967F23
:10AF100005DA55480088401C00B2534908800020DB
:10AF20005249088045480088012803D046480088D7
:10AF300001280AD14C48B0F90000082805DB4FF081
:10AF4000010A01204749088062E04FF0000A002012
:10AF5000444908805CE04FF0000A4448B0F9000022
:10AF6000B0F5967F05DA41480088401C00B23F49A1
:10AF7000088000203C4908803C4BB3F90030062B88
:10AF800030DB2E4B1B886BBB2B4BB3F90030A3F58A
:10AF9000FA62002A01DB134600E05342B3F5967FC4
:10AFA00019DC254BB3F90230A3F5FA61002901DB66
:10AFB0000B4600E04B42B3F5967F0CDC1E4BB3F919
:10AFC0000430A3F5FA60002801DB034600E04342A9
:10AFD000B3F5967F06DD1C4B1B881BB90020214969
:10AFE000088015E001201F49088011E04FF0000A99
:10AFF0000C488068134908600A4880681049086056
:10B000000B48806812490860094880680F49086049
:10B010000AF0FF0006B0BDEC068BBDE8F08700002B
:10B02000AC49002020850020B8490020AD4900200F
:10B030002C850020B4490020BC49002096490020FE
:10B04000A04900209C49002098490020A8490020E0
:10B05000A4490020C4490020C84900209A99999920
:10B060009999D93FB2490020B0490020AE4900204B
:10B07000FEB54FF4827015F0CBFC002837D04FF4AA
:10B08000827015F0CFFC6C4890F82E0018B16A4819
:10B0900090F82F0058B300208DF8000066484068F3
:10B0A000019065480189ADF80810C06818B9002002
:10B0B0006149087412E06048008B5F494883084684
:10B0C000C06848600846008B08810020C8600846B8
:10B0D00090F82E0010B9002015F0C6FC5648016803
:10B0E000684688470020544981F82F0000BF524825
:10B0F00090F82E00002852D04FF4807015F088FC94
:10B1000000284CD04FF4807015F08CFC4A48408BDE
:10B11000494991F82D10884216DD4748408B464931
:10B1200091F82D10401A444948830A4612890B466B
:10B130005B8BD21A0B465B6803EB42000A4692F81F
:10B140002D1015F051FC23E03B48408B3A4991F813
:10B150002D1088420FD13848C06860B101203649AF
:10B1600081F82F00002048830A4692F82D10D068FD
:10B1700015F03AFC0CE03048408B2F4991F82D1027
:10B18000884205D101202C4981F82F0000204883F6
:10B190004FF4827015F046FC042015F065FC4FF466
:10B1A000887015F035FC70B14FF4887015F03AFCDA
:10B1B00000202149087402208DF80000084601682B
:10B1C0006846884700BF4FF48A7015F021FC38B1FB
:10B1D0004FF48A7015F026FC0020174908742AE005
:10B1E0001548456924E0B5FA85F64FF00040F04077
:10B1F0008543B00000F58C74204615F009FCB8B109
:10B20000204615F00FFC01208DF80000A4F58C708D
:10B21000C0F3C7008DF80400A4F58C70012121EA69
:10B2200090018DF80510044801686846884700BF02
:10B23000002DD8D100BFFEBD7C890020F8B50446A2
:10B240000D46164600BF0B48007808B902F090FA88
:10B2500000BF00200090684607F0A5F93246294655
:10B26000204600F009F807469DF8000007F0A2F913
:10B270003846F8BD508C00202DE9F0470746884637
:10B280001646C24607EB47011B4800EBC109D9F837
:10B29000140020B1012811D0022826D11EE0484612
:10B2A00002F09EFA0546B54201D2002405E034467C
:10B2B00032465146484602F0EAFB18E0484602F0A2
:10B2C0008FFA0546B54201D2284600E030460446D2
:10B2D00022465146484602F0DAFB08E03246514623
:10B2E000484602F099FB044601E0002400BF00BF7D
:10B2F0002046BDE8F0870000688C00200FB438B508
:10B30000044606A800906A462046059900F007F812
:10B31000054600200090284638BC5DF814FB2DE956
:10B32000F04F99B082460D46144603A81490402071
:10B33000159000201690CDF860A0179000BF2E78D1
:10B340006D1C06B9DDE0252E79D100274FF00109EB
:10B3500000BF2E78232E12D02B2E0CD02D2E02D0F3
:10B36000302E10D103E047F001076D1C0EE047F0CE
:10B3700002076D1C0AE047F004076D1C06E047F069
:10B3800008076D1C02E04FF0000900BF00BFB9F1D3
:10B39000000FDED14FF0000800BF2E78302E01DB09
:10B3A000392E00DD07E06D1CA6F1300008EB8801A6
:10B3B00000EB4108F1E700BF002013902E782E2EFD
:10B3C00012D16D1C00BF2E78302E01DB392E00DD2E
:10B3D00009E06D1CA6F13000139901EB810100EB2F
:10B3E00041001390EFE700BF2E7800BF6C2E01D014
:10B3F000682E02D16D1C2E7800E000E0F6E700BF59
:10B40000702E5DD008DC252E6AD0582E35D0632EE4
:10B4100009D0642E69D113E0732E3CD0752E1DD057
:10B42000782E62D128E02168081D2060D1F80090B4
:10B4300009F0FF0B594614A802F0CCFA56E058E088
:10B440002168081D2060D1F80090CDE900870A220C
:10B45000494614A8139B02F0D1F947E02168081D62
:10B460002060D1F80090CDE900870A22494614A84F
:10B47000139B02F039FA39E000BF2168081D2060F3
:10B48000D1F80090CDE900871022494614A8139BFB
:10B4900002F02AFA2AE02168081D2060D1F800B0E5
:10B4A00000BF9BF800600BF1010B06B906E03146C6
:10B4B00014A802F08FFA17980028F2DA00BF15E0FE
:10B4C0002168081D2060D1F80090002008210B465B
:10B4D0001022CDE90010494614A802F005FA05E053
:10B4E000252114A802F076FA00E000BF00BF6D1C11
:10B4F00003E0314614A802F06DFA17980028BFF651
:10B500001EAF00BF179800280ADD169820B103A9C6
:10B510005046169AFFF792FEDDE916100844179080
:10B52000179819B0BDE8F08F0246002106E00548E3
:10B53000405C904201D100207047491C0029F6D0A0
:10B540000220F9E7D880040070B505460C4628466D
:10B55000FFF7EAFF061E01D0304670BD012C04D172
:10B560000121284614F02AFF04E01CB900212846D6
:10B5700014F024FF0020F0E710B5002409E00D4985
:10B58000085D0121FFF7E0FF0A49085D14F0C4FDE2
:10B59000641C002CF3D0084814F0D7FB062014F0EC
:10B5A000BBFD072014F0B8FD082014F0B5FD002005
:10B5B00010BD0000D8800400A88004007FB50025DD
:10B5C000174B0FCB8DE80F0006208DF802000720E7
:10B5D0008DF8010008208DF8000000208DF80C0087
:10B5E0004FF00040029006208DF8040000230D4A21
:10B5F00069460D4814F04CFB064606B16D1E00244A
:10B6000004E00A49085D14F0CEFD641C002CF8D05B
:10B61000681C20B9064A07A10020FFF7CFF87FBDBC
:10B62000DC800400E96F0400A8800400D8800400D6
:10B63000354003006273705F737069305F696E69D3
:10B64000745F70726F63657373000000F8B506462F
:10B650000F4614461D4623460022394630460095C3
:10B6600000F050F8F8BDF8B506460F4614461D46E2
:10B670002346012239463046009500F043F8F8BDD4
:10B680002DE9F84F05460E4617469846DDF82890F6
:10B690004FF0030A2846FFF747FF041E02D020465A
:10B6A000BDE8F88F00212846FFF74EFF0020134920
:10B6B000087043463A4631461148CDF8009014F0E0
:10B6C0002BFB04460CB10120EAE70DE0BAF10000C3
:10B6D000AAF1010A02D014F0E7FF05E00121284693
:10B6E000FFF732FF0120DBE7044800780028EDD0A7
:10B6F00001212846FFF728FF0020D1E7C84000209D
:10B70000A88004002DE9FC4781460D4690461E4660
:10B710000A9C4846FFF708FF071E02D03846BDE8DE
:10B72000FC87812C01D90320F9E7B8F1000F16D16D
:10B7300045F080000190601CC0B2144B012201A9A9
:10B7400000904846FFF79CFF07460FB13846E6E7F2
:10B7500022460E49491C3046FAF792FE13E00B4888
:10B76000057022463146401CFAF78AFE0020009000
:10B77000601CC2B2002305494846FFF781FF074617
:10B780000FB13846CBE70020C9E70000B06D0020BC
:10B7900010B50249024811F0FFF910BDC48900201C
:10B7A0000030004010B503494FF0402011F0F4F98B
:10B7B00010BD0000E889002010B50249024811F0D0
:10B7C000EBF910BD0C8A00200030024070B50A4829
:10B7D00014F063F9044600BF254635B100BF07A247
:10B7E00063212846FAF716FD00BF00BF0CB1062002
:10B7F00070BD0020FCE70000B87300202E2E5C2EE8
:10B800002E5C2E2E5C626C655F6366675C686F738E
:10B81000742E630010B514F068F910BD10B515F062
:10B8200077FA10BD01494871704700006C40002054
:10B8300030B5034D28706970AA70EB7030BD000000
:10B840006C40002001498872704700006C40002065
:10B8500001490881704700006C40002070B5044623
:10B860000D46164633462A462146024815F0F2FC9C
:10B8700070BD00006440002001480078704700005F
:10B880005541002010B500240AE0084850F8240073
:10B8900028B1064850F82410054800688847641C01
:10B8A000044800788442F0DB10BD0000284B0020E3
:10B8B000D03D0020D43D002010B50446002116E004
:10B8C0000F4850F82100A04202D14FF0FF3010BDC8
:10B8D0000B4850F8210048B90A480078401C094A32
:10B8E0001070074840F821400020F0E7491C052966
:10B8F000E6DB05A10020FFF701FD6FF00100E6E7A0
:10B90000284B0020D43D0020536C6565705F526564
:10B910006769737420746F6F206D616E79210A00FE
:10B9200002460020002100BF27E0411C22E000EB7E
:10B93000C0030B4402EB8303D3ED000A01EBC10308
:10B94000034402EB830393ED001A70EE810AB6EE16
:10B95000001A20EE810A00EBC0030B4402EB8303C4
:10B9600083ED000A01EBC103034402EB830383ED83
:10B97000000A491C0929DADB401C0928D5DB70477D
:10B9800090ED031AD0ED061A01EE801A80ED031A2D
:10B9900090ED041AD0ED071A01EE801A80ED041A1A
:10B9A00090ED051AD0ED081A01EE801A80ED051A07
:10B9B00090ED0C1AD0ED0F1A01EE801A80ED0C1AE2
:10B9C00090ED0D1AD0ED101A01EE801A80ED0D1ACF
:10B9D00090ED0E1AD0ED111A01EE801A80ED0E1ABC
:10B9E00090ED151AD0ED181A01EE801A80ED151A97
:10B9F00090ED161AD0ED191A01EE801A80ED161A84
:10BA000090ED171AD0ED1A1A01EE801A80ED171A70
:10BA100090ED1B1AD0ED361A01EE801A80ED1B1A3C
:10BA200090ED1C1AD0ED371A01EE801A80ED1C1A29
:10BA300090ED1D1AD0ED381A01EE801A80ED1D1A16
:10BA400090ED241AD0ED3F1A01EE801A80ED241AF1
:10BA500090ED251AD0ED401A01EE801A80ED251ADE
:10BA600090ED261AD0ED411A01EE801A80ED261ACB
:10BA700090ED2D1AD0ED481A01EE801A80ED2D1AA6
:10BA800090ED2E1AD0ED491A01EE801A80ED2E1A93
:10BA900090ED2F1AD0ED4A1A01EE801A80ED2F1A80
:10BAA00090ED1E1AD0ED391A01EE801AD0ED211A50
:10BAB00090ED3C2A42EE001A00EE211A80ED1E1A8B
:10BAC00090ED1F1AD0ED3A1A01EE801AD0ED221A2D
:10BAD00090ED3D2A42EE001A00EE211A80ED1F1A69
:10BAE00090ED201AD0ED3B1A01EE801AD0ED231A0A
:10BAF00090ED3E2A42EE001A00EE211A80ED201A47
:10BB000090ED271AD0ED421A01EE801AD0ED2A1AD4
:10BB100090ED452A42EE001A00EE211A80ED271A18
:10BB200090ED281AD0ED431A01EE801AD0ED2B1AB1
:10BB300090ED462A42EE001A00EE211A80ED281AF6
:10BB400090ED291AD0ED441A01EE801AD0ED2C1A8E
:10BB500090ED472A42EE001A00EE211A80ED291AD4
:10BB600090ED301AD0ED4B1A01EE801AD0ED331A59
:10BB700090ED4E2A42EE001A00EE211A80ED301AA6
:10BB800090ED311AD0ED4C1A01EE801AD0ED341A36
:10BB900090ED4F2A42EE001A00EE211A80ED311A84
:10BBA00090ED321AD0ED4D1A01EE801AD0ED351A13
:10BBB00090ED502A42EE001A00EE211A80ED321A62
:10BBC00090ED211AD0ED3C1A01EE801AD1ED021A47
:10BBD00061EE801A90ED1C2A01EE821AD1ED011A55
:10BBE00061EE801A90ED1D2A01EEC21A80ED211A35
:10BBF00090ED221AD0ED3D1A01EE801AD1ED021A15
:10BC000061EE801A90ED1B2A01EEC21AD1ED001AE6
:10BC100061EE801A90ED1D2A01EE821A80ED221A43
:10BC200090ED231AD0ED3E1A01EE801AD1ED011AE3
:10BC300061EE801A90ED1B2A01EE821AD1ED001AF6
:10BC400061EE801A90ED1C2A01EEC21A80ED231AD3
:10BC500090ED2A1AD0ED451A01EE801AD1ED021AA4
:10BC600061EE801A90ED252A01EE821AD1ED011ABB
:10BC700061EE801A90ED262A01EEC21A80ED2A1A92
:10BC800090ED2B1AD0ED461A01EE801AD1ED021A72
:10BC900061EE801A90ED242A01EEC21AD1ED001A4D
:10BCA00061EE801A90ED262A01EE821A80ED2B1AA1
:10BCB00090ED2C1AD0ED471A01EE801AD1ED011A41
:10BCC00061EE801A90ED242A01EE821AD1ED001A5D
:10BCD00061EE801A90ED252A01EEC21A80ED2C1A31
:10BCE00090ED331AD0ED4E1A01EE801AD1ED021A02
:10BCF00061EE801A90ED2E2A01EE821AD1ED011A22
:10BD000061EE801A90ED2F2A01EEC21A80ED331AEF
:10BD100090ED341AD0ED4F1A01EE801AD1ED021ACF
:10BD200061EE801A90ED2D2A01EEC21AD1ED001AB3
:10BD300061EE801A90ED2F2A01EE821A80ED341AFE
:10BD400090ED351AD0ED501A01EE801AD1ED011A9E
:10BD500061EE801A90ED2D2A01EE821AD1ED001AC3
:10BD600061EE801A90ED2E2A01EEC21A80ED351A8E
:10BD700090ED091AD1ED021A61EE211A90ED361AF2
:10BD800001EE801AD0ED121A91ED012A61EE821AAD
:10BD900001EEC01A80ED361A90ED0A1AD1ED021AA2
:10BDA00061EE211A90ED371A01EE801AD0ED131AC8
:10BDB00091ED012A61EE821A01EEC01A80ED371A68
:10BDC00090ED0B1AD1ED021A61EE211A90ED381A9E
:10BDD00001EE801AD0ED141A91ED012A61EE821A5B
:10BDE00001EEC01A80ED381A90ED001AD1ED021A5A
:10BDF00061EE211A90ED3F1A01EEC01AD0ED121A31
:10BE000091ED002A61EE821A01EE801A80ED3F1A50
:10BE100090ED011AD1ED021A61EE211A90ED401A4F
:10BE200001EEC01AD0ED131A91ED002A61EE821ACC
:10BE300001EE801A80ED401A90ED021AD1ED021A3F
:10BE400061EE211A90ED411A01EEC01AD0ED141ADC
:10BE500091ED002A61EE821A01EE801A80ED411AFE
:10BE600090ED001AD1ED011A61EE211A90ED481AF9
:10BE700001EE801AD0ED091A91ED002A61EE821AC6
:10BE800001EEC01A80ED481A90ED011AD1ED011AA9
:10BE900061EE211A90ED491A01EE801AD0ED0A1ACE
:10BEA00091ED002A61EE821A01EEC01A80ED491A66
:10BEB00090ED021AD1ED011A61EE211A90ED4A1AA5
:10BEC00001EE801AD0ED0B1A91ED002A61EE821A74
:10BED00001EEC01A80ED4A1A90ED391AD0ED3C1AE5
:10BEE00000EE211AD0ED0C1A91ED022A61EE821AB1
:10BEF00001EE801AD0ED151A91ED012A61EE821A39
:10BF000001EEC01A80ED391A90ED3A1AD0ED3D1AC3
:10BF100000EE211AD0ED0D1A91ED022A61EE821A7F
:10BF200001EE801AD0ED161A91ED012A61EE821A07
:10BF300001EEC01A80ED3A1A90ED3B1AD0ED3E1A90
:10BF400000EE211AD0ED0E1A91ED022A61EE821A4E
:10BF500001EE801AD0ED171A91ED012A61EE821AD6
:10BF600001EEC01A80ED3B1A90ED421AD0ED451A51
:10BF700000EE211AD0ED031A91ED022A61EE821A29
:10BF800001EEC01AD0ED151A91ED002A61EE821A69
:10BF900001EE801A80ED421A90ED431AD0ED461A58
:10BFA00000EE211AD0ED041A91ED022A61EE821AF8
:10BFB00001EEC01AD0ED161A91ED002A61EE821A38
:10BFC00001EE801A80ED431A90ED441AD0ED471A25
:10BFD00000EE211AD0ED051A91ED022A61EE821AC7
:10BFE00001EEC01AD0ED171A91ED002A61EE821A07
:10BFF00001EE801A80ED441A90ED4B1AD0ED4E1AE6
:10C0000000EE211AD0ED031A91ED012A61EE821A99
:10C0100001EE801AD0ED0C1A91ED002A61EE821A21
:10C0200001EEC01A80ED4B1A90ED4C1AD0ED4F1A6C
:10C0300000EE211AD0ED041A91ED012A61EE821A68
:10C0400001EE801AD0ED0D1A91ED002A61EE821AF0
:10C0500001EEC01A80ED4C1A90ED4D1AD0ED501A39
:10C0600000EE211AD0ED051A91ED012A61EE821A37
:10C0700001EE801AD0ED0E1A91ED002A61EE821ABF
:10C0800001EEC01A80ED4D1A90ED0F1AD1ED021A93
:10C0900061EE211A90ED3C1A01EE801AD0ED181ACB
:10C0A00091ED012A61EE821A01EEC01AD1ED021A59
:10C0B00061EE801A90ED372A01EE821AD1ED011A55
:10C0C00061EE801A90ED382A01EEC21A80ED3C1A1A
:10C0D00090ED101AD1ED021A61EE211A90ED3D1A81
:10C0E00001EE801AD0ED191A91ED012A61EE821A43
:10C0F00001EEC01AD1ED021A61EE801A90ED362AD7
:10C1000001EEC21AD1ED001A61EE801A90ED382AC4
:10C1100001EE821A80ED3D1A90ED111AD1ED021A4E
:10C1200061EE211A90ED3E1A01EE801AD0ED1A1A36
:10C1300091ED012A61EE821A01EEC01AD1ED011AC9
:10C1400061EE801A90ED362A01EE821AD1ED001AC6
:10C1500061EE801A90ED372A01EEC21A80ED3E1A88
:10C1600090ED061AD1ED021A61EE211A90ED451AF2
:10C1700001EEC01AD0ED181A91ED002A61EE821A74
:10C1800001EE801AD1ED021A61EE801A90ED402A7C
:10C1900001EE821AD1ED011A61EE801A90ED412A6A
:10C1A00001EEC21A80ED451A90ED071AD1ED021A80
:10C1B00061EE211A90ED461A01EEC01AD0ED191A5F
:10C1C00091ED002A61EE821A01EE801AD1ED021A79
:10C1D00061EE801A90ED3F2A01EEC21AD1ED001AED
:10C1E00061EE801A90ED412A01EE821A80ED461A26
:10C1F00090ED081AD1ED021A61EE211A90ED471A5E
:10C2000001EEC01AD0ED1A1A91ED002A61EE821AE1
:10C2100001EE801AD1ED011A61EE801A90ED3F2AED
:10C2200001EE821AD1ED001A61EE801A90ED402ADB
:10C2300001EEC21A80ED471A90ED061AD1ED011AEF
:10C2400061EE211A90ED4E1A01EE801AD0ED0F1A10
:10C2500091ED002A61EE821A01EEC01AD1ED021AA8
:10C2600061EE801A90ED492A01EE821AD1ED011A91
:10C2700061EE801A90ED4A2A01EEC21A80ED4E1A44
:10C2800090ED071AD1ED011A61EE211A90ED4F1AC7
:10C2900001EE801AD0ED101A91ED002A61EE821A9B
:10C2A00001EEC01AD1ED021A61EE801A90ED482A13
:10C2B00001EEC21AD1ED001A61EE801A90ED4A2A01
:10C2C00001EE821A80ED4F1A90ED081AD1ED011A95
:10C2D00061EE211A90ED501A01EE801AD0ED111A7C
:10C2E00091ED002A61EE821A01EEC01AD1ED011A19
:10C2F00061EE801A90ED482A01EE821AD1ED001A03
:10C3000061EE801A90ED492A01EEC21A80ED501AB2
:10C3100090ED011AD1ED021A61EE211A90ED061A84
:10C3200001EE801AD0ED021A91ED012A61EE821A17
:10C3300001EEC01A80ED061A90ED001AD1ED021A36
:10C3400061EE211A90ED071A01EEC01AD0ED021A23
:10C3500091ED002A61EE821A01EE801A80ED071A33
:10C3600090ED001AD1ED011A61EE211A90ED081A34
:10C3700001EE801AD0ED011A91ED002A61EE821AC9
:10C3800001EEC01A80ED081A90ED0A1AD1ED021ADA
:10C3900061EE211A90ED0F1A01EE801AD0ED0B1A02
:10C3A00091ED012A61EE821A01EEC01A80ED0F1A9A
:10C3B00090ED091AD1ED021A61EE211A90ED101AD2
:10C3C00001EEC01AD0ED0B1A91ED002A61EE821A2F
:10C3D00001EE801A80ED101A90ED091AD1ED011AC4
:10C3E00061EE211A90ED111A01EE801AD0ED0A1AB1
:10C3F00091ED002A61EE821A01EEC01A80ED111A49
:10C4000090ED131AD1ED021A61EE211A90ED181A6F
:10C4100001EE801AD0ED141A91ED012A61EE821A14
:10C4200001EEC01A80ED181A90ED121AD1ED021A21
:10C4300061EE211A90ED191A01EEC01AD0ED141A0E
:10C4400091ED002A61EE821A01EE801A80ED191A30
:10C4500090ED121AD1ED011A61EE211A90ED1A1A1F
:10C4600001EE801AD0ED131A91ED002A61EE821AC6
:10C4700001EEC01A80ED1A1A9FED191A20EE011A6A
:10C4800061EE000A002212E002EBC203134400EB4B
:10C49000830393ED001AF6EE001A00EEA11A02EBE8
:10C4A000C203134400EB830383ED001A521C032ADA
:10C4B000EADB062210E002EBC203134400EB830325
:10C4C00093ED001A31EE201A02EBC203134400EB85
:10C4D000830383ED001A521C092AECDB704700002D
:10C4E00017B7D13801480249086070470090D0035F
:10C4F000F84A002010B512F021FC28B195480088B8
:10C50000C0F304209449086012F070FC10B1934805
:10C510009349486712F0A6FC30B18E48E0380068B5
:10C52000C0F342308F49086012F0C8FC28B18E4831
:10C53000006820F080708C49086012F0DDFC48B182
:10C5400000208A4908604FF08041C1F810018549F8
:10C55000091F086012F0FCFC18B103208149643106
:10C56000086012F013FD68B10520814908600120C0
:10C570007F497831086000207D49083108603F20FC
:10C58000091F086012F020FD002855D07148E030E6
:10C590000068784908606F48E4300068091D086049
:10C5A0006C48E8300068091D08606A48EC30006893
:10C5B000091D08606748F0300068091D086065487B
:10C5C000F4300068091D08606248F8300068694965
:10C5D000203108605F48FC300068091D086066482B
:10C5E0000068091D08606448001D0068091D086096
:10C5F000614808300068091D08605F480C30006819
:10C60000091D08605C48103000685A4940310860D4
:10C61000594814300068091D0860574818300068F0
:10C62000091D086054481C300068091D0860524804
:10C6300020300068091D086012F054FB30B14548F5
:10C64000CC38006800F04F004C49086012F0A2FBA3
:10C6500040B14B48006800F0010018B16FF00100D4
:10C660004749086012F0E0FB28B14648006840F4F2
:10C670008060444908603C487438006840F47000A9
:10C6800039497439086000BF00BF00BFBFF34F8F46
:10C6900000BF00BF00BF00BF00BF00BFBFF36F8F70
:10C6A00000BF00BF00BF3848006800F00100F0B1D3
:10C6B00001203649086000BF354800680028FBD0DB
:10C6C0003148006820F001004FF01021C1F80C0241
:10C6D00000BF2F4800680028FBD000202B490860CD
:10C6E00000BF2B4800680028FBD001F055FA26480F
:10C6F0000C38006800F0004028B92348083800686A
:10C7000000F0004018B301202049086000BF204815
:10C7100000680028FBD015201B490C39086000BFB9
:10C720001B4800680028FBD0152117480838016015
:10C7300000BF174800680028FBD00020134908609C
:10C7400000BF134800680028FBD001F025FAFFF76E
:10C75000C9FE10BD24030010403501400DF0ADBAF4
:10C7600000C007403C050040FCED00E00C0100402B
:10C770001056004020C5004024040010E40E004084
:10C78000000400403C1700400C12001004E501407A
:10C7900000E401400148006870470000604000204C
:10C7A0007CB500251B4903C9CDE9000102208DF8A5
:10C7B00002000020ADF80000174A6946174814F03F
:10C7C00033FE044604B16D1E0123212200211348CB
:10C7D00014F0B6FD044664B10123212200210F4864
:10C7E00014F0AEFD044624B10D4A0EA10020FDF761
:10C7F000E5FF0A4814F0FCFD084814F005FE0F4858
:10C8000000F09EFD681C20B90D4A0EA10020FDF726
:10C81000D5FF7CBD808004008D500400788004002A
:10C82000D53F03006273705F7274635F636F6E66FF
:10C8300069675F70726F6365737300003D55030035
:10C84000054003006273705F7274635F696E6974A0
:10C850005F70726F63657373000000000246002111
:10C8600011E00B4850F82100904202D16FF0010016
:10C870007047074850F8210020B9054840F82120AA
:10C880000020F5E7491C2029EBDB4FF0FF30EFE7F4
:10C89000B86C00207047000030B589B00546002410
:10C8A000002009E0C0F105021E498B5C2146621C94
:10C8B000D4B201AA5354401C0628F3DB00222046C0
:10C8C000611CCCB201A90A542046611CCCB201A95A
:10C8D0000A5401222046611CCCB201A90A54204608
:10C8E000611CCCB201A90A5400222046611CCCB2C2
:10C8F00001A90A542046611CCCB201A90A540122A4
:10C900002146601CC4B201A842542146601CC4B236
:10C9100001A84254234601AA2946002000F0C6F986
:10C9200009B030BD0D3F0020F0B504460D46164657
:10C9300024482549086004202449C1F804032448F8
:10C9400004602348083005602248046022480560DE
:10C9500030460CF0E3FF1E49183108601C480C38C3
:10C96000006840F004001A490C3908604FF0FF30AD
:10C9700016498860086002200321002804DB4A076A
:10C98000130E164A135406E04A07170E144A00F015
:10C990000F031B1FD75400BF022000280DDB00BF70
:10C9A00000BF00F01F02012191404209920002F1F4
:10C9B000E022C2F8001100BF00BF00BF00200949FB
:10C9C0000860F0BD03020200082300400020004080
:10C9D0000C250040D43F0020D83F002000E400E0B8
:10C9E00018ED00E01C21004070B504460D461646C7
:10C9F000324629462046FFF797FF054A05A1002049
:10CA0000FDF7DCFE064A07A10020FDF7D7FE70BD4A
:10CA100031CA020055415254305F52780000000084
:10CA20004DCC020055415254305F54780000000054
:10CA300070B565E03348007810B101285BD12BE078
:10CA4000FBF746F8032800D270BD0020FBF710F872
:10CA5000AA2803D00120FBF741F91CE00220FBF7D4
:10CA600007F80446E043C4B20120FBF701F8264969
:10CA7000087008460078844209D1084600780528E5
:10CA800005DB20480078401C1E49087002E00120A8
:10CA9000FBF724F900BF32E0FBF71AF81A490978CE
:10CAA000884200D2D0E70025002406E02046FAF7AD
:10CAB000DFFF2844C5B2601CC4B213480078401E92
:10CAC000A042F3DC10490978491E88B2FAF7D0FF7A
:10CAD000A84208D10C480078FDF78CFF0A4800787E
:10CAE000FBF7FCF802E00120FBF7F8F8002005490D
:10CAF000087000BF03E000200249087000BF00BFBB
:10CB000098E70000EC3F0020ED3F002010B5024602
:10CB100010480068092802D34FF0FF3010BD0E48BE
:10CB20000C4B1B6800EB0310C1600B48094B1B68E2
:10CB300000EB031002700948074B064C246803EB16
:10CB40000413586003480068401C024B1860002022
:10CB5000E4E70000E43F0020D86300206864002080
:10CB60002DE9F043C0B0074688461646002400234E
:10CB7000701D00F0FF09AA200DF8030019465B1C88
:10CB80001DF801002044C4B20DF8039019465B1C47
:10CB90001DF801002044C4B26FEA0900C0B20DF8CC
:10CBA000030019465B1C1DF801002044C4B20DF8B7
:10CBB000037019465B1C1DF801002044C4B2002517
:10CBC0000CE018F805000DF803001846591CCBB20C
:10CBD0001DF800002044C4B2681CC5B2B542F0DBA9
:10CBE0001846591CCBB20DF80040002505E01DF891
:10CBF000050000F007F8681CC5B29D42F7DB40B0A5
:10CC0000BDE8F0830549086000BF054909680029AF
:10CC1000FBD00021024A1160704700001C25004033
:10CC20001C21004008490AE00A68824204D100231E
:10CC30004376136A0B6001E002F1200100BF0A682D
:10CC4000002AF1D170470000E83F002070B50025B0
:10CC5000154804681FE0E068D0B1E068401EE0605D
:10CC6000E068A8B9207A00280ADD207A401E2072E8
:10CC70006068E060227E207C6169FFF771FF07E059
:10CC80002046FFF7CFFFE06910B12046E1698847F1
:10CC9000607E0543246A002CDDD12946AFF25300A3
:10CCA000FDF768FD70BD0000E83F00202DE9F04170
:10CCB0000446884615461E4613480768ECB184F8BA
:10CCC0001080656126766068E0602078002803DDCA
:10CCD0002078401E207201E0002020720120607642
:10CCE00004E0A74201D1BDE8F0813F6A002FF8D1EE
:10CCF00005480068206204480460324629464046E0
:10CD0000FFF72EFF00BFEEE7E83F002070B50546B5
:10CD10000C4600201F4908601F4820490860022077
:10CD2000002817DB00F01F02012191401C4A430933
:10CD300042F8231000BF00BF00BFBFF34F8F00BFFA
:10CD400000BF00BF00BF00BF00BFBFF36F8F00BFB9
:10CD500000BF00BF00BF0220002807DB00F01F0259
:10CD6000012191400F4A430942F8231000BF284691
:10CD700013F0BAF9204613F0B7F916200A490860F3
:10CD80000A4908600A48FDF76BFD0A48FDF768FD8F
:10CD900070BD00000025004084020200082300400E
:10CDA00080E100E080E200E0D43F0020D83F002096
:10CDB00031CA02004DCC02002049086820490968A8
:10CDC000B9B100221E4B1A601E4A1268D1B21B4A2A
:10CDD0001268501C1C4A904201D3A2F580601B4A85
:10CDE0001268904204D0154A12681170134A1060FC
:10CDF00000BF13493C31096819B10021104A3C3287
:10CE000011600F490839096819B100210C4A083A24
:10CE100011600B49091F096819B10021084A121F46
:10CE200011600749143109680949D1F8241119B171
:10CE30000021034A1C32116070470000DC3F0020D3
:10CE40000821004018250040D8630020E03F002062
:10CE50000020004010B5FFF7A3FC0DF0A9FDF9F785
:10CE6000F9FF0CF061FFFAF705F9FAF7C1FA0EF0D5
:10CE70005BFC0CF06FFF03F0C5F804F02BF904F035
:10CE80003DFD02F005FE05F029FA03F007FF04F06E
:10CE90000BFA04F085FB03F0C1FD05F009FB03F07C
:10CEA00009FE04F07DFF04F023F904F047FD05F0CE
:10CEB00057F8FFF7EFFC10BD2DE9F041FDF710FC2E
:10CEC00010BBFEF7DFFC0EF0E5FC044618F02AF874
:10CED0000F49086008460068A0B90D2008600846A0
:10CEE000046804B90DE000BF4FF47A7505B904E099
:10CEF000084EAF013846B04700BF601E041EF3D194
:10CF000000BF00BF00F002FAFBF764FABDE8F08151
:10CF1000D03D0020817D040010B588B00020049031
:10CF20000590069007903048007900282BD02E48B5
:10CF300090F82F00432855D12B4890F83A1090F8DC
:10CF4000392090F83800284BDB79CDE90030CDE965
:10CF5000022125488379427924A104A800F0BEFD6E
:10CF600004A8F9F7B1FA044604AB224626A1002032
:10CF7000FEF7C4F904A8F9F7A7FA0446214604A865
:10CF80000EF006FD2EE0184890F82F00432825D11A
:10CF9000154890F83A1090F8392090F83800124B64
:10CFA000DB79CDE90030CDE902210F488379427960
:10CFB0000EA104A800F092FD04A8F9F785FA044632
:10CFC00004AB224615A10020FEF798F904A8F9F752
:10CFD0007BFA0446214604A819F074FB0C2113A027
:10CFE0000EF0D6FC08B010BD085200202530325893
:10CFF00025303258253032582530325825303258B5
:10D0000025303258000000007363616E4E616D651B
:10D01000282564293A25730A000000006164764ED1
:10D02000616D65282564293A25730A00313233324F
:10D030003133323133313200B0EE401A81EE200A02
:10D04000DFED021A20EE210A704700000000C842FE
:10D0500010B52DED048BB0EE408A9FED230AB0EEA3
:10D06000409A9FED210AF0EE408A2048007848B1AE
:10D07000B2EE040AC8EE000A1D48C0ED000A002006
:10D080001A490870B2EE040AC8EE000AF0EE609A7F
:10D090001748DFED180AB0EE690A0BF04AFCF0EE13
:10D0A000408A9FED150AF4EEC08AF1EE10FA04D220
:10D0B0009FED0D0AB0EE409A11E09FED100AF4EEDC
:10D0C000C08AF1EE10FA04DD9FED0D0AB0EE409A31
:10D0D00005E0B0EE680A0FF07DFBB0EE409AB0EECE
:10D0E000490ABDEC048B10BD00000000FC3F00208D
:10D0F000F03F00200AD7233C0000A0430000D243A9
:10D100000000C84208B500BF4FF480700B4940587A
:10D1100008B1012000E0002078B10948006880478C
:10D1200000BF00204FF48071044A88500846114621
:10D130004058009000BF00BF00BF08BD0000014084
:10D14000784A00202DE9F0410246C2F30744C2F3B9
:10D150000726D5B2802300200021CCE0880006EA13
:10D160000307D7B1664F3F88DFF898C12CF81070DD
:10D17000634FB7F802C0DFF88C81471C28F817C04E
:10D180005F4FB7F804C0871C28F817C05C4FB7F88A
:10D1900006C0C71C28F817C019E05B4F3F88DFF8AE
:10D1A00064C12CF81070584FB7F802C0DFF85481F2
:10D1B000471C28F817C0544FB7F804C0871C28F83C
:10D1C00017C0514FB7F806C0C71C28F817C0880011
:10D1D00004EA030717B34A4FB7F800C0494F403776
:10D1E00027F810C0464FB7F80280464F403700F18D
:10D1F000010C27F81C80424FB7F80480414F40379C
:10D2000000F1020C27F81C803D4FB7F806803D4F17
:10D21000403700F1030C27F81C8021E03A4FB7F8A3
:10D2200000C0384F403727F810C0374FB7F802809A
:10D23000344F403700F1010C27F81C80324FB7F80B
:10D240000480304F403700F1020C27F81C802E4F2D
:10D25000B7F806802B4F403700F1030C27F81C80ED
:10D26000880005EA030717B3254FB7F800C0254F1C
:10D27000803727F810C0224FB7F80280214F80373F
:10D2800000F1010C27F81C801D4FB7F804801D4FDA
:10D29000803700F1020C27F81C80194FB7F8068080
:10D2A000184F803700F1030C27F81C8021E0164F3F
:10D2B000B7F800C0134F803727F810C0124FB7F8E7
:10D2C0000280104F803700F1010C27F81C800E4FB0
:10D2D000B7F804800B4F803700F1020C27F81C8050
:10D2E000094FB7F80680074F803700F1030C27F885
:10D2F0001C805B08491C0829FFF630AFBDE8F081AF
:10D30000B67D0400D85E0020BE7D040010B5002468
:10D310000AE0084850F8240028B1064850F82410C4
:10D32000054800688847641C044800788442F0DBA4
:10D3300010BD00003C4B0020D03D0020D53D00201A
:10D340000246002116E00E4850F82100904202D11A
:10D350004FF0FF3070470A4850F8210048B909489B
:10D360000078401C074B1870054840F82120002029
:10D37000F0E7491C0629E6DB6FF00100EAE7000050
:10D380003C4B0020D53D002010B50BF0ABFA10BD92
:10D390002DE9F74FADF5825D8946154600210DF563
:10D3A000805081638B46416388468A46002601632C
:10D3B0000027006C2844B0F5F02F05D9022013B0E7
:10D3C0000DF5805DBDE8F08F41F2380169440DF53F
:10D3D0008050006CFBF7ECFF04460CB12046EEE7F2
:10D3E00041F2340169440DF58050006CFBF7C0FF39
:10D3F00004460CB12046E2E70DF58050406BC0F5C5
:10D400008060B5EB800F03D84FF0010B002711E0CF
:10D410004FF0010B0DF58050406BC0F58061A5EB1E
:10D420008107C7F30B0008B1012000E0002000EBEA
:10D43000173083442F464FF000087DE00DF58051F2
:10D44000098F414488B241F230016944FBF7A4FFDF
:10D4500004460CB12046B2E7B8F1000F12D10DF529
:10D460008050406BC0F58060B7EB800F06D90DF59A
:10D470008050406BC0F58060800000E03846064672
:10D48000AF1B0CE000210DF580504163B7F5805FC4
:10D4900002D94FF4805000E038460646BF1B0DF518
:10D4A00080514A6B096B01EB820041F23C026A44F5
:10D4B000314600F091FB04460CB120467FE70DF5A4
:10D4C000805090F83C0018B34FF480520CA90DF531
:10D4D0008050006BFDF734FB04460CB120466EE72C
:10D4E00009EB8A010CAB0DF58052526B03EB820005
:10D4F0003246F8F7C5FF4FF480530CAA01210DF511
:10D500008050006BFBF76EFE04468CB1204656E758
:10D5100009EB8A010DF58052536B126B02EB83000D
:10D5200000233246FBF720FE04460CB1204646E7B6
:10D530000AEB960A08F10108D845FFF47FAF0020F6
:10D540003DE7000010B50246002A01DC022010BDB4
:10D550002148B0F90000801A01D50120F7E71F48E3
:10D560001F4B1B6800F833201D48006840B94FF47A
:10D57000E8201A4B1A4C246803EBC403586016E0E9
:10D5800017480068401E154B03EBC0004368144861
:10D590000068401E114C14F830004FF4805414FB06
:10D5A00000330E480E4C246800EBC400436031B1D8
:10D5B0000A480B4B1B6800EBC30040680860064834
:10D5C0000088801A00B2044B188005480068401C8F
:10D5D000034B18600020BAE7AC3F0020B85E002083
:10D5E000B03F00207CB5064601A9304600F03EF869
:10D5F00004460CB120467CBD002517E00F49019A76
:10D6000001EBC201496801EB05306946FBF7D0FE2A
:10D6100004460CB10620EEE7BDF80000FAF782FBE5
:10D6200004460CB10620E6E7681CC5B20348019920
:10D6300010F83100A842E1DC0020DCE7B85E0020F1
:10D64000F8B506460C466946304600F00FF8054628
:10D650000DB12846F8BD2CB10348009910F83100EF
:10D66000000320600020F5E7B85E002010B50246F8
:10D670000B46002115E00E4800EBC10040689042C7
:10D680000ED80B4800EBC1004468094810F831007F
:10D6900004EB0030904203D903B11960002010BDA3
:10D6A000491C044800688142E5D30320F7E70000E5
:10D6B000B85E0020B03F00202DE9F84306460F4633
:10D6C000144669463046FFF7D1FF054615B1284696
:10D6D000BDE8F883CFB1C4B10D48009900EBC1009B
:10D6E00041680B48009A10F8320001EB00383019FD
:10D6F000404501D90420EBE7224639463046FDF784
:10D700002AFA05460DB10420E2E70020E0E7000018
:10D71000B85E00202DE9F84306460F4614466946D8
:10D720003046FFF7A3FF054615B12846BDE8F8834C
:10D73000CFB1C4B10D48009900EBC10041680B485E
:10D74000009A10F8320001EB00383019404501D939
:10D750000520EBE7224639463046FFF719FE05461D
:10D760000DB10520E2E70020E0E70000B85E0020F0
:10D7700010B5124C02202061606111A0A061134914
:10D78000E1614FF4007121620021A1626162E162F6
:10D790000BA0A0640E49E164102121650021A16560
:10D7A0006165E1650BA1E01DF8F7B0FE0AA1204616
:10D7B000F8F7ACFE2020A07110BD0000508C0020B6
:10D7C0005465726D696E616C00000000C88C0020A9
:10D7D000C88E00205254540053454747455200001C
:10D7E00010B501460A69CB689A4204D88C68641E59
:10D7F000E41AA01801E0D41A601E10BD2DE9FC5FE8
:10D8000006460F4692469846DDE90C45002F01DAA0
:10D81000784200E0384683464FF0010903E09BFB65
:10D82000FAFB09F10109D345F9DAC84500D9C14627
:10D8300034B1002F03DB05F00400042800D1641E7E
:10D8400005F0020010B1B8F1000F11D005F0010091
:10D8500070B96CB108E0641E2021304600F0BAF8BF
:10D86000F068002800DA02E00CB1A145F3D300BF54
:10D87000F068002836DB002F05DA7F422D21304684
:10D8800000F0A8F807E005F00400042803D12B21DC
:10D89000304600F09FF8F068002823DB05F0020016
:10D8A000022814D105F0010088B9B8F1000F0ED19B
:10D8B0006CB108E0641E3021304600F08BF8F0684F
:10D8C000002800DA02E00CB1A145F3D300BFF068F4
:10D8D000002807DB4346524639463046CDE900452D
:10D8E00000F002F8BDE8FC9F2DE9FC5F8046894608
:10D8F00015461E460C9CCDF804900127BB4605E05A
:10D900000198B0FBF5F001900BF1010B0198A842D2
:10D91000F6D25E4500D9B3460D9800F00100D0B9AB
:10D92000CCB10D9800F00200022803D116B93020C6
:10D93000009001E02020009009E0641E404600991C
:10D9400000F048F8D8F80C00002800DA02E00CB12A
:10D95000A345F2D300BFD8F80C00002835DB09E05E
:10D96000012E01D9761E04E0B9FBF7FAAA4500D2D0
:10D9700001E06F43F4E700BF00BFB9FBF7FA0AFB11
:10D980001799134810F80A10404600F023F8D8F809
:10D990000C00002800DA03E0B7FBF5F7002FECD10C
:10D9A00000BF0D9800F0010078B174B109E0641E69
:10D9B0002021404600F00EF8D8F80C00002800DACC
:10D9C00002E00CB1A345F2D300BFBDE8FC9F00000C
:10D9D0002685040070B504460E46A568681C61687B
:10D9E000814206D320684655681CA060E068401C50
:10D9F000E060D4E9011088420DD1A2682168206955
:10DA0000FDF71CFCA168884203D04FF0FF30E060B6
:10DA100001E00020A06070BD2DE9F0470446894672
:10DA200017464FF0000AE56800BFD4F81080A845FB
:10DA300003D9A8EB0500461E04E0A5EB0800401C36
:10DA4000A1680E1A06B90126A068401BB04201D990
:10DA5000304601E0A068401B0646BE4201D2304677
:10DA600000E0384606466168481932464946F8F7EC
:10DA700007FDB244B144BF1B3544A068A84200D1A1
:10DA80000025E560002FD0D15046BDE8F0872DE994
:10DA9000F047044689461546E668A068871BAF42F2
:10DAA00008D9616888192A464946F8F7E9FC7019CF
:10DAB000E06010E0B8466168881942464946F8F7C8
:10DAC000DFFCA5EB070809EB070142466068F8F7A1
:10DAD000D7FCC4F80C80BDE8F08700000FB4084BF9
:10DAE00010B504A902AA039801F02AFA044602A973
:10DAF000002001F056FC204610BC5DF814FB00002D
:10DB0000A3F3020003B401984100009850EAC12039
:10DB100018BF04204A0D18BF40F0010040F2FF7208
:10DB2000B2EB515F08BF40F00200012808BF05209A
:10DB300002B0704713B5DDE900200AB1012200E010
:10DB4000002240EA020121F00040024A101AC00FF0
:10DB50001CBD00000000F07F00BF00BF00BFBFF38E
:10DB60004F8F00BF00BF00BF0948006800F4E060AD
:10DB700008490843001D0649086000BF00BF00BFF8
:10DB8000BFF34F8F00BF00BF00BF00BF00BFFDE766
:10DB90000CED00E00000FA0500BF00BF00BFBFF3BE
:10DBA0004F8F00BF00BF00BF0948006800F4E0606D
:10DBB00008490843001D0649086000BF00BF00BFB8
:10DBC000BFF34F8F00BF00BF00BF00BF00BFFDE726
:10DBD0000CED00E00000FA052DE9F84305460C467F
:10DBE000904600272819B0F5F02F02D90220BDE891
:10DBF000F88305F0030000B90DB90320F7E704F03E
:10DC0000030000B90CB90420F1E7A4080FE00423D5
:10DC10006A4600212846FBF7E5FA06460EB1304673
:10DC2000E5E70098401C00B103E02D1D7F1CA742D2
:10DC3000EDD300BFA74201D0012000E0002088F80A
:10DC400000000020D3E7000070B5C1482DED020BA5
:10DC50002DED0E8B82B0119D25F000449FEDBEDBB3
:10DC60009FEDBFEB84423EDBA4F140511098A1F13F
:10DC70007F6108430FD0BC48844202DC28D1109851
:10DC800030B39DED100B02B0BDEC0E8B02B0BDE8C1
:10DC9000704001F0E9B89DED100B53EC1D2B51ECD9
:10DCA000100BF8F7E3FC9DED100B41EC180B53EC57
:10DCB0001E2B51EC100BF8F7D9FC53EC182BF8F78E
:10DCC0002EFC41EC100B02B0BDEC0E8B02B070BD0F
:10DCD000012001F02FF902B0BDEC0E8B02B0BDE8BF
:10DCE000704001F0D5B8A1489FEDA18B844256DA6F
:10DCF0009DED100BB4F1795F0ADA51EC100BFFF7D0
:10DD000001FF042808BF01F0D3F89DED100BDAE7FE
:10DD100053EC102B51EC100BF8F7A8FC41EC190B4D
:10DD200095480621B0EE490AF0EE690A784400F001
:10DD300087FF53EC192B51EC100BF8F797FC41ECD3
:10DD40001A0B8E48B0EE490AF0EE690A04217844B5
:10DD500000F076FF53EC192B51EC100BF8F786FC12
:10DD600053EC182BF8F7DBFB41EC100B51EC1A0BC2
:10DD700053EC102BF8F7ECFCCDE900019DED000B06
:10DD800053EC102B9DED100B51EC100BF8F76EFCC3
:10DD90009DED101B53EC112BF8F7C1FBD2E09DED6C
:10DDA000100B51EC100B0AF0CDFC53EC182BF8F7CC
:10DDB0005AFC9FED730BCDE9000153EC102B9DED48
:10DDC000000B51EC100BF8F751FC41EC190B6E48AD
:10DDD0000621B0EE490AF0EE690A784400F030FFFF
:10DDE00053EC192B51EC100BF8F740FC41EC1B0BDA
:10DDF0006648B0EE490AF0EE690A0421784400F062
:10DE00001FFF53EC192B51EC100BF8F72FFC53ECC0
:10DE1000182BF8F784FB41EC1C0B51EC190B19F093
:10DE200091F941EC180B5A489FED5BABA04222DC04
:10DE300053EC1C2B51EC1B0BF8F78AFCCDE90001CD
:10DE40009DED000B51EC180B53EC102BF8F70EFC6A
:10DE500053EC182BF8F763FB53EC1A2BF8F706FC7E
:10DE600053EC1D2BF8F7FCFB53EC1E2BF8F7FBFBD8
:10DE700041EC100B5FE08DED008B002000909DEDDC
:10DE8000000B51EC180B53EC102BF8F748FB9DEDF1
:10DE9000000B41EC1E0B53EC102B51EC100BF8F760
:10DEA000E5FB53EC192BF8F7DEFB53EC1E2BF8F7D0
:10DEB0004FFC41EC190B53EC1C2B51EC1B0BF8F7EE
:10DEC00047FC41EC1B0B53EC1A2B51EC190BF8F7E8
:10DED000CDFB53EC1D2BF8F7C6FB41EC190B53ECB3
:10DEE0001A2B51EC180BF8F7C1FB53EC1B2BF8F76E
:10DEF000BDFB53EC192BF8F7B3FB9DED000B41EC88
:10DF0000180B53EC1A2B51EC100BF8F7AFFB9FEDED
:10DF1000249B53EC192BF8F7A6FB41EC100B51ECAA
:10DF2000180B53EC102BF8F79BFB53EC192BF8F75D
:10DF30009AFB41EC100B002D3FF7C5AE51EC100BD6
:10DF400081F0004141EC100BBDE600000000000034
:10DF50000000F03F00000000075C143326A6913C4F
:10DF6000182D4454FB21F93F0000F07F0000E03FF2
:10DF7000000000000000F03FC8A80100D6A8010082
:10DF8000000000000000E03F1AA8010028A80100DE
:10DF90003333EF3F000000000000000000000040AD
:10DFA000182D4454FB21E93F70B59B482DED020B21
:10DFB0002DED068B079D25F00044A04218DC974804
:10DFC000844202DC0AD1069840B19DED060BBDECFF
:10DFD000068B02B0BDE8704000F046BF002DCCBFFC
:10DFE0009FED8F0B9FED900BBDEC068B02B070BDCB
:10DFF0008F48A04215DD8F48A042D8BF4FF0FF34B4
:10E0000058DD9DED060B51EC100BFFF77BFD04284E
:10E0100008BF00F04DFF9DED060BBDEC068B02B076
:10E0200070BD9DED060B51EC100B0AF08BFBCDE99A
:10E03000060181489FED828BA0423CDD8248A042D0
:10E040001FDD00249FED82AB9DED060B53EC1A2BD8
:10E0500051EC100BF8F763FA9DED060B41EC190B30
:10E0600053EC1A2B51EC100BF8F700FB53EC182B68
:10E07000F8F7F6FA53EC192BF8F76AFBCDE906012D
:10E0800049E09DED060B012453EC182B51EC100BCD
:10E09000F8F745FA9DED060B41EC190B53EC182BE4
:10E0A00051EC100BF8F7DCFA53EC192BF8F750FB96
:10E0B000CDE906012FE06848A0421FDD02249FED54
:10E0C000689B9DED060B53EC192B51EC100BF8F7E8
:10E0D000CDFA53EC182BF8F722FA9DED060B41EC24
:10E0E000180B53EC192B51EC100BF8F7B9FA53EC51
:10E0F000182BF8F72DFBCDE906010CE09DED060B82
:10E10000032453EC102B9FED580B51EC100BF8F738
:10E110001FFBCDE906019DED060B53EC102B51ECD6
:10E12000100BF8F7A3FA41EC180B53EC182BF8F787
:10E130009DFA41EC190B4E480621B0EE490AF0EE6B
:10E14000690A784400F07CFD53EC182B51EC100B5D
:10E15000F8F78CFA41EC180B4648B0EE490AF0EE9D
:10E16000690A0521784400F06BFD53EC192B51EC42
:10E17000100BF8F77BFA41EC100B51EC180B53EC39
:10E18000102B002C0EDAF8F7CAF99DED061B53ECA4
:10E19000112BF8F76BFA9DED061B53EC112BF8F7DA
:10E1A00062FA35E0F8F7BBF99DED061B53EC112B35
:10E1B000F8F75CFA41EC100B2F48784400EBC400F0
:10E1C00090ED001B51EC100B53EC112BF8F748FAB3
:10E1D0009DED061B53EC112BF8F742FA41EC100BA6
:10E1E0002648784400EBC40090ED001B51EC100B66
:10E1F00053EC112BF8F737FA41EC100B002DA2BFAE
:10E20000BDEC068B02B070BD51EC100B81F00041EB
:10E2100041EC100B01E70000000010440000F07F0B
:10E22000182D4454FB21F93F182D4454FB21F9BF0C
:10E230000000DC3F0000203E0000F33F0000000033
:10E24000000000000000F03F0000E63F000000007A
:10E2500000000000000000400080034000000000BB
:10E26000000000000000F83F000000000000F0BFC8
:10E270006AA5010020A50100AAA4010062A4010072
:10E2800070B56B4E2DED040B2DED028B82B0DDF8D9
:10E290001CC0DDE905235C422CF000411C4341EA2F
:10E2A000D474049D22F00040B44205D86C422C4343
:10E2B00040EAD474B4420BD99DED061B9DED040BCE
:10E2C00002B0BDEC028B04B0BDE8704000F0D6BDDA
:10E2D000ACF14054A4F17F641C430BD0022404EA47
:10E2E000AC7444EAD27405439FED538B9FED542BDD
:10E2F00007D015E09DED040B51EC100B04F0AEF9C6
:10E3000042E0002C11BF012C9DED040B02B0BDECCE
:10E31000028B04BF04B070BD022C38D0032C3BD05C
:10E320000B439FED491B9FED4A0B0AD0B14218D118
:10E33000B04209D121F0804120F080400791059042
:10E340000FE0002A15DA10E0434B7B44002C08BF95
:10E3500093ED000B0DD0012C10D0022C17D0032C04
:10E360001AD0B0421DD1002A03DAB0EE410AF0EE15
:10E37000610A02B0BDEC028B04B070BD93ED000BDE
:10E3800051EC100B81F0004141EC100BF1E7B0EEC5
:10E39000480AF0EE680AECE7B0EE420AF0EE620AD4
:10E3A000E7E7401A00153C28C8BF8DED000B19DCCB
:10E3B000BCF1000FBEBF10F13C0F9FED290B8DED9E
:10E3C000000B0FDB9DED060B53EC102B9DED040BAA
:10E3D00051EC100BF8F7BCF90AF0B4F904F03EF96F
:10E3E000CDE90001002C08BF9DED000BC1D0012C30
:10E3F00010D0022C9FED1C0B53EC102B9DED000B4D
:10E4000051EC100B0DD0F8F72BF953EC182BF8F753
:10E4100027F9B9E7019880F0004001909DED000BCD
:10E42000A7E7F8F71DF953EC182BF8F71CF9ABE741
:10E430000000F07F00000000182D4454FB2109402B
:10E44000182D4454FB2109C0182D4454FB21F9BF59
:10E45000182D4454FB21F93FC2A301000000000025
:10E460000000000000000000075C143326A6A13C59
:10E4700010B52F499FED2C1B2DED020B84B0059894
:10E4800020F000408842D8BF9DED040B2DDD2949C6
:10E49000884209D1049840B94FF0010000F04AFDCC
:10E4A00000F0F6FC06B010BD05DB9DED040B00F09E
:10E4B000DBFC06B010BD68469DED040B00F0ECF8E7
:10E4C00010F0030004BF9DED021B9DED000B0CD06E
:10E4D00001280ED09DED021B9DED000B022817D0E8
:10E4E000012000F029FC06B010BD00F0F1FA06B0E2
:10E4F00010BD9DED021B9DED000B012000F01CFCEA
:10E5000051EC100B81F0004106B041EC100B10BD36
:10E5100000F0DEFA51EC100B81F0004106B041EC46
:10E52000100B10BD00000000000000000000000003
:10E53000FB21E93F0000F07F2DED020B019820F058
:10E54000004001909DED000B02B0704700000000FC
:10E5500010B52F499FED2C1B2DED020B84B00598B3
:10E5600020F000408842DCBF00209DED040B32DD2E
:10E570002849884209D1049840B94FF0010000F0C1
:10E58000D9FC00F085FC06B010BD05DB9DED040B49
:10E5900000F06AFC06B010BD68469DED040B00F06B
:10E5A0007BF810F0030011D0012818D09DED021B5C
:10E5B0009DED000B02281AD000F08AFA51EC100BE6
:10E5C00081F0004106B041EC100B10BD9DED021B27
:10E5D0009DED000B012000F0AFFB06B010BD9DEDDE
:10E5E000021B9DED000B00F073FA06B010BD012078
:10E5F00000F0A2FB51EC100B81F0004106B041ECA1
:10E60000100B10BD00000000000000000000000022
:10E61000FB21E93F0000F07F00B52DED048BB0EE4B
:10E62000409AF0EE609A83B051EC190BF8F752FA69
:10E6300041EC180B18EE100A18EE901A8DED008BB5
:10E64000002818BF0120084320F00040C0F17F607F
:10E6500000F1E040C00F14D019EE101A19EE900A24
:10E660008DED009B002918BF0121084320F00040D8
:10E67000C0F17F6000F1E040C00F04BF012000F056
:10E6800059FCB0EE480A03B0F0EE680ABDEC048B0A
:10E6900000BD0000000000002DE9F14F04462DED03
:10E6A000020B2DED088B8AB09FEDE70B80ED020B7E
:10E6B000139EE74826F0004585420ADC9DED120BCB
:10E6C000002084ED000B0AB0BDEC088B03B0BDE860
:10E6D000F08FE0489FEDE0AB9FEDE1BBA84247DD46
:10E6E000E14F9FEDE39B9FEDE48B9DED120B53EC0F
:10E6F0001A2B51EC100B002E1CDDF7F7B1FF41EC8B
:10E70000100BBD4208D053EC1B2B51EC100BF7F74C
:10E71000A7FFC4E900010BE053EC192B51EC100BDF
:10E72000F7F79EFF53EC182BF7F79AFFC4E90001A7
:10E730000120C8E7F7F7F3FE41EC100BBD4208D00B
:10E7400053EC1B2B51EC100BF7F7E9FEC4E9000169
:10E750000BE053EC192B51EC100BF7F7E0FE53ECE8
:10E76000182BF7F7DCFEC4E900014FF0FF30AAE7F1
:10E77000C348A84279DB9DED120B51EC100B09F058
:10E78000E1FF41EC180B9FEDC00B53EC102BF7F79A
:10E790006DFF9FEDBF1B53EC112BF7F7C0FEF8F791
:10E7A00064F80746F8F743F841EC190B53EC1A2BC1
:10E7B000F7F75CFF53EC182BF7F755FF41EC180BFC
:10E7C00053EC1B2B51EC190BF7F750FFDFF8C8A2E5
:10E7D00041EC100B4FEA15580125FA4453EC102B6D
:10E7E00051EC180BF7F73CFF032DC4E900013DD0B5
:10E7F000C1F30A5005EB4511A8EB00001139814225
:10E8000034DA0AEB051BB0EE48AA9BED000BF0EEE4
:10E8100068AA53EC102B51EC190BF7F727FF41ECCA
:10E820001B0B51EC1A0B53EC1B2BF7F719FF41ECA8
:10E83000180B51EC1A0B53EC182BF7F711FF53EC94
:10E840001B2BF7F70DFF9BED020B41EC1A0B53EC62
:10E85000102B51EC190BF7F709FF53EC1A2BF7F7B4
:10E86000FFFE41EC100B6D1CB8E70EE0002EA8BFB8
:10E870003846BFF628AF94ED000B51EC100B81F039
:10E880000041C4E9000178421DE7C6F3130040F4DB
:10E89000801EC6F30A50A0F2F530471100F01F05A4
:10E8A000C5F12000DDF848B00890002006900790E0
:10E8B0000520EC467949002D07EB0002794408BF9A
:10E8C00051F8221009D051F8223001EB8201AB40FF
:10E8D0004A68089922FA01F11943A1FB0E26A1FB0F
:10E8E0000B131A449A4234BF0123002303EB06089A
:10E8F0000CEB8003D3E901A60E448E4234BF012104
:10E90000002192448A4411B1924502D903E0924514
:10E9100001D2012100E00021C3E901A641444CF8E5
:10E920002010011EA0F10100C4DC029800F100508B
:10E93000850F0298DDE903678000DDF81480F7F7A2
:10E9400076FF41EC1A0B3046F7F782FF9FED541B20
:10E9500053EC112BF7F78AFE41EC1B0B3846F7F707
:10E9600077FF9FED511B53EC112BF7F77FFE41EC26
:10E97000180B4046F7F76CFF9FED4D1B53EC112B26
:10E98000F7F774FE41EC190B51EC180B53EC192BF3
:10E99000F7F7C5FD53EC1B2BF7F7C1FD53EC1A2B12
:10E9A000F7F7BDFDCDE90801002008909DED080BAB
:10E9B00053EC1A2B51EC100BF7F752FE53EC1B2BB8
:10E9C000F7F74EFE53EC182BF7F74AFE53EC192BD2
:10E9D000F7F749FE9FED381B53EC112BF7F746FE76
:10E9E0009FED370B41EC180B53EC102B9DED080BF2
:10E9F00051EC100BF7F73AFE53EC182BF7F78FFD9D
:10EA00009FED310B41EC180B53EC102B9DED080BD7
:10EA100051EC100BF7F72AFE53EC182BF7F77FFD9C
:10EA200041EC100B139810F0004F06D06D4251ECE2
:10EA3000100B81F0004141EC100B284684ED000BD7
:10EA400041E600000000000000000000000000009F
:10EA5000FB21E93F7CD9024000004054FB21F93FF3
:10EA60003163621A61B4D03DFB21F93F0000000020
:10EA70000000601A61B4D03D7370032E8A19A33B65
:10EA8000FB2139410000000083C8C96D305FE43FBD
:10EA9000000000000000E03F3A9F0100889E010056
:10EAA000000000000000103E000000000000103CCC
:10EAB000000000000000103A182D4454FB21F93DDD
:10EAC0003326A611460B113C00000054FB21F93DF2
:10EAD00010B52DED040B2DED088B82B0B0EE419AF0
:10EAE000F0EE619A0B9820F000449FED4BABB4F12F
:10EAF000795F11DA9DED0A0B51EC100BF7F7B5FEBB
:10EB0000002801BFB0EE4A0AF0EE6A0A02B0BDEC7E
:10EB1000088B04BF04B010BD9DED0A0B53EC102B05
:10EB200051EC100BF7F7A2FD41EC180B3C48062105
:10EB3000B0EE480AF0EE680A784400F081F853EC31
:10EB4000182B51EC100BF7F791FD9DED0A0B41ECE2
:10EB50001B0B53EC192B51EC100BF7F787FD41EC15
:10EB6000190B53EC1B2B51EC180BF7F77FFD53ECF3
:10EB7000192BF7F775FD9FED2C0B41EC190B53EC9E
:10EB8000102B51EC180BF7F771FD41EC100B2848D6
:10EB9000844210DA53EC192B51EC100BF7F760FD9F
:10EBA00053EC1A2BF7F75FFD41EC100B02B0BDECF4
:10EBB000088B04B010BD1F48A042BCBF9FED1E1BB8
:10EBC0008DED001B06DBA4F50010019000200090E5
:10EBD0009DED001B51EC100B53EC112BF7F740FD92
:10EBE0009DED000B41EC180B53EC102B51EC1A0B64
:10EBF000F7F736FD41EC1A0B53EC192B51EC180BBF
:10EC0000F7F72EFD53EC1A2BF7F72DFD41EC100B07
:10EC1000CCE7000000000000000000000000F03F12
:10EC2000A49B010000000000000000000000E03F85
:10EC30003333D33F0000E93F000000000000D23F23
:10EC400070B504462DED028B4D1E00EBC500B0EEF5
:10EC5000408AF0EE608A90ED000B35F0060017D088
:10EC600053EC182B51EC100BF7F700FD41EC100B97
:10EC70006D1E04EBC50090ED001B51EC100B53EC26
:10EC8000112BF7F74CFC41EC100B35F00600E7D1E7
:10EC9000022D36D0042D1CD0062D1CBFBDEC028BDE
:10ECA00070BD53EC182B51EC100BF7F7DFFC94ED13
:10ECB0000A1B53EC112BF7F732FC53EC182BF7F728
:10ECC000D5FC94ED081B53EC112BF7F728FC41EC15
:10ECD000100B53EC182B51EC100BF7F7C7FC94ED0D
:10ECE000061B53EC112BF7F71AFC53EC182BF7F714
:10ECF000BDFC94ED040B53EC102BF7F710FC41EC2A
:10ED0000100B53EC182B51EC100BF7F7AFFC94EDF4
:10ED1000021B53EC112BF7F702FC53EC182BF7F7FF
:10ED2000A5FC94ED001B53EC112BF7F7F8FBBDECA1
:10ED3000028B41EC100B70BD31B504462DED040B78
:10ED40002DED0A8BB0EE41BAF0EE61BA0B989DED55
:10ED50000A0B20F00040B0F1795F0DDA51EC100B96
:10ED6000FEF7D0FE042808BF00F0A2F89DED0A0BC4
:10ED7000BDEC0A8B05B030BD53EC102B51EC100BE1
:10ED8000F7F774FC41EC180B9DED0A0B53EC182BB4
:10ED900051EC100BF7F76AFC41EC190B2C48B0EE64
:10EDA000480AF0EE680A05217844FFF749FF9FED15
:10EDB0002ACBB0EE40AAF0EE60AA9CB353EC1C2B19
:10EDC00051EC190BF7F752FC41EC1C0B53EC1A2BCE
:10EDD00051EC190BF7F74AFC9FED210B41EC190B95
:10EDE00053EC102B51EC1B0BF7F740FC53EC192B99
:10EDF000F7F736FC53EC182BF7F738FC53EC1B2BCA
:10EE0000F7F72EFC53EC1C2BF7F72AFC9DED0A1BA1
:10EE100053EC112BF7F727FCBDEC0A8B05B041EC46
:10EE2000100B30BDFFE753EC1A2B51EC180BF7F722
:10EE30001DFC53EC1C2BF7F772FB53EC192BF7F767
:10EE400015FC9DED0A1B53EC112BF7F768FBE3E76C
:10EE5000349A010000000000495555555555C5BF6D
:10EE6000000000000000E03F10B553EC102B51EC07
:10EE7000100BF7F754FB41EC100B10BD10B553EC21
:10EE8000112B51EC100BF7F74AFB41EC100B10BDA6
:10EE90009FED050B10B553EC102B51EC100BF7F751
:10EEA00057FC41EC100B10BD0000000000000000FA
:10EEB0009FED050B10B553EC102B51EC100BF7F731
:10EEC000D5FB41EC100B10BD00000000000000104D
:10EED00002E008C8121F08C1002AFAD17047704723
:10EEE000002001E001C1121F002AFBD17047000081
:10EEF0000146202908DA012088400A4A104008B15A
:10EF0000012070470020FCE7402909DAA1F1200028
:10EF1000012202FA00F008B10120F2E70020F0E738
:10EF20000120EEE7FC06FFBD00BFEFF310810846AD
:10EF300072B670470149086070470000FC4A002023
:10EF40002DE9FF4F8DB00F460546002606E0252827
:10EF50000BD0DDE90F1290476D1C761C2878002835
:10EF6000F5D111B03046BDE8F08F0024A246A1468D
:10EF70000122EC4900E0044315F8013F203B02FA6E
:10EF800003F00842F7D128782A2810D06FF02F021A
:10EF90002878A0F13001092914D80AEB8A0102EB84
:10EFA000410144F0020400EB010A6D1CF0E701CFBF
:10EFB0005FEA000A03D544F40054CAF1000A44F0A1
:10EFC00002046D1C28782E2817D115F8010F44F083
:10EFD00004042A280ED06FF02F022878A0F1300107
:10EFE00009290AD809EB890102EB410100EB01096B
:10EFF0006D1CF2E757F8049B6D1C28786C280FD025
:10F0000006DC4C2817D068280DD06A2814D104E0FB
:10F01000742810D07A280FD10DE044F400140AE0CF
:10F0200044F4801401E044F440146978814202D130
:10F0300004F580146D1C6D1C2A786E2A1FD00CDC20
:10F04000632A31D004DC002A8BD0582A11D1A3E0E6
:10F05000642A68D0692A0CD165E0732A2ED004DCBA
:10F060006F2A73D0702A04D19BE0752A6FD0782A5A
:10F070006ED01046DDE90F129047761C50E1C4F3C4
:10F080000250022806D0032809D0042801CF09D055
:10F09000066045E101CFF117C0E9006140E101CF11
:10F0A00006803DE106703BE117F8040B8DF8000087
:10F0B00000208DF80100EB46012003E057F804BB67
:10F0C0004FF0FF3061074FF0000102D40DE008F16E
:10F0D0000101884649450FDA8045F8DB1BF8081026
:10F0E0000029F4D108E008F1010188468142FADBE9
:10F0F0001BF808100029F6D1DDE90F23AAEB080060
:10F100008146214600F036F9304400EB080604E061
:10F11000DDE90F121BF8010B9047B8F10108F7D297
:10F1200021464846F7E00A21C4F302534FF0000B92
:10F130000891022B04D001CFC117032B09D00AE09C
:10F14000FF1D27F00707F7E8020108E032E01FE0A3
:10F1500020E000B2C117042B01D140B2C117031E39
:10F1600071F1000307DA4FF0000CD0EB0C006CEBF0
:10F1700001012D2302E0230504D52B238DF8243033
:10F18000012303E0E30701D02023F7E7984658E086
:10F190000A2110E010210EE010204FF0000B089023
:10F1A0000CE010214FF0000B44F004044FF008096C
:10F1B000089103E008214FF0000B0891C4F30253BB
:10F1C000022B04D001CF0021032B06D006E0FF1D47
:10F1D00027F00707F7E8020103E080B2042B00D113
:10F1E000C0B24FF0000823072BD5702A07D0DDF8F6
:10F1F00020C08CF0100C5CEA0B0C05D00EE0402314
:10F200008DF82430012308E050EA010306D03023B2
:10F210008DF824308DF8252002239846DDF820C093
:10F220008CF0080C5CEA0B0C0BD150EA010301D105
:10F23000630706D530238DF824304FF00108A9F17B
:10F240000109582A04D038A20B9208AA0A920BE0AE
:10F250003AA2F9E75B46089AF7F7D2F80B9B9B5C5A
:10F260000A9A521E0A92137050EA0102F2D10A98C9
:10F27000ADEB000000F1200B600702D524F48034D0
:10F2800001E04FF00109D94502DDA9EB0B0000E0D8
:10F29000002000EB0B0141440890AAEB010AE003B7
:10F2A00006D4DDE90F232146504600F063F80644FA
:10F2B0004FF0000908E009A911F80900DDE90F1273
:10F2C000904709F10109761CC145F4DBE0030CD538
:10F2D000DDE90F232146504600F04CF8064404E0D7
:10F2E000DDE90F1230209047761C0899481E0890DF
:10F2F0000029F5DC08E00A980A990078491C0A916F
:10F30000DDE90F129047761CBBF10001ABF1010B58
:10F31000F1DC21465046DDE90F2300F019F80644E0
:10F320006D1C1BE609280100303132333435363785
:10F330003839616263646566000000003031323341
:10F3400034353637383941424344454600000000E1
:10F350002DE9F041044600251E461746880404D4D2
:10F3600005E039462020B0476D1C641EF9D52846BB
:10F37000BDE8F0812DE9F041044600251E46904687
:10F38000C80301D5302700E02027880404D505E014
:10F3900041463846B0476D1C641EF9D52846BDE885
:10F3A000F0810A68531C0B601070704770B50446FA
:10F3B000207850B9054A128891B2606812F09CF822
:10F3C000054615B901200249087070BDC4400020EF
:10F3D000C040002070B505460C4605B10CB90020B0
:10F3E00070BD287840082178B0EB510F01D0002083
:10F3F000F6E70622611C681CF7F77BF808B90120C4
:10F40000EEE70020ECE7014601F0030008B9012017
:10F4100070470020FCE7024650680068401E084024
:10F4200008B9012070470020FCE70246002104E0F3
:10F43000505C08B101207047491C0629F8D3002010
:10F44000F9E710B50346D868884206D88818401EE8
:10F450001C69A04201D8012010BD0020FCE700007B
:10F4600010B504466CB10848C068A04209D80648E7
:10F470000069A04205D320460DF0A1FD08B101208E
:10F4800010BD0020FCE70000144B002070B50446BE
:10F490000D4604F22740FFF7C8FF0646012D06D0AF
:10F4A000022D0DD0032D11D0042D19D113E0A07918
:10F4B00028B194F8240010B90EB1012070BD00BF2E
:10F4C000E07910B10EB10220F8E700BF207A08B150
:10F4D0000320F3E700BF607A08B10420EEE700BF25
:10F4E0000020EBE70146481C052290FBF2F302FBEB
:10F4F0001300C0B270472DE9F04704460D462F4671
:10F5000095F82080B4F81C9000260BE007EB46121B
:10F510004946A06903F0D6FB10B10120BDE8F08791
:10F52000701CC6B24645F1DB0020F7E7014691F8B2
:10F530002420012A01D1EE2000E01F20704770B581
:10F5400004460D46164632462946204603F0BAFBCD
:10F5500070BD000008B10149086070479047002065
:10F5600030B5ADB004200190AC2102A8F6F7A1FFA0
:10F5700002208DF8080000208DF80A0005208DF883
:10F580000B0001A803900121ADF854101149169108
:10F5900001218DF884104FF4A071249144F2506140
:10F5A00025910D482B9002A90C4803F0F7FB044667
:10F5B00000BF254635B100BF09A27A212846F6F7DB
:10F5C00029FE00BF00BF0121044803F0E4FB2DB079
:10F5D00030BD000010410020811E0400B46E0020E8
:10F5E0002E2E5C2E2E5C2E2E5C626C655F63666731
:10F5F0005C736C6176652E630000000070B50321BA
:10F60000074803F06DFC044600BF254635B100BF36
:10F6100004A299212846F6F7FDFD00BF00BF70BD8A
:10F62000B46E00202E2E5C2E2E5C2E2E5C626C653D
:10F630005F6366675C736C6176652E630000000033
:10F6400070B5084991F8540074DF044600BF2546A0
:10F6500035B100BF04A29F212846F6F7DBFD00BFAD
:10F6600000BF70BDB46E00202E2E5C2E2E5C2E2EA0
:10F670005C626C655F6366675C736C6176652E6364
:10F680000000000070B58CB004460D461646002000
:10F6900005E0C0F10F01615C0DF80010401C10285E
:10F6A000F7D30D2104A8F6F704FF002005E02A5C3B
:10F6B000C0F10F0304A9CA54401C0328F7D36846BD
:10F6C00046DF002005E0C0F10F0208A9895C315433
:10F6D000401C0328F7D30CB070BD000010B50446E1
:10F6E00002480178204603F07DFD10BD434A00200A
:10F6F00010B51248007900B303200BF031FA401C1A
:10F70000D8B10F4802790FA10020FBF7F7FD0C4894
:10F7100001790079401C0A4A107105290DDB00208F
:10F720001146C870002103200BF094FC0123044A09
:10F73000D21CA2210020F8F707F810BD08520020C3
:10F740008A3E002067616D655F6D616E61676572FD
:10F750002E47616D654D6F64654865617274436ED7
:10F76000743A25640D0A000000B589B000200790A6
:10F77000089001200BF0F4F9B0F1FF3F01D109B07E
:10F7800000BD00200BF0E6F9012810DB01AA0021E2
:10F7900008460BF0D5F9BDF80400ADF81C00BDF823
:10F7A0000600ADF81E00BDF80800ADF82000BDF958
:10F7B0001C005849B1F90010884269DABDF91E00F1
:10F7C0005549B1F90010884262DDBDF91E00534968
:10F7D000B1F9001088425BDABDF920005049B1F957
:10F7E0000010884254DABDF920004E49B1F90010EA
:10F7F00088424DDD4C480068401C4B490860084673
:10F800000068012823D1F9F79FFD142804DD47493A
:10F810000320FAF777FA03E045490320FAF772FA72
:10F820000121AFF2BB00FAF7A5FF4FF68820394956
:10F830000880394908804FF4E160384908804FF664
:10F840002420384908804FF4C8703549088036486C
:10F8500000680A285CD10320FAF770FA0021AFF2A1
:10F86000F700FAF787FF4FF6C0102A4908804FF6D5
:10F870008820294908804FF4E160284908804FF624
:10F880002420284908804FF4C870254908803FE0AB
:10F8900025480068E0B10020234908600320FAF7FA
:10F8A0004DFA0021AFF23F10FAF764FF4FF68820BF
:10F8B00018490880184908804FF4E160174908800A
:10F8C0004FF62420174908804FF4C8701449088067
:10F8D00018480078E0B90120164908700320FAF7AB
:10F8E0002DFA0021AFF27F10FAF744FF4FF688207F
:10F8F00008490880084908804FF4E16007490880FA
:10F900004FF62420074908804FF4C8700449088046
:10F9100000BF34E7E83D0020EA3D0020EC3D002038
:10F92000F03D0020EE3D0020E43D0020007F00FF80
:10F9300000106FFFDC3D002000B589B0002007906B
:10F9400008900BF00DF9B0F1FF3F01D109B000BDF7
:10F9500000200BF0FFF8012810DB01AA0021084667
:10F960000BF0EEF8BDF80400ADF81C00BDF8060081
:10F97000ADF81E00BDF80800ADF82000BDF920006C
:10F98000B0F5966F27DD23480068401C21490860C8
:10F9900008460068012811D1F9F7D6FC142804DDC7
:10F9A0001D490320FAF7AEF903E01C490320FAF7DA
:10F9B000A9F90121AFF27F00FAF7DCFE15480068D3
:10F9C0000A2825D30320FAF7B9F90021AFF29700EE
:10F9D000FAF7D0FE1CE00F48006850B100200D4936
:10F9E00008600320FAF7AAF90021AFF2B300FAF792
:10F9F000C1FE0B48007801280AD100200849087090
:10FA00000320FAF79BF90021AFF2D300FAF7B2FE18
:10FA100000BF9BE7E03D0020007F00FF00106FFF6C
:10FA2000DC3D00200146074806E042688A4202D1D8
:10FA30004A684260704740684268002AF5D100BFBA
:10FA4000F8E70000183F00200146074804E042683C
:10FA50008A4200D1704740684268002AF7D14A6064
:10FA6000416000BFF6E70000183F0020044803E0B3
:10FA7000012142681170406841680029F8D170473F
:10FA8000183F00200148007870470000643F0020C4
:10FA90002DE9F04119210020002213461446154695
:10FAA00000BF4FF0A0473E4642EA430747EA8007BF
:10FAB00047EA042747EA054C06F5E06747F821C006
:10FAC00000BF00BF1148007920B11149A820F7F705
:10FAD0005DFD03E00E49A820F7F784FB0D49A72040
:10FAE000F7F780FB0C49A720F7F750FD0B4A0CA154
:10FAF0004FF47A70FAF762FE00F032F80B4A0CA16C
:10FB00000A20FAF75BFEBDE8F081000008520020F1
:10FB10007D4C03008D4C03000150030061FB02008B
:10FB20006170705F6368617267650000EDFC0200E0
:10FB30006170705F6368617267655F6D6F6E697435
:10FB40006F725F626174746572795F636861726716
:10FB5000655F646174615F70726F636573730000E9
:10FB600070B500240025A82000F0A0F8192010F09E
:10FB7000A6FB064616F0A0FD04463848007918B1E9
:10FB80000BF000FF054602E016F096FD0546E6B9CB
:10FB900033480078012817D032A10020FBF7AEFBD4
:10FBA00001202F49087000213248FAF7E3FD0220B6
:10FBB000FAF7C4F82CB100202F49087016F078F934
:10FBC00002E001202C49087070BDFDB1F9F7BCFBC3
:10FBD00064281BDB29480078642817DB204800785C
:10FBE000032830D02548027825A10020FBF786FBAA
:10FBF00003201B49087001211E48FAF7BBFD254967
:10FC00000220FAF77FF816F053F91CE01448007848
:10FC1000022818D020A10020FBF770FB0220104919
:10FC2000087001211348FAF7A5FD1F490220FAF7D1
:10FC300069F82CB116F03CF900200F49087002E079
:10FC400001200D4908703CB10B48007820B100201C
:10FC50000949087016F02CF900BFB5E708520020DA
:10FC6000643F0020636861726765206F75742E2E93
:10FC70002E0A000061FB0200683F0020653F002063
:10FC800063686172676520646F6E653A25642E2E25
:10FC90002E0A0000007F00FF6368617267652069BB
:10FCA0006E2E2E2E0A00000000106FFF30B589B0B6
:10FCB00004460025F9F748FB01462A466D1C01A8B9
:10FCC00081540948007930B12B4601AA2146002011
:10FCD000F7F73AFD05E02B4601AA21460020F7F789
:10FCE00057FB09B030BD0000085200202DE9F0415B
:10FCF000192010F0E4FA8046B8F1000F21D1042059
:10FD0000F6F7BEFF4FF4167110FB01F7F81707EB7B
:10FD10001050001300EB4000400004B24748B0F917
:10FD20000000A04201DD204602E04448B0F9000096
:10FD30004249088000204249088032204149086039
:10FD40007AE04048006808B30420F6F799FF4FF4C2
:10FD5000167110FB01F7F81707EB1050001300EBBA
:10FD60004000400004B23648B0F90000A04201DA79
:10FD7000204602E03248B0F900003149088031489D
:10FD80000068401E2F490860BDE8F0810420F6F7A6
:10FD900077FF4FF4167110FB01F7F81707EB1050BF
:10FDA000001300EB4000400004B22548B0F9000009
:10FDB000A04201DA204602E02148B0F900002049C3
:10FDC00008800720F6F75CFF4FF4167110FB01F76F
:10FDD000F81707EB1050001300EB4000400000EB59
:10FDE0008000032190FBF1F005B21548008813490B
:10FDF0000988401A06B2502E07DA0420F8F7E0F816
:10FE000011A10420F8F7ECF802E00420F7F798FFBE
:10FE100040F6C410854204DD502E0ADAB5F57A6F3B
:10FE200007DD0520F8F7CCF80DA10520F8F7D8F884
:10FE300002E00520F7F784FF00BFA5E7703F002030
:10FE4000723F00206C3F00206578636570745F63CB
:10FE500068617267696E675F6368697000000000BF
:10FE60006578636570745F626174746572790000AF
:10FE700010B58AB0002401A84CDF019880100190D1
:10FE800001222146641C02A84254F9F75DFA01469A
:10FE90002246641C02A881540198C2B22146641C07
:10FEA00002A8425400222146641C42542146641C8C
:10FEB00042542146641C42542146641C425440482A
:10FEC000D0F81B00020E2046611CCCB202A90A54D5
:10FED0003B48D0F81B00C0F307422046611CCCB25F
:10FEE00002A90A543648B0F81B00C0F30722204686
:10FEF000611CCCB202A90A543148C27E2046611C62
:10FF0000CCB202A90A5401F0DFF82146621CD4B237
:10FF100002AA505401F0D2F82146621CD4B202AABF
:10FF2000505401F0C5F8020E2046611CCCB202A963
:10FF30000A5401F0BDF8C0F307422046611CCCB260
:10FF400002A90A5401F0B4F8C0F307222046611C4C
:10FF5000CCB202A90A5401F0ABF8C2B22046611C2F
:10FF6000CCB202A90A541648D0F81F00020E20464F
:10FF7000611CCCB202A90A541148D0F81F00C0F38A
:10FF800007422046611CCCB202A90A540C48B0F8C2
:10FF90001F00C0F307222046611CCCB202A90A54FC
:10FFA0000748C27F2046611CCCB202A90A542346EE
:10FFB00002AAA1210020F7F7EBF90AB010BD00005A
:10FFC0000852002010B50446002006E0411C62687B
:10FFD000525C07490A54411CC8B20828F6DBF8F7FE
:10FFE00003FA18B103A10B20F7F7FAFF10BD0000C8
:10FFF00013520020636C6561722073746570206613
:020000040003F7
:1000000061696C0010B50849A120F7F7EBF800F022
:1000100097FA0648007928B9054A06A14FF4FA6014
:10002000FAF7CCFB10BD0000214F0300085200205E
:10003000410003006170705F636C69656E7400005D
:1000400010B516F039FBA0B103200AF089FD401C61
:1000500068B1084801780078401C064A10700429ED
:1000600007DB002011460870FFF702FF01E0FFF7F1
:10007000FFFE10BDA43E002070B504466068807885
:100080006168497840EA01251748D0F82B00B0B1E3
:100090001548D0F82B00401E2821B0FBF1F0401C81
:1000A000124908801048D0F82B00401E2821B0FBD0
:1000B000F1F201FB1200401C0D49088004E0002011
:1000C0000A4908800A49088055B901200949087081
:1000D0000020094908800846008800F00FF802E077
:1000E000284600F0FDF870BD08520020F83D0020C1
:1000F000FA3D0020F53D0020F63D00202DE9F843B3
:1001000005460024F8F742FB691EA02202FB010706
:1001100002222146641C4B484254002007E04A4911
:100120000B5C2146621CD4B2464A5354401C08283A
:10013000F5DB4648008802122046611CCCB24149DA
:100140000A54424802782046611CCCB23D490A5408
:100150002A122046611CCCB23A490A542046611C3E
:10016000CCB238490D54002D2ED102F0ABF88046A8
:1001700002F0AEF808EB000602F0AAF8804602F0A2
:10018000A1F881464B46324631A10020CDF80080CF
:10019000FBF7B4F8320E2046611CCCB229490A5450
:1001A000C6F307422046611CCCB226490A54C6F366
:1001B00007222046611CCCB222490A542046611C09
:1001C000CCB220490E541AE02048008885420DD157
:1001D0002F48008882001B4801193846FDF76CFA49
:1001E0002B48007804EB8000C4B208E015480119E0
:1001F000A0223846FDF760FA04F1A000C4B228231B
:100200002348028823A10020FBF778F82AA10020C8
:10021000FBF774F8002606E00A48825D2CA1002056
:10022000FBF76CF8761CA642F6DB2BA10020FBF74F
:1002300065F82346034AA1212848F7F7A9F8BDE845
:10024000F8830000364F002013520020F83D0020B4
:100250003D3D3D3D3E737465703D25642C6170707D
:100260005F737465705F476574537465705F4C2885
:10027000293D25642C6170705F737465705F4765FC
:1002800074537465705F5228293D25640A0000008C
:10029000FA3D00203D3D3D3D3E6C6173744E756DF1
:1002A0003D25642C5041434B5F535445505F4C45B2
:1002B0004E3D25640A0000006170705F636C6965E3
:1002C0006E745F53656E6453746570416C6C3A0074
:1002D00025303258200000000D0A0000FC3D0020AF
:1002E000F0B5BFB005460024F8F750FA691EA02209
:1002F00002FB010702222146641C0DF801200020A8
:1003000007E02D490B5C2146621CD4B20DF8013088
:10031000401C0828F5DB2948008802122046611C91
:10032000CCB20DF80020254802782046611CCCB2E2
:100330000DF800202A122046611CCCB20DF80020D6
:10034000EAB22046611CCCB20DF800201B480088A0
:1003500085420DD11A48008882000DEB0401384611
:10036000FDF7AAF91648007804EB8000C4B208E053
:100370000DEB0401A0223846FDF79EF904F1A00020
:10038000C4B210A10020FAF7B9FF002606E01DF85C
:10039000062012A10020FAF7B1FF761CA642F6DB78
:1003A00010A10020FAF7AAFF23466A46A1210020E7
:1003B000F6F7EEFF3FB0F0BD13520020F83D0020ED
:1003C000FA3D00206170705F636C69656E745F5305
:1003D000656E64537465704E3A00000025303258E3
:1003E000200000000D0A000070B5A2B04124802159
:1003F0006846F6F75EF800208DF8000000BF05E0C3
:1004000041A10A5C411C0DF80120401C0B28F7D3C8
:1004100020A86DDF054600BF2E4636B100BF3DA2C5
:1004200073213046F5F7F6FE00BF00BF00200AE05A
:10043000C0F105020DF181018B5C2146621CD4B232
:100440000DF80130401C0628F2DB00222046611C1A
:10045000CCB20DF8002001222046611CCCB20DF870
:1004600000202046611CCCB20DF800202046611C03
:10047000CCB20DF800202046611CCCB20DF8002053
:10048000002007E02A490B5C2146621CD4B20DF81B
:100490000130401C0628F5DB25483538006B020E7C
:1004A0002046611CCCB20DF8002021483538006B85
:1004B000C0F307422046611CCCB20DF800201C4856
:1004C0003538008EC0F307222046611CCCB20DF8EF
:1004D00000201748353890F830202146601CC4B2FF
:1004E0000DF801201248353890F834202146601C60
:1004F000C4B20DF8012023466A46A1210020F6F778
:1005000047FF22B070BD0000534D41525420534864
:100510004F4500002E2E5C2E2E5C2E2E5C617070DE
:100520005C6170705F636C69656E742E63000000BF
:100530003D5200200148007870470000F43D002043
:1005400010B5034A03A14FF47A70FAF737F910BDDA
:10055000650503006170705F636C69656E745F733D
:100560007465700010B51F48007820B101280DD0C7
:10057000022830D11BE01C480078012805D1194918
:100580000870FCF707F91949086028E0FCF702F940
:1005900016490968401A42F21071884203D30220BA
:1005A0001049087002E0012000F068FD17E0F8F73C
:1005B000D5FB18B10EA10B20F7F712FDF8F736FDA9
:1005C00018B111A10B20F7F70BFD002006490870A8
:1005D0000449087003E000200249087000BF00BF12
:1005E00010BD0000203E0020F43D0020243E0020ED
:1005F0007361766520696E666F726D6174696F6E86
:10060000206661696C000000736176652073746513
:1006100070206661696C0000012001490870704714
:10062000F43D002010B52A48007810B101284CD1C3
:1006300009E016F041F828B1012025490870002092
:100640002449087042E00BF09DF9C0B121480078C0
:10065000F8B901201F49087000F01AFA1E49087005
:1006600001230A46A3211D48F6F792FEFCF792F8F3
:10067000044622461AA10020FAF740FE09E0154878
:100680000078002805DD0020124908701348F6F7AD
:1006900027FE1F48008870B1FCF77CF81D490968E7
:1006A000401A1B490988884205D300201849088050
:1006B0000320F9F743FB15F0FFFF28B90020044998
:1006C00008700648F6F70CFE00E000BF00BF10BD42
:1006D000D53E0020D43E0020D63E0020A83E00207B
:1006E0003D3D3D3D3D3D3D3D3D3D3D3D3D3D3D3D3A
:1006F0003D3D3D3D3E424C455F486F73745F545FE6
:10070000434F4E4E45545F4C45443A25640A000021
:10071000CC3E0020D03E002010B57748007820B1B4
:10072000012821D0022875D175E0FFF703FF30B909
:1007300015F0C2FF18B9FFF7A5F9012813D001F091
:10074000BBF880B96DA10020FAF7D8FD0121AFF206
:100750003700FAF70FF814F0CFFD00206C4908605D
:10076000012065490870C5E0FFF7E4FEC8B915F03F
:10077000A3FFB0B9FFF786F9012812D165A10E20B9
:10078000F7F72EFC6AA10020FAF7B8FD0FF0ADF9DB
:100790000021AFF27B00F9F7EDFF00205649087009
:1007A00016E00BF0EFF898B168A10020FAF7A6FD6B
:1007B0000021AFF29B00F9F7DDFF6A48007920B114
:1007C0000020694908806949087002204A49087078
:1007D0004F480068401C4E490860642819D3FFF751
:1007E000A9FE40B95F4890F82F00432803D160A1CB
:1007F0000F20F7F7F5FB65A10020FAF77FFD0FF05A
:1008000074F90021AFF2EF00F9F7B4FF00203A4984
:1008100008706FE06AE003200AF0A2F9401C18B3E8
:1008200052480078022842D04F4800883C283EDCDD
:10083000F1EE0E0AB1EE0E0AF7F726F830B90220F3
:100840004A49087000204849088030E0464800883E
:100850003C2803D157A10F20F7F7C2FB424800887C
:10086000401C4149088022E04048007801281ED001
:100870003D4800883C281ADCDFED570A9FED560AF8
:10088000F7F702F830B901203849087000203649DE
:1008900008800CE0344800883C2803D14FA10F2089
:1008A000F7F79EFB30480088401C2F490880FFF76F
:1008B00041FE58B915F000FF40B9FFF7E3F80128F1
:1008C00004D10BF05FF808B10BF014F80BF05AF8F4
:1008D00058B94BA10020FAF711FD0021AFF2C71063
:1008E000F9F748FF00200449087003E0002002499E
:1008F000087000BF00BF10BDD73E00203D3D3D3D0C
:100900003D3D3D3E7363616E5F73746172740A00B6
:10091000D83E002061647620646973636F6E6E74E4
:100920006564206F7665722074696D650000000053
:100930003D3D3D3D3D3D3D3E6E72665F626C655F97
:100940007363616E5F73746F700A00003D3D3D3DDF
:100950003D3D3D3E686F73745F6973636F6E6E6596
:1009600063740A0008520020DC3E0020DE3E0020B6
:100970007363616E2072696768742073686F657352
:10098000206F7665722074696D6500003D3D3D3DC8
:100990003D3D3D3E6170705F6572725F53657420CE
:1009A0006E72665F626C655F7363616E5F73746FB6
:1009B000700A000075706461746520426C65206384
:1009C0006F6E6E20696E74657276616C20372E359D
:1009D0006D73206661696C000000C84275706461C7
:1009E000746520426C6520636F6E6E20696E74655D
:1009F0007276616C203130306D73206661696C00F5
:100A00003D3D3D3D3D3D3D3E686F73745F646973A0
:100A1000636F6E6E6563740A0000000010B50E48C7
:100A2000007920B10D4A0EA16420F9F7C7FE0F48E6
:100A3000F6F7F2FE0E48F6F7B7FE0E4A0EA1642056
:100A4000F9F7BCFE1049A320F6F7CCFB0F49AC2008
:100A5000F6F7C8FB10BD000008520020190703007C
:100A60006170705F636F6E6E656374004552030062
:100A700001520300250603006170705F636F6E6EA4
:100A80006563745F6C656400914B0300D94B030090
:100A900010B50024064890F82F00432801D0022406
:100AA00003E00AF06FFF00B10124204610BD0000F2
:100AB0000852002010B5054A05A10020F9F77EFE76
:100AC0000A48F6F78DFD002010BD0000F10A030072
:100AD0006170705F646174615F7472616E7366658A
:100AE000725F50726F63657373000000D10B030077
:100AF00010B503200AF034F8401C28B904200AF08D
:100B00002FF8401C002836D02048007830B9012149
:100B10001F48F9F72FFE01201C490870FBF73AFE29
:100B20001C490968401AB0F5FA7F16D3FBF732FE6C
:100B30001849086015F0C0FD38B917A10020FAF770
:100B4000DDFBFEF77DFDFEF759FD1F48007920B162
:100B50000AF018FF08B914F0CFFBFBF71BFE1B4986
:100B60000968401A032810D3FBF714FE17490860E0
:100B7000F8F7D6FD09E00548007830B100210448B7
:100B8000F9F7F8FD00200149087010BD603F002012
:100B9000F10A0300583F00206170705F6461746166
:100BA0005F7472616E736665725F50726F636573B6
:100BB00073206164766572746973696E675F7374BC
:100BC0006172740D0A000000085200205C3F002092
:100BD00070B504460D46E078042803D12946204626
:100BE000F8F75CFE00F08EF970BD00002DE9F047CB
:100BF00004460D461646324629462046F8F77AF94D
:100C00001CA10020FAF77AFB142001210A460023D8
:100C10001F469C4600BF4FF0A049C84641EA420922
:100C200049EA830949EA072949EA0C4908F5E06AD3
:100C30004AF8209000BF00BF002159B900BF00BF93
:100C400082061346012707FA00F2C3F80C2500BFFD
:100C500000BF0CE000BF00BF4FF0A04213460127C9
:100C600007FA00F2C3F8082500BF00BF00BF00BFAD
:100C7000BDE8F0876170705F6572726F725F666168
:100C8000756C745F68616E646C65722C53797374F3
:100C9000656D2072657365740A00000010B5084A1E
:100CA00008A14FF47A70F9F789FD0949A220F6F7F7
:100CB00099FA084A08A14EF66020F9F77FFD10BDA9
:100CC000E90C03006170705F67616D6500000000F2
:100CD000494D0300F1F602006170705F4175746F59
:100CE0004F757467616D650010B55648007800282F
:100CF00004DD54480078401E52490870524800787C
:100D000010B1012829D129E0032009F029FF401C56
:100D100000BB4C48C078012811D1012103200AF002
:100D200099F94A480078401CC0B248490870142814
:100D300005DB0020087046A10920F7F751F941486A
:100D40000078002809DD4948007930B1002000F022
:100D5000E3F802E001203C49087071E04348007963
:100D600000283CD00AF00EFE10B336480078A0B937
:100D7000012000F0D1F835480078401CC0B233495A
:100D800008700A2810DB0020087039A1FAF7B6FABB
:100D90003FA10920F7F724F906E02C480078002845
:100DA00002DD00202949087000202649487016E01D
:100DB000244841784078401C224A50700A290EDDB0
:100DC00000201146C870214908701F490870002191
:100DD00003200AF03FF934A10920F7F701F9194877
:100DE000C07870B9002019490870174908700021AF
:100DF00003200AF02FF91D48007910B1002000F0FF
:100E00008BF815F059FCB8B90E4881788078401CF1
:100E10000C4A9070052912DD00201146C8700B495C
:100E2000087009490870002103200AF013F92AA16B
:100E30000920F7F7D5F802E000200249887000BFCA
:100E400000BF10BD8A3E0020903E00208F3E002053
:100E500073686F657320696E746F2067616D6520BC
:100E60006D6F6465206661696C00000008520020A7
:100E70004552525F4E554D5F47414D452061707060
:100E80005F67616D655F50726F636573730D0A0014
:100E90006E6F206765742072696768742073686F6D
:100EA0006573206461746100496E2067616D65201F
:100EB0006D6F64652C72696768742073686F657301
:100EC00020646973636F6E6E746564206C6F6E6707
:100ED0002074696D65000000496E2067616D6520B2
:100EE0006D6F64652C636C69656E742064697363EF
:100EF0006F6E6E746564206C6F6E672074696D65CB
:100F00000000000003480078032802D003200149B4
:100F1000087070478A3E002038B5044600940123CB
:100F20006A46A2210020F6F70FFC38BD00B589B053
:100F30004D48007830B1012821D002284AD003283A
:100F40001CD17DE0032009F00BFEB0F1FF3F15D16D
:100F500046480078012811D101214548F9F70AFCDB
:100F6000012105200AF076F801203F490870002091
:100F70003E490870FBF70EFC3E49086071E0052011
:100F800009F0EEFD70B90220374908700A2138488F
:100F9000F9F782FC002038490880FBF7FBFB354954
:100FA00008600FE0FBF7F6FB32490968401A47F288
:100FB0003051884206D3FBF7EDFB2E490860032031
:100FC00029490870032009F0CBFD10B903202649F8
:100FD000087046E0002009F0BDFD01281CDB01AAD5
:100FE0000021084609F0ACFDBDF80A00ADF81C0070
:100FF000BDF80C00ADF81E00BDF80E00ADF82000E5
:101000001D48B0F9001007A807F020FA1A48008818
:10101000401C00B218490880FBF7BCFB1549096861
:10102000401A42F21071884202D303200E49087020
:10103000032009F095FD10B903200B49087010E05A
:101040004FF47A710A48F9F727FC002105200AF0CD
:1010500001F800210648F9F78DFB002002490870CD
:1010600000BF00BF09B000BD003F0020F83E0020D7
:101070002D0F0300043F0020023F002010B504465E
:101080000123094AA1210020F6F75EFB07480078FA
:1010900040B9022C06DB054804700123024AA12155
:1010A000F6F752FB10BD0000793E0020543E0020B0
:1010B00001480068704700002C3E0020014800787D
:1010C00070470000293E002001480078704700006A
:1010D000283E002010B504480079012803D10349B7
:1010E000A120F6F753FA10BD08520020B5500300B6
:1010F00010B50548007928B1044A05A14FF47A706B
:10110000F9F75CFB10BD00000852002069A0020046
:101110004C6F73735061636B5F70726F6365737351
:101120000000000030B58BB00025012009F018FD4B
:10113000401C002841D0042009F012FD401C00286A
:101140003BD109F007FD05B2002433E001AA214696
:10115000002009F0F5FCBDF81000ADF81C00BDF84A
:101160001200ADF81E00BDF81400ADF82000BDF867
:101170000400ADF82400BDF80600ADF82600BDF867
:101180000800ADF82800BDF9281007A805F018FAE6
:1011900001280ED10A48D0F81B00401C0849C1F8AC
:1011A0001B000846D0F81B2006A10020FAF7A6F87D
:1011B00002E0641CAC42C9DB00BF0BB030BD0000D4
:1011C000085200204461696C79537465702063751E
:1011D0007272656E7420737465703A25640D0A002E
:1011E00038B500251D4804681D480068844201D2B6
:1011F00004F180741A480068201A1A4909680844E2
:101200001849086008460068C50B1748854207D38F
:1012100013480095224615A103680020FAF76EF8DE
:10122000B4F1807F04D9A4F180700D49086001E019
:101230000B480460B5F5616F0ED3FFF7EDF901209F
:10124000134908700020074908602B46084611A181
:1012500002680020FAF752F838BD000004B50040DB
:10126000FC3E0020F43E0020D0FB01002121212182
:101270002121212121212121212121207365632088
:101280006F7665722C25642C25642C25640A000079
:10129000F83E002074696D65434E54282564292862
:1012A0002564290A0000000010B50A4A0AA164203A
:1012B000F9F784FA0F4809F0FFF80F4A0FA14FF42D
:1012C000FA70F9F77BFA134A13A14FF47A70F9F721
:1012D00075FA10BD251103006170705F6D6174684F
:1012E0005F4461696C79537465705F50726F6365B8
:1012F00073730000291303002D0F03006170705FEA
:101300006779726F5F4669785F70726F6365737338
:1013100000000000E11103006170705F6D6174688E
:101320005F486F7572000000F0B587B006460F4643
:101330000025032009F014FC401C00287DD00AF091
:10134000E5FA404285490870002009F003FC05B227
:10135000142D00DC0EB907B0F0BD002448E001AA4E
:101360002146002009F0ECFBBDF80A0004EB440123
:101370007B4A22F81100BDF80C0004EB440102EB9B
:1013800041014880BDF80E0004EB440102EB41012D
:101390008880BDF8040004EB4401724A22F8110071
:1013A000BDF8060004EB440102EB41014880BDF8A2
:1013B000080004EB440102EB41018880BDF81000F5
:1013C00004EB4401684A22F81100BDF8120004EB56
:1013D000440102EB41014880BDF8140004EB4401D4
:1013E00002EB410188806149069841F82400641CA1
:1013F000AC42B4DB012009F0ADFB01280EDB01AAF1
:101400000021012009F09CFBBDF81000584908801C
:10141000BDF812004880BDF8140088805548007956
:1014200020B1284612F034FE0CE006E0FAF724FA68
:1014300040B1284612F02CFE04E000204E490880FE
:1014400015F038F8042009F08BFB401C00287CD0F4
:101450000AF05CFA404241490870002009F07AFB2A
:1014600005B2142D00DC06B975E7002448E001AA96
:101470002146002009F064FBBDF80A0004EB44019A
:10148000374A22F81100BDF80C0004EB440102EBCE
:1014900041014880BDF80E0004EB440102EB41011C
:1014A0008880BDF8040004EB44012E4A22F81100A4
:1014B000BDF8060004EB440102EB41014880BDF891
:1014C000080004EB440102EB41018880BDF81000E4
:1014D00004EB4401244A22F81100BDF8120004EB89
:1014E000440102EB41014880BDF8140004EB4401C3
:1014F00002EB410188801D49069841F82400641CD4
:10150000AC42B4DB012009F025FB01280EDB01AA67
:101510000021012009F014FBBDF8100014490880D7
:10152000BDF812004880BDF8140088800D4A1049AB
:101530000D48F9F76BFB40B10E48D0F81B00401C7A
:101540000C49C1F81B00084600E005E0D0F81B205C
:101550000AA10020F9F7D2FE00BFFCE6E63E00201B
:10156000A850002030500020205100209851002029
:10157000E03E002008520020E83E00203D3D3D3D79
:101580003D3D5265616C54696D65537465703D3DB8
:101590003D3D3D737465702025640D0A0000000018
:1015A00070B50E486DDF044600BF254635B100BF5B
:1015B0000BA2AE212846F4F72DFE00BF00BF0E4A55
:1015C0000EA10020F9F7FAF81049A620F5F70AFE57
:1015D0000F49A620F5F7DAFF70BD0000943E002009
:1015E0002E2E5C2E2E5C2E2E5C6170705C617070F5
:1015F0005F6F74612E630000151603006170705FE9
:101600006F74615F50726F6365737300A54C030064
:101610001550030010B58AB0002005906D48007881
:1016200020B1012864D002286FD184E06A48007993
:1016300000281ADD69480078012858D168A10020E7
:10164000F9F75CFE0120634908700AF053F90EF0C7
:101650004CFA4EF660216748F9F71EF9012305AAF6
:10166000A6210020F5F794FE41E0634800680128B8
:101670003DD100206049086015F01EF810B114F04B
:10168000E3FF01E0FDF7DCFF0020069007900890E3
:1016900009905A48407859498A78C978574B1B793C
:1016A000CDE90031CDE9022054484379827954A133
:1016B00006A8FCF713FA06A8F4F706FF044606ABE3
:1016C000224656A10020F9F719FE06A8F4F7FCFE01
:1016D0000446214606A814F0F5FF14F0ADFF0120E2
:1016E0003C4908704FF4FA614248F9F7D5F86DE0CB
:1016F00039480079002809DD00203849087035494B
:1017000008704BA1F9F7FAFD14E057E014F0D4FF8C
:1017100070B94DA10020F9F7F1FDFDF76FFF4EF60E
:1017200060213448F9F7B8F802202A49087001E02E
:1017300014F08AFF4AE014F0BFFF10B100202549E1
:10174000087000212B48F9F7A7F8FDF779FF002072
:1017500006900790089009901F4890F83A1090F86A
:10176000392090F838001C4BDB79CDE90030CDE909
:1017700002211948837942793CA106A8FCF7AEF909
:1017800006A8F4F7A1FE044606AB22463EA10020BF
:10179000F9F7B4FD06A8F4F797FE0446214606A81B
:1017A00014F090FF3DA10E20F6F71AFC14F044FF50
:1017B000FDF724FF00200749087007E000200549D5
:1017C000087000210B48F9F767F800BF00BF0AB0A6
:1017D00010BD0000A33E002008520020A03E0020C3
:1017E0002D2D2D2D2D2D3E6973486F73744F54414F
:1017F0000A000000151603009C3E0020943E0020C5
:1018000053485F253032582530325825303258251C
:101810003032582530325825303258004F5441204C
:101820006E616D65282564293A25730A0000000061
:101830002D2D2D2D2D2D3E6C656674206F75742019
:10184000746F206466750A006170705F6F74615F09
:1018500050726F6365737320616476657274697327
:10186000696E675F73746172740D0A0025303258B7
:1018700025303258253032582530325825303258EC
:101880002530325800000000414456206E616D65DD
:10189000282564293A25730A000000006164762037
:1018A000646973636F6E6E746564206F7665722011
:1018B00074696D6500000000014800787047000001
:1018C000A03E002010B50A48007800280BDD012357
:1018D000084AA6210020F5F75BFD05480078401E68
:1018E0000349087002E00448F8F7BAFF10BD000091
:1018F000A13E0020A23E0020C518030010B5064AF4
:1019000006A14FF47A70F8F759FF074A07A14FF480
:101910007A70F8F753FF10BD69F702004261744412
:10192000697370616C79000039F902004261744496
:10193000697370616C795F4E0000000070B50E48ED
:101940006DDF044600BF25463DB100BF0BA24FF43A
:1019500098712846F4F75EFC00BF00BF0D4A0EA147
:101960006420F8F72BFF11490120FBF7CFF810494D
:101970000220FBF7CBF870BD0C3F00202E2E5C2E12
:101980002E5C2E2E5C6170705C6170705F7061699E
:10199000722E6300B51903006170705F7061697227
:1019A0005F50726F6365737300000000C5530300DE
:1019B0008552030030B589B0FEF764F801282FD0B6
:1019C000A7480078012811D0A648007928B1A64A76
:1019D00013210846FBF708F804E0A34A1321162058
:1019E000FBF702F801209E4908702CE09F48008810
:1019F000322828DA9D480088401C9C490880994874
:101A0000007900B3984A13210846FAF7EDFF012048
:101A1000FAF742FF944A13211620FAF7E5FF12E085
:101A20008F480078022807D013210846FBF76EF98B
:101A300002208B49087006E08C480088002802DDEF
:101A400000208A49088000248948007810B10128C4
:101A50007AD168E087480078002863D04320814924
:101A600081F82F0024217F480B30F4F722FD4FF43A
:101A7000FA70F8F757FB00207E49087001207C4976
:101A8000087000240CE07748401D015D7A4801553C
:101A900074483530015D7848801D0155601CC4B222
:101AA000062CF0DB6F48006B7349091F08616D4815
:101AB00090F8340008756B4890F82F004875F7F7D8
:101AC0004DF918B16DA10C20F6F78AFAF7F72AF94B
:101AD00018B170A10C20F6F783FAF7F7A7FA18B13E
:101AE00071A10B20F6F77CFA5E4890F83A1090F856
:101AF000392090F8383090F83700CDE90132039161
:101B00000090584890F8363090F835206AA10020AF
:101B1000F9F7F4FB76A10020F9F7F0FBFAF73AFEAB
:101B20007A49086098E0FAF735FE78490968401A62
:101B300042F2107188420BD3FAF72CFE7349086009
:101B400000204B49087000E082E071A1F9F7D6FB54
:101B50004448007900283CD009F014FF10B109F086
:101B6000C9FE74E06FA10020F9F7C8FB00200590C2
:101B70000690079008903B4890F83A1090F839206A
:101B800090F83800374BDB79CDE90030CDE9022100
:101B90003448837942796AA105A8FBF79FFF05A81D
:101BA000F4F792FC054605AB2A466CA10020F9F734
:101BB000A5FB05A8F4F788FC0546294605A809F009
:101BC000E7FEF9F727FEF9F701FE00202849087023
:101BD0003DE014F071FD10B114F036FD37E0002047
:101BE00005900690079008901E4890F83A1090F8DB
:101BF000392090F838001B4BDB79CDE90030CDE976
:101C000002211848837942794DA105A8FBF766FFA8
:101C100005A8F4F759FC054605AB2A4654A1002057
:101C2000F9F76CFB05A8F4F74FFC0546294605A813
:101C300014F048FDFDF704FD14F0FEFC50A1002057
:101C4000F9F75CFBFDF7DAFC00200949087003E0B6
:101C500000200749087000BF00BF09B030BD000078
:101C6000203F00200852002090D00300143F0020A5
:101C7000213F0020163F00208452002073617665CA
:101C800020696E666F726D6174696F6E206661693E
:101C90006C00000073617665206261636B75702073
:101CA0006661696C0000000073617665207374657D
:101CB00070206661696C00006D466C6173682E6D02
:101CC000436C69656E742E6D6163416464723A257C
:101CD00030325820253032582025303258202530D7
:101CE0003258202530325820253032580A00000062
:101CF0003E3E3E3E3E3E3E3E506169725F737461C1
:101D00007465203D31200D0A00000000243F0020B2
:101D1000506169725F7374617465203D30200D0AF3
:101D2000000000003E3E3E3E3E53545F7363616ED2
:101D30005F7374617274203D30200D0A0000000052
:101D40002530325825303258253032582530325817
:101D50002530325825303258000000007363616E20
:101D60004E616D65282564293A25730A000000003C
:101D70006164764E616D65282564293A25730A00F1
:101D80003E3E3E3E3E3E3E3E616476657274697301
:101D9000696E675F7374617274203D30200D0A00B4
:101DA00010B5034A03A142F21070F8F707FD10BD09
:101DB000C91D03006170705F736166655F50726F6B
:101DC000636573730000000010B50B48807D002828
:101DD00011DD0A480078401C084908700846007860
:101DE000062808DB002004498875F6F79BFF04A14C
:101DF0000020F9F783FA10BD80520020613F0020D7
:101E0000636C656172206D4261636B75702E457203
:101E1000726F725374617274466C61670A000000DD
:101E200010B5002400BF04E0002149480155601CA2
:101E3000C4B2062CF8DB0020454908398873062017
:101E4000F5F7A8FF38B10121414808384173062051
:101E50003F49083988730120F5F79CFF18B101202C
:101E60003B49083908720220F5F794FF18B10120A8
:101E70003749083908720320F5F78CFF18B10120A3
:101E80003349083908720120F5F784FF38B9022078
:101E9000F5F780FF18B90320F5F77CFF18B1012092
:101EA0002B49083988730020F5F774FF38B10121F8
:101EB00027480838417202202549083988730520CF
:101EC000F5F768FF38B101212148083881720320F5
:101ED0001F49083988730420F5F75CFF38B10121E8
:101EE0001B480838C1720420194908398873072033
:101EF000F5F750FF38B10121154808380173052066
:101F000013490839887312480838807B70B1002063
:101F10000F490839C873FAF73DFC0D4908390861C3
:101F2000FAF738FC0A49083948610FE000200849EF
:101F30000839C8730748007820B107490620F7F729
:101F4000E1FE03E005490620F7F7DCFE10BD0000C6
:101F5000F05100203C3F0020FF0000FF070700FF7A
:101F600010B5002009490870486088730120C873C3
:101F7000002008614861087742F210708861044AC5
:101F800004A10A20F8F71AFC10BD0000E851002057
:101F9000B11F03006170705F73656C665F63686595
:101FA000636B696E675F50726F63657373000000E7
:101FB00010B59148007820B101282DD0022868D1B1
:101FC00058E0FDF75FFD032803D0FDF75BFD022815
:101FD00021D1F5F7E9FEA0B1022008F0C1FD401CB7
:101FE00020B10021022009F035F814E0F9F7EEFBEA
:101FF000F8F7C4FD01208049087000207F4908706F
:1020000009E0F9F7E3FBF8F7B9FD01207A49087018
:1020100000207A4908703DE07948007F01280DD101
:102020007749087002207449087001217548F8F753
:10203000A1FB75A10020F9F761F91AE0FAF7AAFBF4
:102040006F498969401A42F21071884211D9022001
:102050006949087000206A490877032067490870B9
:10206000714807F08FFEF9F7D5FB70A10020F9F752
:1020700045F90FE0FDF706FD012809D100205E4972
:1020800008707448FDF7CEFC73A10020F9F736F90B
:1020900000E000BF00BF5948007830B101281ED0D1
:1020A00002284DD0032875D188E0554800780128D2
:1020B00014D14FF4FA70F8F735F8022008F050FD0B
:1020C000B0F1FF3F03D10121022008F0C3FF01203E
:1020D0004A490870FAF75EFB4949486089E0FDF714
:1020E000D1FC012803D103204449087027E00220D5
:1020F00008F036FD40B902204049087000206349CD
:102100000870FFF78DFE1AE0FAF744FB3C49496876
:10211000401A44F62061884211D30120F5F750FFA0
:102120000220F5F74DFF0320F5F74AFF0620F5F7EB
:1021300047FF02203149087000205449087058E0D8
:102140002F48807B51490978884224DDFAF722FB29
:102150002B494969401AC8282FD3FAF71BFB284995
:1021600048610846C07B38B949490620F7F7CAFDDF
:1021700001202349C87320E04FF07F410620F7F784
:10218000C1FD00201E49C87340480078401C3F49EB
:10219000087012E02CE0FAF7FDFA19490969401AB3
:1021A00040F6B831884208D3FAF7F4FA14490861C6
:1021B000002036490870FFF733FE1AE000200F496F
:1021C00008700F4908704FF07F410620F7F79AFD1D
:1021D0000620F7F7B3FD01200949C873022008F073
:1021E000BFFC401C18B10021022008F033FF00E0C2
:1021F00000BF00BF10BD0000443F0020453F00204D
:10220000E8510020B11F03006F625F73656C665F69
:10221000636865636B2E69735F7363616E5F73756B
:1022200063636573730D0A002C3F00206F625F7358
:10223000656C665F636865636B2E7363616E5F7464
:102240007269676765725F74696D656F75740D0A91
:10225000000000003C3F00206F625F73656C665FAA
:10226000636865636B2E7363616E20424C455F4308
:102270006C69656E745F545F4348415247455F50D7
:10228000554C4C4F55540D0A00000000463F0020AD
:10229000000007FF10B50446022C00D101E0012028
:1022A00010BD00BF02A10020F9F728F80120F7E7D0
:1022B000496E746F20626F6F746C6F616465720A2F
:1022C000000000000148D0F81B00704708520020B1
:1022D0000148D0F81F0070470852002010B50B4885
:1022E000007920B90A4A0BA16420F8F767FA0D4A71
:1022F0000DA14FF47A70F8F761FA1049A520F4F7B0
:1023000071FF0F49A520F5F741F910BD08520020D3
:10231000E1230300737465705F5265616C53656EF1
:102320006400000045230300737465705F526561AB
:102330006C436F6E6E65637400000000D94D03003E
:102340007150030008B5042008F00AFC401C98B343
:1023500020480078FF2804DA1E480078401C1D49F8
:1023600008701C4800783C2813DB0021042008F08A
:1023700071FE1948007800282BDD002016490870EE
:102380000220009001236A46A5210020F5F7DCF920
:102390001FE011480078002804DD0F480078401E37
:1023A0000D4908700C48007898B901230B4AA52103
:1023B0000020F5F7C9F90CE0FFE70748007800288E
:1023C00007DD0020044908700123044AA521F5F720
:1023D000BBF908BD893E0020883E00207C3E0020DD
:1023E0001CB5042008F0BCFBB0F1FF3F58D000241E
:1023F00001222146641C0DF801202A48D0F81B0058
:1024000029490968401A020E2146641C0DF8012072
:102410002448D0F81B0024490968401AC0F3074239
:102420002146641C0DF801201E48B0F81B001E490F
:102430000988401AC0F307222146641C0DF80120C8
:102440001848C07E18490978401AC2B22146641C57
:102450000DF8012015480068020E2146641C0DF895
:10246000012012480068C0F307422146641C0DF8A1
:1024700001200E480088C0F307222046611CCCB220
:102480000DF80020094802782046611CCCB20DF8F6
:10249000002023466A46A5210020F4F779FF00BFFB
:1024A0001CBD000008520020803E0020843E002019
:1024B00010B50249AB20F4F795FE10BDD54E0300D0
:1024C00010B5024805F08EFC10BD0000C04A002087
:1024D00010B503460C460AB9072010BD19684A61B9
:1024E000012C01D1012000E0002008610020F4E768
:1024F00038B5134800680090082358221149124843
:1025000000680CF098FD04460CB1204638BD0F4A17
:1025100069460F4805F06CFC04460CB12046F5E70F
:1025200001210B4805F0D6FC01230A4A1946084848
:1025300005F02AFC0120084908702046E6E7000063
:1025400010850400E88B002000850400694E04001B
:10255000C04A0020FFFF7F00CC4A00202DE9F04157
:1025600006460D4617463446207F10B10020BDE8D0
:10257000F081A76107F086FA401941F10001C4E932
:102580000201206900B125612146002014F00EFFF0
:10259000EDE770B50446254600202877294601203E
:1025A00014F004FF70BD10B50446204612F05AFF27
:1025B00010BD000070B5044625460E488068B0B1D5
:1025C000ADB9FCF7B1FC06460A4800680A49086044
:1025D000084840684FF0E021C1F804010020054997
:1025E00088601EB900BF62B600BF00BF00BF00BF59
:1025F00070BD0000308A002000E100E0F8B505461B
:102600000C4617462088001DB84201D90C20F8BDA1
:10261000684679DF064600BF304600B1F7E700BFE5
:102620000320218868542088401C2080192021889C
:1026300068542088401C208020884119BDF8000083
:1026400014F0F5FE2188084420800020DFE770B5F3
:1026500004460D4620460AF027FE70BD10B541EC39
:10266000100BFBF7A1FC51EC100B10BD2DE9F04154
:102670002DED028B04460E4617461D46B0EE408AED
:10268000B0EE000A86ED000A95ED020A20EE080A77
:1026900086ED010A95ED010AF1EE480A20EE200AC6
:1026A00086ED020A95ED020AF1EE480A20EE200AB4
:1026B00086ED030AB0EE000A86ED040A95ED000AE5
:1026C00020EE080A86ED050A95ED010A20EE080ABB
:1026D00086ED060A95ED000AF1EE480A20EE200A82
:1026E00086ED070AB0EE000A86ED080A3946304644
:1026F0000AF0CCF824213046F3F7DBFE94ED010A12
:1027000020EE080AD5ED020A20EE200AD4ED000AD8
:10271000B0EE001A01EE200AD4ED020A60EE880A3B
:1027200095ED011A00EEC10A86ED000A94ED010A4A
:10273000F0EE000A20EE200AD4ED000A60EE880ACE
:1027400095ED021A00EEC10AD4ED020A60EE880A85
:1027500095ED001A00EE810A86ED010A94ED000A5B
:1027600020EE080AD5ED010A20EE200AD4ED020A77
:10277000B0EE001A01EE200AD4ED010A60EE880ADC
:1027800095ED001A00EEC10A86ED020A94ED040AE6
:1027900020EE080AD5ED020A20EE200AD4ED030A45
:1027A000B0EE001A01EE200AD4ED050A60EE880AA8
:1027B00095ED011A00EEC10A86ED030A94ED040AB4
:1027C000F0EE000A20EE200AD4ED030A60EE880A3B
:1027D00095ED021A00EEC10AD4ED050A60EE880AF2
:1027E00095ED001A00EE810A86ED040A94ED030AC5
:1027F00020EE080AD5ED010A20EE200AD4ED050AE4
:10280000B0EE001A01EE200AD4ED040A60EE880A48
:1028100095ED001A00EEC10A86ED050A94ED070A4F
:1028200020EE080AD5ED020A20EE200AD4ED060AB1
:10283000B0EE001A01EE200AD4ED080A60EE880A14
:1028400095ED011A00EEC10A86ED060A94ED070A1D
:10285000F0EE000A20EE200AD4ED060A60EE880AA7
:1028600095ED021A00EEC10AD4ED080A60EE880A5E
:1028700095ED001A00EE810A86ED070A94ED060A2E
:1028800020EE080AD5ED010A20EE200AD4ED080A50
:10289000B0EE001A01EE200AD4ED070A60EE880AB5
:1028A00095ED001A00EEC10A86ED080A2246394667
:1028B00030460CF086F8BDEC028BBDE8F08110B517
:1028C0000446637903F00302217920880AF0A9FC09
:1028D00010BD10B50446207918B9204600F008F85C
:1028E00003E02046FFF7EBFF00BF00BF10BD000074
:1028F0002DE9FC41064637884FF000080022444885
:102900000178384600F084FC7079C0F3800028B963
:102910000021304610F01EFBBDE8FC8107F58071F8
:1029200088B26B460122072110F0C2FB054645B173
:102930002946384613F05CFB0021304610F00AFBB4
:10294000EAE7384609F016FA04464FF6FF718C4262
:102950001BD1019809F05EF904464FF6FF708442DE
:1029600013D02146384609F0E3F93846FCF7B6FEA5
:1029700058B9384613F0C2FA3846FCF7AFFE20B912
:102980000021304610F0E6FAC6E74FF6FF708442A9
:1029900015D110F025FD04464FF6FF70844208D192
:1029A0000421384613F024FB0021304610F0D2FAFF
:1029B000B2E72146384609F0BBF94FF0010807F5A8
:1029C000807188B22246072110F0E8FB054625B940
:1029D0000121304610F0BEFA17E0862D07D13846A7
:1029E00013F0CCFA0121304610F0B4FA0DE029467C
:1029F000384613F0FDFA0021304610F0ABFAB8F17A
:102A0000000F02D0204609F09DF900BF84E70000C6
:102A1000404A002010B5034693ED002AB0EE420A6A
:102A200093ED002AF0EE420A91ED002AB0EE421A30
:102A300091ED002AF0EE421A01203CE003EB800405
:102A400094ED002AB4EEC02AF1EE10FA05DD03EB96
:102A5000800494ED002AB0EE420A03EB800494ED6A
:102A6000002AB4EEE02AF1EE10FA05D203EB80045E
:102A700094ED002AF0EE420A01EB800494ED002A66
:102A8000B4EEC12AF1EE10FA05DD01EB800494EDFD
:102A9000002AB0EE421A01EB800494ED002AB4EE55
:102AA000E12AF1EE10FA05D201EB800494ED002A40
:102AB000F0EE421A401C9042C0DB9FED0B2A30EE34
:102AC000822AB4EEC02AF1EE10FA08D39FED062A4E
:102AD00031EE822AB4EEC12AF1EE10FA01D20120C1
:102AE00010BD0020FCE700009A99993E2DE9F041C5
:102AF00004460F46154615B90E20BDE8F0810020AA
:102B0000286000BF0CB90E20F7E700BF00BF2068A7
:102B100008B90E20F1E700BF00BFE088C11700EB45
:102B200091718910A0EB810109B10720E5E700BF91
:102B3000384600F0DDFAC6B2142E01D10520DCE7DC
:102B40002079B04201DC0420D7E7E188206806FB49
:102B5000010028600020D0E72DE9FC4105468846A9
:102B60001646002437880020308095F82D0058B193
:102B70003A463146404600F00FFC044600BF20466E
:102B800008B1BDE8FC8100BFA87850B13A46314693
:102B90004046FFF733FD044600BF204600B1F0E792
:102BA00000BFE87860B1E97848B23B46324641461A
:102BB00005F0F8FE044600BF204600B1E1E700BF83
:102BC000686868B1696891F900003B463246414641
:102BD00014F00CFC044600BF204600B1D1E700BF52
:102BE000288900280EDD43460622022105F108004F
:102BF000CDE9006714F0C6FC044600BF204600B1D2
:102C0000BFE700BF288A00280EDD434607220321C4
:102C100005F11000CDE9006714F0B4FC044600BFD4
:102C2000204600B1ADE700BF288B00280EDD4346EB
:102C30001522142105F11800CDE9006714F0A2FC5B
:102C4000044600BF204600B19BE700BF286A58B188
:102C50003B4632464146286A02F0C5FF044600BFA3
:102C6000204600B18DE700BF686A58B13B46324646
:102C70004146686A0BF046FA044600BF204600B1A0
:102C80007FE700BF95F82C0000280BDD3B4632465D
:102C90004146284613F0D4FA044600BF204600B14E
:102CA0006FE700BF287858B13B4632464146284678
:102CB0000BF06FFF044600BF204600B161E700BF84
:102CC00020465EE72DE9F843064688461546002073
:102CD00000900DB9BDE8F88309236A4641463046A5
:102CE00000F02BF80446BDF800003718BDF80000CE
:102CF00068B164B12846F3F7E7FBA04207D122464A
:102D000039462846F3F7F5FB08B90120E2E7002031
:102D1000E0E7F8B504460E461546002000902B4625
:102D20006A463146204600F008F807460FB90020F1
:102D3000F8BDBDF800002044FAE7F0B504460D46A2
:102D40001E4604B10AB90020F0BD002103E0605C1A
:102D5000401C084481B2481CA84206DA1088884208
:102D6000F5DC481C205CB042F1D1A94201DB002017
:102D7000EAE7881C87B2605C10B1605C401E00E02E
:102D8000002083B213B1F818A84201DD0020DBE770
:102D900017801846D8E780F83010704770B50446A1
:102DA0000D4605B10CB90E2070BD05F1780002F09A
:102DB00032FE08B90720F7E70020A0702C2205F1A9
:102DC0007801201DF3F75CFB002084F83000D5F873
:102DD000A4006063D5F8A800A0634FF6FF70A4F8C4
:102DE000240404F58260C4F82004002140F22C4041
:102DF000C4F82614A4F82A140155207810B9FF202D
:102E000084F8540004F15500C4F810042046FCF77F
:102E10008DFB40F21441085304F2144204F15501B1
:102E20002846FFF799FE064600BF304600B1BBE7D3
:102E300000BF04F231204FF4836108512046FCF7B3
:102E400075FBA4F81C044FF48360015904F21C4282
:102E500005F13C00FFF780FE064600BF304600B19A
:102E6000A2E700BF012151200155208B81B24820EB
:102E70000153012084F83C000021216450200155B9
:102E80006169616404F13C02002104F1540072DFC5
:102E9000064600BF304600B186E700BF0120207023
:102EA000304681E770B504460D462E46208810282E
:102EB00004D0112807D026280FD109E0214630463A
:102EC0000FF05EFB0AE0214630460FF0D4FC05E02F
:102ED000214630460FF0F4FE00E000BF00BF70BD99
:102EE00070B504460E46207808B9082070BDA6705B
:102EF000002140F22C40C4F82614A4F82A140155ED
:102F0000A07910B1A078012809D0E07910B1A0789B
:102F1000012804D0E07970B1A07802280BD1606B51
:102F200030B1012084F82D040820616B884702E04D
:102F3000002084F82D0431462046FCF7A7FAA07043
:102F4000606BA0B1A078032802D0A07804280ED12D
:102F5000607960B194F82E0448B9002084F83004F8
:102F6000012084F82F040720616B884702E00020CD
:102F700084F82F04182104F13C00F3F79AFA012099
:102F800084F83C0004F12C0010F06AFB20B194F8A6
:102F90002C105120015502E001215120015594F8D7
:102FA000240060B104F1280010F05AFB20B194F81D
:102FB00028105220015502E0012152200155002124
:102FC00050200155A078052824D2DFE800F01F0327
:102FD0000A11180004F13C01204613F0DFF9054600
:102FE00019E004F13C01204613F0C0F9054612E057
:102FF00004F13C01204613F0E3F905460BE004F12F
:103000003C01204613F00AFA054604E0002084F84B
:10301000310000E000BF00BFA07898B104F13C028D
:1030200004F15400D4F8201472DF05460DB128468F
:103030005CE794F8301094F8540073DF05460DB146
:10304000284653E7606B18B194F83100616B8847EC
:1030500000204BE72DE9F041044600BF14B90E20D3
:10306000BDE8F08100BF1C2221461C48F3F708FA96
:103070001B481A490860206860B120687ADF05465D
:103080000DB12846ECE7164821680A6802604968D5
:10309000416005E012487BDF05460DB12846DFE7B9
:1030A000002617E006EB86000E4901EB800700BF03
:1030B0004FF6FF70388000BF0B4800EB4610786079
:1030C0000A4A0021381DFFF703FA05460DB1032017
:1030D000C6E7761C002EE5D00020C1E70C86002054
:1030E000F2490020F8850020D8850020957404005E
:1030F00010B50446204600F0A1F808B1204610BDE6
:103100001420FCE710B50446204600F097F820B1E3
:10311000214603480CF031F810BD0020FCE7000008
:103120006C85002070B504460D461646204614F006
:10313000FBF908B9002070BD034951F8240032465C
:10314000294605F0EDFFF6E77885002010B5044626
:10315000204600F073F820B1214603480CF00DF82A
:1031600010BD0020FCE700007485002010B5044667
:10317000204600F063F820B1214603480BF0FDFF24
:1031800010BD0020FCE700007085002070B50446EB
:103190000025204600F052F850B1214605480BF0BA
:1031A000ECFF06460EB1022000E00120054600BFFC
:1031B000284670BD6885002070B50446002520466D
:1031C00000F03CF850B1214605480BF0D6FF06460A
:1031D0000EB1022000E00120054600BF284670BD68
:1031E0006485002070B505460C46204614F09CF915
:1031F00050B1284600F022F830B1044901EB8400B8
:1032000029460BF0BAFF70BD0020FCE7788500204E
:1032100070B505460C461646204614F085F950B1A7
:10322000284600F00BF830B1034901EB8400324628
:10323000294605F0A8FB70BD7885002010B504462E
:10324000142C01DB002010BD214602480BF095FF35
:10325000F9E700006085002010B5044600BF0CB9F6
:103260000E2010BD00BF00BF06480078012801D025
:103270000820F6E700BF04480168204611F070FD01
:10328000EFE70000F0490020E44900200146002259
:1032900000BF09B90E20704700BF00BF086808B919
:1032A0000E20F8E700BF00BF486808B90E20F2E71B
:1032B00000BF0020064B18600120064B1870064B1B
:1032C00008681860054B486818601046E3E700007E
:1032D000EC490020F0490020E4490020E8490020A2
:1032E00070B504460D4600BF04B970BD00BF00BFF5
:1032F00005B9FAE700BF00BF14480078012800D0E4
:10330000F3E700BF2E462088112815D0302804D0BE
:10331000322807D0332814D109E0211D30460FF0A0
:10332000DBFB0FE0211D30460EF0CEFF0AE0211D31
:1033300030460FF0DFF905E0211D30460FF08EFA20
:1033400000E000BF00BF00BFCFE70000F049002051
:1033500070B504460D4600BF0CB90E2070BD00BF0D
:1033600000BF0B480078012801D00820F6E700BF15
:103370000848006808B90820F0E794F8C80208B1C6
:103380001120EBE72946204603F076FEE6E7000031
:10339000F0490020EC4900202DE9FC4105460C468F
:1033A000174620880930B84202D90C20BDE8FC81BC
:1033B00068466DDF064600BF304600B1F6E700BF45
:1033C0000820218868542088401C20801B202188E8
:1033D00068542088401C208020882844DDF8011093
:1033E0000160BDF8051081802088801D20809DF837
:1033F0000000400818B900202188685402E001202C
:10340000218868542088401C20800020CEE70000DE
:1034100070B50CF0D9FB044600BF204600B170BD6A
:1034200000BF00BF084D28464FF0030C00DF00BF6F
:10343000044600BF204600B1F1E700BF0CF0DEFB00
:1034400004462046EBE70000F48E0020014600BF52
:1034500009B90E20704700BF014801600020F9E75C
:10346000F44A002010B54FF0FF3100203DDF044644
:1034700000BF204600B110BD00BFB12100203CDFDD
:10348000044600BF204600B1F5E700BF044841698B
:103490000120884702200DF03DF90020EBE70000F5
:1034A000D88E002010B50548006841690020884783
:1034B000FFF7D8FF0446204610BD0000F44A002064
:1034C00010B588B0044620216846F2F7F2FF0320C9
:1034D000ADF8000020788DF802009DF80D0020F076
:1034E000200020308DF80D009DF80D0020F0080020
:1034F00008308DF80D0001208DF810008DF80C00BB
:103500001720ADF8040001208DF813008DF812008B
:103510008DF811006088A21D694602F065F808B0B8
:1035200010BD000030B585B00546244B0FCB8DE8AB
:103530000F0000BF15B90E2005B030BD00BF4FF61B
:10354000FF701F4988802868486100200876084677
:10355000406908B91B4848611948FFF777FF0446DE
:1035600000BF204600B1E7E700BF00BF01208DF893
:1035700012004FF65960ADF8100000BF104A921CBF
:1035800004A90120A8DF044600BF204600B1D3E70C
:1035900000BF0B49684662DF044600BF204600B109
:1035A000CAE700BF0648FFF78BFF044600BF20466E
:1035B00000B1C1E700BF0020BEE70000E4850400C1
:1035C000D88E00201D82030070B504460D4600BF52
:1035D00004B970BD00BF2088102806D0112808D07B
:1035E00051280AD0532810D10BE020460EF0BEFF20
:1035F0000CE020460FF024F908E020460FF0AEFA68
:1036000004E020460FF0C2F900E000BF00BF00BF99
:10361000DFE7000070B504460426207B012802D0B5
:10362000022822D109E004F005FE05460DB9012665
:1036300002E0112D00D1062619E0607B142801DC80
:10364000607B08B905260FE0627B04F10E01124889
:10365000F2F716FF607B1049091F8861084612F0D7
:103660000BFF054605B9012601E0022600BF00BF99
:10367000012E0FD0207B314600F058F8054625B1C9
:10368000064800684169032088470448006841698A
:103690000220884770BD0000048F0020F44A0020FB
:1036A00070B505460E4600BF1E48006820B11D4893
:1036B000406808B1012000E0002000B970BD00BFE3
:1036C000184800F10801426828469047044600BFA8
:1036D000082C24D07CB900201349096848760121C0
:1036E000022000F023F80446CCB10F48006841697D
:1036F0000320884713E000200B490968487606211B
:10370000022000F013F8044624B10748006841691C
:10371000032088470448006841690220884700BFA9
:10372000CCE70000F48E0020F44A0020F0B587B00A
:1037300004460D4603270020019002900390049058
:103740000320069020208DF814008DF815408DF888
:1037500016500E48C088ADF8040002208DF806000F
:103760000020ADF8080006A8039005A804900749BA
:10377000888801A9AEDF064626B9BDF818000328DF
:1037800000D00C26304607B0F0BD0000D88E0020D7
:1037900030B1012805D0022804D0032807D102E067
:1037A00006E005E004E000BF002100BF00E000BF2C
:1037B00000BF70472DE9F04104460F46A688304609
:1037C000FFF7E4FC0546012D03D0204600F0C2F8C7
:1037D00018B120460EF062FC08E0022D02D02088CD
:1037E0001D2803D1002120460EF074FBBDE8F081B6
:1037F0002DE9F04104460F46A6882088102806D0FF
:10380000112819D019283FD01A284AD118E011F0F0
:1038100041FA304611F0C2F830B900BF22A2F021BF
:103820000420F2F7F7FC06E0E07B022803D13146E2
:103830002C480BF0B1FC34E0304611F04FFA30E088
:10384000207A0509042D01DB012000E0002002465A
:10385000314624480C3005F096F8032D01DB012099
:1038600000E00020024631461E48083005F08BF883
:10387000022D01DB012000E00020024631461948FC
:10388000001D05F080F80CE0207A48B9607AC0F39A
:10389000C0052A46314613480C3005F074F800BFC5
:1038A00000BF00BFBDE8F0812E2E5C2E2E5C2E2EB8
:1038B0005C2E2E5C2E2E5C2E2E5C636F6D706F6EF8
:1038C000656E74735C626C655C636F6D6D6F6E5C6E
:1038D000626C655F636F6E6E5F73746174652E6397
:1038E000000000006885002070B504460D46208861
:1038F000102806D0112808D012280ED0502810D138
:1039000007E020460EF0C0FD0CE020460EF07FFFE1
:1039100008E020460FF006FA04E020460EF09CFD79
:1039200000E000BF00BF70BD70B504460D4600BF8B
:103930000748007800B970BD00BF204608F0D4F8F1
:10394000204612F063FF204605F0D6FE00BFF2E7E6
:10395000304A002001460888262801D101207047FE
:103960000020FCE710B5002408E0074850F82400C8
:1039700018B1054951F824008047641C03480078B9
:103980008442F2DB10BD0000987500208C470020B7
:1039900010B5002408E0074850F8240018B1054984
:1039A00051F824008047641C034800788442F2DB0D
:1039B00010BD0000A47500208D4700202DE9F041C6
:1039C00007460C46207820B1012824D0022829D1AE
:1039D00027E0618804F10E02384600F035F805460C
:1039E00000BF2E4636B100BF10A276213046F2F756
:1039F00011FC00BF00BF384600F02EF9054600BF9D
:103A00002E4636B100BF09A279213046F2F702FCFA
:103A100000BF00BF06E0A1890A4AA068126890476B
:103A200000E000BF00BFBDE8F08100002E2E5C2E3C
:103A30002E5C2E2E5C626C655F6366675C686F73DC
:103A4000742E63008041002070B504460E46154672
:103A500000BF0CB90E2070BD00BF26812DB1698852
:103A6000A18128886081A988E1813146A0690BF095
:103A7000FDFCF0E770B586B004460D461A4B0FCB3F
:103A800001AE0FC600BF14B90E2006B070BD00BF56
:103A900000BF0DB90E20F8E700BF00BFA86808B945
:103AA0000E20F2E700BFE11D01A862DF064600BF5D
:103AB000304600B1E9E700BFE0798DF8160001203B
:103AC000ADF814004FF6FF70208128682061686807
:103AD0006061002060810021E181A868A06105A8E3
:103AE000FFF7BAFBD1E700004083040070B586B051
:103AF00005460E46344604B10DB906B070BD2089A6
:103B00004FF6FF71884203D02089A988884200D0EF
:103B1000F3E72888112806D0392816D129462046EF
:103B20000EF04AFF12E0A888218988420CD1206952
:103B300050B102208DF804004FF6FF70208101A9DA
:103B400020462269904700BF00E000BF00BF00BFD1
:103B5000D3E770B586B005460C46142101A8F2F7EC
:103B6000A8FC04F10E06207800283AD1A08801288C
:103B700037D1A079E979884233D1002022E000EBE7
:103B8000C00136F81110022902D0032917D107E02D
:103B900000EBC00106EB41010A89ADF816200FE0E9
:103BA00000EBC00106EB41010989ADF8121000EBF2
:103BB000C00106EB41014A89ADF8142000E000BFC6
:103BC00000BF401C217A8142D9D8286948B1608859
:103BD000ADF8060000208DF8040001A928462A69E6
:103BE000904706B070BD000070B588B004460E4620
:103BF000154600BF14B90E2008B070BD00BF2021CB
:103C00006846F2F756FCF42D01DD0720F4E7208921
:103C10004FF6FF71884201D10820EDE701208DF8B1
:103C200000000C4802900394E189ADF81210ADF841
:103C300016500021ADF81410069602208DF81000E1
:103C400001218DF8111022896946A0690BF038FC1A
:103C5000D2E70000A192030010B5044600BF0CB9E2
:103C60000E2010BD00BF20894FF6FF71884201D0A1
:103C7000A08908B90820F4E70121204601F066FC7C
:103C8000EFE72DE9F04186B00446884617461D4609
:103C900000BF1CB90E2006B0BDE8F08100BF01AA2C
:103CA00029466069FEF722FF064600BF304600B194
:103CB000F1E700BF4FF6FF70854201D0019808B9C7
:103CC0000520E8E70198007808B90820E3E738887C
:103CD000F42801DD0720DEE7002002900390049025
:103CE0000590A088ADF80800CDF814800497012055
:103CF0008DF80A0002A92846AEDFCCE770B58EB079
:103D000004460E463E4B0FCB09AD0FC500BF14B99C
:103D10000E200EB070BD00BF00BF0EB90E20F8E738
:103D200000BF3068A061214609A862DF054600BFD8
:103D3000284600B1EDE700BF20788DF8360001205D
:103D4000ADF83400A21C0DA9A8DF054600BF284627
:103D500000B1DEE700BF202101A8F2F7AAFB022094
:103D6000ADF8040020788DF80600F420ADF80800C6
:103D70000120ADF80A008DF810009DF8110020F028
:103D8000080008308DF811009DF8110020F00400A3
:103D9000001D8DF8110001208DF815008DF816001A
:103DA000608804F10C0201A901F01EFC05460DB16A
:103DB0002846AEE7202101A8F2F77BFB0320ADF8EF
:103DC000040020788DF80600F420ADF808000120EA
:103DD000ADF80A008DF810009DF8110020F01000D9
:103DE00010308DF8110001208DF815008DF81600A7
:103DF0008DF817006088221D01A901F0F5FB88E706
:103E00005083040070B504460D4605B104B970BD79
:103E10002E462088102804D0502807D057280FD1CC
:103E200009E0214630460EF067FB0AE021463046A5
:103E30000EF0A4FF05E0214630460EF0D9FD00E06B
:103E400000BF00BF00BFE2E710B5002408E007484C
:103E500050F8240018B1054951F824008047641C2B
:103E6000034800788442F2DB10BD0000007300209C
:103E70005241002010B5002408E0074850F8240003
:103E800018B1054951F824008047641C03480078A4
:103E90008442F2DB10BD000040730020534100203B
:103EA00070B50446204613F0BCFA0546C5F3400041
:103EB00070BD70B50446204613F0B3FA054605F010
:103EC000010070BD38B50CF0E1FE044600BF254688
:103ED0003DB100BF15A240F2A3112846F2F79AF9AE
:103EE00000BF00BF00200090694601200CF0CEFD0D
:103EF000044600BF25463DB100BF0CA240F2A91107
:103F00002846F2F787F900BF00BF68460CF01CFE98
:103F1000044600BF25463DB100BF04A240F2AD11EA
:103F20002846F2F777F900BF00BF38BD2E2E5C2E71
:103F30002E5C2E2E5C626C655F6366675C686F73D7
:103F4000742E630010B504A11120F4F749F810B9DC
:103F50000748F6F785FC10BD6273705F6164635FAC
:103F6000696E69745F6572726F720D0A00000000FD
:103F7000453F030010B504A11320F4F731F810B940
:103F80000748F6F76DFC10BD6273705F666C617375
:103F9000685F696E69745F6572726F720D0A000006
:103FA000753F030010B504A11420F4F719F810B9F7
:103FB0000748F6F755FC10BD6273705F70776D5F50
:103FC000696E69745F6572726F720D0A000000009D
:103FD000A53F030010B504A11620F4F701F810B9AD
:103FE0000748F6F73DFC10BD6273705F7274635F43
:103FF000636F6E6669675F6572726F720D0A0000AB
:10400000D53F030010B504A11620F3F7E9FF10B95E
:104010000748F6F725FC10BD6273705F7274635F2A
:10402000696E69745F6572726F720D0A000000003C
:104030000540030010B504A11220F3F7D1FF10B919
:104040000748F6F70DFC10BD6273705F737069303E
:104050005F696E69745F6572726F720D0A000000AD
:104060003540030010B504A11520F3F7B9FF10B9CE
:104070000748F6F7F5FB10BD6273705F7764745FF5
:10408000696E69745F6572726F720D0A00000000DC
:104090006540030030B503460C4600201FE09FED4D
:1040A000110A02EB800181ED000A002114E002EB0D
:1040B000800595ED000A01EB800503EB8505D5ED44
:1040C000000A04EB810595ED001A00EE810A02EB6F
:1040D000800585ED000A491C0429E8DB401C0928FD
:1040E000DDDB30BD0000000030B5A1B005460C4658
:1040F00094ED140A8DED010A94ED180A8DED020A73
:1041000094ED190A8DED030A94ED1A0A8DED040A57
:1041100094ED380A8DED050A94ED3C0A8DED060A02
:1041200094ED3D0A8DED070A94ED3E0A8DED080AE7
:1041300094ED410A8DED090A94ED450A8DED0A0AC8
:1041400094ED460A8DED0B0A94ED470A8DED0C0AAD
:1041500094ED4A0A8DED0D0A94ED4E0A8DED0E0A8E
:1041600094ED4F0A8DED0F0A94ED500A8DED100A73
:10417000002012E001A901EB001101EB800191ED9B
:10418000000ADFEDFE0A30EE200A01A901EB001162
:1041900001EB800181ED000A401C0328EADB9DED64
:1041A000100ADFEDF70A30EE200A8DED100A11A992
:1041B00001A809F0E3FF94ED020ADDED110A20EEFB
:1041C000200AD4ED060A9DED151A00EE810AD4ED01
:1041D000070A9DED191A00EE810AD4ED080A9DED3B
:1041E0001D1A00EE810A85ED000A94ED020ADDED4C
:1041F000120A20EE200AD4ED060A9DED161A00EEF2
:10420000810AD4ED070A9DED1A1A00EE810AD4ED59
:10421000080A9DED1E1A00EE810A85ED010A94ED53
:10422000020ADDED130A20EE200AD4ED060A9DED08
:10423000171A00EE810AD4ED070A9DED1B1A00EE55
:10424000810AD4ED080A9DED1F1A00EE810A85ED62
:10425000020A94ED020ADDED140A20EE200AD4EDE4
:10426000060A9DED181A00EE810AD4ED070A9DEDAD
:104270001C1A00EE810AD4ED080A9DED201A00EE0A
:10428000810A85ED030A94ED0B0ADDED110A20EE9B
:10429000200AD4ED0F0A9DED151A00EE810AD4ED27
:1042A000100A9DED191A00EE810AD4ED110A9DED58
:1042B0001D1A00EE810A85ED040A94ED0B0ADDED6E
:1042C000120A20EE200AD4ED0F0A9DED161A00EE18
:1042D000810AD4ED100A9DED1A1A00EE810AD4ED80
:1042E000110A9DED1E1A00EE810A85ED050A94ED76
:1042F0000B0ADDED130A20EE200AD4ED0F0A9DED26
:10430000171A00EE810AD4ED100A9DED1B1A00EE7B
:10431000810AD4ED110A9DED1F1A00EE810A85ED88
:10432000060A94ED0B0ADDED140A20EE200AD4ED06
:104330000F0A9DED181A00EE810AD4ED100A9DEDCA
:104340001C1A00EE810AD4ED110A9DED201A00EE30
:10435000810A85ED070A94ED140ADDED110A20EEBD
:10436000200AD4ED180A9DED151A00EE810AD4ED4D
:10437000190A9DED191A00EE810AD4ED1A0A9DED75
:104380001D1A00EE810A85ED080A94ED140ADDED90
:10439000120A20EE200AD4ED180A9DED161A00EE3E
:1043A000810AD4ED190A9DED1A1A00EE810AD4EDA6
:1043B0001A0A9DED1E1A00EE810A85ED090A94ED98
:1043C000140ADDED130A20EE200AD4ED180A9DED43
:1043D000171A00EE810AD4ED190A9DED1B1A00EEA2
:1043E000810AD4ED1A0A9DED1F1A00EE810A85EDAF
:1043F0000A0A94ED140ADDED140A20EE200AD4ED29
:10440000180A9DED181A00EE810AD4ED190A9DEDE7
:104410001C1A00EE810AD4ED1A0A9DED201A00EE56
:10442000810A85ED0B0A94ED1D0ADDED110A20EEDF
:10443000200AD4ED210A9DED151A00EE810AD4ED73
:10444000220A9DED191A00EE810AD4ED230A9DED92
:104450001D1A00EE810A85ED0C0A94ED1D0ADDEDB2
:10446000120A20EE200AD4ED210A9DED161A00EE64
:10447000810AD4ED220A9DED1A1A00EE810AD4EDCC
:10448000230A9DED1E1A00EE810A85ED0D0A94EDBA
:104490001D0ADDED130A20EE200AD4ED210A9DED60
:1044A000171A00EE810AD4ED220A9DED1B1A00EEC8
:1044B000810AD4ED230A9DED1F1A00EE810A85EDD5
:1044C0000E0A94ED1D0ADDED140A20EE200AD4ED4B
:1044D000210A9DED181A00EE810AD4ED220A9DED05
:1044E0001C1A00EE810AD4ED230A9DED201A00EE7D
:1044F000810A85ED0F0A94ED260ADDED110A20EE02
:10450000200AD4ED2A0A9DED151A00EE810AD4ED99
:104510002B0A9DED191A00EE810AD4ED2C0A9DEDAF
:104520001D1A00EE810A85ED100A94ED260ADDEDD4
:10453000120A20EE200AD4ED2A0A9DED161A00EE8A
:10454000810AD4ED2B0A9DED1A1A00EE810AD4EDF2
:104550002C0A9DED1E1A00EE810A85ED110A94EDDC
:10456000260ADDED130A20EE200AD4ED2A0A9DED7D
:10457000171A00EE810AD4ED2B0A03E0BE37863508
:1045800017B7D1389DED1B1A00EE810AD4ED2C0A25
:104590009DED1F1A00EE810A85ED120A94ED260AA0
:1045A000DDED140A20EE200AD4ED2A0A9DED181A3A
:1045B00000EE810AD4ED2B0A9DED1C1A00EE810A53
:1045C000D4ED2C0A9DED201A00EE810A85ED130A28
:1045D00094ED2F0ADDED110A20EE200AD4ED330A06
:1045E0009DED151A00EE810AD4ED340A9DED191ADD
:1045F00000EE810AD4ED350A9DED1D1A00EE810A08
:1046000085ED140A94ED2F0ADDED120A20EE200A42
:10461000D4ED330A9DED161A00EE810AD4ED340A6A
:104620009DED1A1A00EE810AD4ED350A9DED1E1A91
:1046300000EE810A85ED150A94ED2F0ADDED130ACF
:1046400020EE200AD4ED330A9DED171A00EE810A00
:10465000D4ED340A9DED1B1A00EE810AD4ED350A23
:104660009DED1F1A00EE810A85ED160A94ED2F0AC2
:10467000DDED140A20EE200AD4ED330A9DED181A60
:1046800000EE810AD4ED340A9DED1C1A00EE810A79
:10469000D4ED350A9DED201A00EE810A85ED170A4A
:1046A00094ED380ADDED110A20EE200AD4ED3C0A23
:1046B0009DED151A00EE810AD4ED3D0A9DED191A03
:1046C00000EE810AD4ED3E0A9DED1D1A00EE810A2E
:1046D00085ED180A94ED380ADDED120A20EE200A65
:1046E000D4ED3C0A9DED161A00EE810AD4ED3D0A88
:1046F0009DED1A1A00EE810AD4ED3E0A9DED1E1AB8
:1047000000EE810A85ED190A94ED380ADDED130AF1
:1047100020EE200AD4ED3C0A9DED171A00EE810A26
:10472000D4ED3D0A9DED1B1A00EE810AD4ED3E0A40
:104730009DED1F1A00EE810A85ED1A0A94ED380AE4
:10474000DDED140A20EE200AD4ED3C0A9DED181A86
:1047500000EE810AD4ED3D0A9DED1C1A00EE810A9F
:10476000D4ED3E0A9DED201A00EE810A85ED1B0A6C
:1047700094ED410ADDED110A20EE200AD4ED450A40
:104780009DED151A00EE810AD4ED460A9DED191A29
:1047900000EE810AD4ED470A9DED1D1A00EE810A54
:1047A00085ED1C0A94ED410ADDED120A20EE200A87
:1047B000D4ED450A9DED161A00EE810AD4ED460AA5
:1047C0009DED1A1A00EE810AD4ED470A9DED1E1ADE
:1047D00000EE810A85ED1D0A94ED410ADDED130A14
:1047E00020EE200AD4ED450A9DED171A00EE810A4D
:1047F000D4ED460A9DED1B1A00EE810AD4ED470A5E
:104800009DED1F1A00EE810A85ED1E0A94ED410A06
:10481000DDED140A20EE200AD4ED450A9DED181AAC
:1048200000EE810AD4ED460A9DED1C1A00EE810AC5
:10483000D4ED470A9DED201A00EE810A85ED1F0A8E
:1048400094ED4A0ADDED110A20EE200AD4ED4E0A5D
:104850009DED151A00EE810AD4ED4F0A9DED191A4F
:1048600000EE810AD4ED500A9DED1D1A00EE810A7A
:1048700085ED200A94ED4A0ADDED120A20EE200AA9
:10488000D4ED4E0A9DED161A00EE810AD4ED4F0AC2
:104890009DED1A1A00EE810AD4ED500A9DED1E1A04
:1048A00000EE810A85ED210A94ED4A0ADDED130A36
:1048B00020EE200AD4ED4E0A9DED171A00EE810A73
:1048C000D4ED4F0A9DED1B1A00EE810AD4ED500A7B
:1048D0009DED1F1A00EE810A85ED220A94ED4A0A29
:1048E000DDED140A20EE200AD4ED4E0A9DED181AD3
:1048F00000EE810AD4ED4F0A9DED1C1A00EE810AEC
:10490000D4ED500A9DED201A00EE810A85ED230AB0
:1049100021B030BD30B502460B46002046E00021F4
:1049200041E003EB001494ED000A01F1120402EBE4
:104930008404D4ED000A20EE200A012404EB800454
:1049400003EB8404D4ED000A01F1360402EB840485
:1049500094ED001A00EE810A022404EB800403EBBC
:104960008404D4ED000A01F13F0402EB840494EDC9
:10497000001A00EE810A032404EB800403EB840494
:10498000D4ED000A01F1480402EB840494ED001A0E
:1049900000EE810A00EBC0040C44104D05EB8404CA
:1049A00084ED000A491C0929BBDB401C0928B6DB41
:1049B00000200FE002EB800191ED000A074901EBB6
:1049C0008001D1ED000A30EE600A02EB800181ED3A
:1049D000000A401C5128EDDB30BD00008C82002015
:1049E00010B502460023002003E032F810402344B3
:1049F000401C8842F9DBB3FBF1F080B210BD00002F
:104A0000F0BBE9BBF7EE001A424AC2ED021AF7EE1C
:104A1000001A414AC2ED021A3E4AD2ED001AF4EEE3
:104A2000C01AF1EE10FA01D282ED000A394AD2ED35
:104A3000011AF4EEE01AF1EE10FA01D2C2ED010A09
:104A4000344AD2ED021AF4EEC11AF1EE10FA01D294
:104A500082ED021A304AD2ED001AF4EEC01AF1EEDD
:104A600010FA01DD82ED000A2B4AD2ED011AF4EEB4
:104A7000E01AF1EE10FA01DDC2ED010A264A00E06B
:104A800008E0D2ED021AF4EEC11AF1EE10FA01DDDF
:104A900082ED021A00B999B3204A1268FAB91D4A88
:104AA000D2ED001A1C4A92ED002A71EEC21A9FED57
:104AB0001C2AF4EEC21AF1EE10FA0EDC154AD2ED01
:104AC000011A154A92ED012A71EEC21A9FED142ABD
:104AD000F4EEC21AF1EE10FA00DD00E000BF05228C
:104AE0000E4B1A600B4A82ED000AC2ED010A82EDFC
:104AF000021A094A82ED000AC2ED010A82ED021A89
:104B0000064A1268002A04DD044A1268521E034B4A
:104B10001A607047E8830020DC830020644900208D
:104B2000CDCC4C3F7CB50446204607F023F9054622
:104B300000236A4609210EF0AFFB052805D10122AA
:104B4000024801782046FEF763FB7CBD0C4A00203A
:104B50007CB504460E460020019042F6A620ADF832
:104B6000040001208DF806000748006800906A469E
:104B700001A92046A0DF05462DB90122034801788E
:104B80002046FEF745FB7CBD3C8204000D4A002018
:104B900038B5044600200090FBF77AFF00909DF89E
:104BA000002005A10020F6F7A9FB01236A46A321F6
:104BB0000020F2F7EDFB38BD212121216170705FEB
:104BC000636F6E6E657465645F676574526967686C
:104BD000743A25640A00000038B5044625460020D2
:104BE0000090686800788DF80000686840788DF85B
:104BF0000100686840786968097800EB0120104975
:104C00000880084602880FA10020F6F777FB0223F0
:104C10006A46AC210020F2F797FDF7F7BBFD144977
:104C20000860F4F791FB142804DD12490320F5F71E
:104C300069F803E010490320F5F764F838BD000077
:104C4000CC3E00203D3D3D3D3D3D3D3E63625F42EB
:104C50004C455F424C494E4B5F4C45442C64697354
:104C6000706C617974696D653A25640A0000000012
:104C7000D03E0020007F00FF00106FFF01464A6811
:104C80001278014B1A707047653F002070B50446DA
:104C9000254611F00DF92B7AA72100206A68F2F75A
:104CA00053FD70BD38B5054616A10020F6F726FB6A
:104CB0002C461B480079002811DD6068007818B97F
:104CC00001201849087038BD60680078012816D1A5
:104CD0000123A62100206268F2F736FD0FE00120D3
:104CE000009001236A46A6210020F2F751FB012023
:104CF0000D4908600DA10020F6F700FB00BF00BFC2
:104D0000E1E700003E3E3E3E3E3E3E3E3E3E424CE1
:104D1000455F436C69656E745F525F4446550A0097
:104D200008520020A03E00209C3E00203E3E3E3E19
:104D30003E3E3E3E3E3E4446552073746172742EA4
:104D40002E2E2E0A0000000070B504462546686825
:104D500000781649C8700846C07838B10121032090
:104D600006F078F900201149087103E000210320C2
:104D700006F070F90D48C078012802D0022806D14B
:104D800002E0F4F7E3FC02E0F4F7E6FC00BF00BF4A
:104D90000123064AD21CA2210020F2F7D5FC0348C9
:104DA000C27803A10020F6F7A9FA70BD8A3E002060
:104DB0003E3E3E3E3E3E3E3E3E3E63625F424C4590
:104DC0005F436C69656E745F525F47414D454D4F5F
:104DD00044453A25640D0A0038B5044625466868FE
:104DE000007800909DF80000012807D100201449A8
:104DF00008700121042006F02DF906E09DF800005E
:104E000018B90021042006F025F901236A46A521DE
:104E10000020F2F799FC9DF8000001280AD109480A
:104E2000007838B90848D0F81B000849086000200D
:104E3000074908609DF800000249087038BD00006D
:104E4000893E00207C3E002008520020803E002049
:104E5000843E002070B505462C4660684078616845
:104E6000097840EA012617480079D8B1606880784F
:104E7000012803D13046F5F755F91DE060688078C8
:104E800048B93046F5F74EF9237AA421002062682C
:104E9000F2F75AFC10E0237AA42100206268F2F7AE
:104EA00053FC09E060688078022802D0606880784E
:104EB00010B93046F5F736F9324603A10020F6F76F
:104EC0001DFA70BD085200204D542052554E3A250F
:104ED00064200A0038B504462546686800780090CA
:104EE0009DF8000010B1012810D107E000200B4907
:104EF00008704FF47A70F5F715F907E001200749BB
:104F000008704FF47A70F5F70DF900BF00BF012368
:104F10006A46AB210020F2F717FC38BD283F00207D
:104F200070B505462C466068067836B1012E0BD068
:104F3000022E0DD0032E1FD114E0FBF755FA10A15D
:104F40000020F6F7DBF918E01420FCF797F814E0DE
:104F5000042005F005FEB0F1FF3F02D12046FBF72B
:104F60008BF80AE0237AA12100206268F2F710FA98
:104F70002046FBF727F800E000BF00BF70BD00002F
:104F80002121212121212121212121212121213DF5
:104F90003D3D3D3D3D3D3E6170705F636C69656EBA
:104FA000745F696E666F6D6174696F6E5F53656E75
:104FB000640A000010B504460E48007800B910BD20
:104FC0000D4800880D490988884210DA0A4800888F
:104FD000401C80B20849088008490988884202DBE1
:104FE00000200449087004480088FBF787F800BFD8
:104FF000E5E70000F53D0020F63D0020F83D0020EB
:1050000070B5044625462B7AA72100206A68F2F77E
:10501000BFF970BD70B504462546074A07A14FF495
:10502000FA70F5F7CBFB0A200A4908706868007827
:105030000949087070BD0000C51803006170705FF9
:105040006F74615F73656E646C65667473746174AC
:1050500065000000A13E0020A23E002070B504467D
:1050600025462B7AAD2100206A68F2F791F970BDD0
:1050700070B505462C4660680078012814D1606838
:10508000407800066168897840EA01406168C97823
:1050900040EA012061680979084304490860FDF786
:1050A0009FF903200249087070BD0000843E002073
:1050B000883E00202DE9FF410646344660680778A7
:1050C00017B1012F71D13FE0002006E000F141014E
:1050D0006268525C37490A54401C0628F6DB3548A2
:1050E000353890F83A1090F8392090F8383090F828
:1050F0003700CDE90132039100902E48353890F801
:10510000363090F835202CA10020F6F7F7F8472527
:105110006068405D0106681C6268105C41EA0041FD
:10512000A81C105C41EA0020E91C515C084321499D
:1051300035390863281D6168095C1E48353880F8D8
:105140003410FBF751F931E0606840782849087065
:1051500060688078274908706068C07800066168D8
:10516000097940EA01406168497940EA01206168B3
:1051700089790843204908606068C0790006616841
:10518000097A40EA01406168497A40EA0121606891
:10519000807A014307483538C0F81F1000201749AE
:1051A0000870FAF765FE01E0FFE700BF00BFBDE849
:1051B000FF8100003D5200206D466C6173682E6DCA
:1051C000436C69656E742E6D6163416464723A2547
:1051D00030325820253032582025303258202530A2
:1051E0003258202530325820253032580A0000002D
:1051F000283E0020293E00202C3E0020543E002066
:1052000010B502A10020F6F779F810BD3D3D3D3DF7
:105210003D3D3D3E63625F486F73745F436F6E6EEA
:105220006563740A0000000010B5044600210E20DA
:105230000BF0A7F8F5F73EFC10BD10B50446F5F7E6
:1052400019FC10BD10B507A10020F6F757F80C485F
:10525000007928B1F3EE0E0AB3EE0E0A11F04CFA03
:1052600010BD00003D3D3D3D3D3D3D3E63625F5311
:105270006C6176655F436F6E6E6563740A00000053
:10528000085200202DE9FE43804645464FF00009B4
:105290000024FAF7F7FB012801D1BDE8FE83384866
:1052A000007900B9F9E7002405E06868005D01A90C
:1052B0000855601CC4B2062CF7DB686880790006CC
:1052C0006968C97940EA01406968097A40EA0120C1
:1052D0006968497A40EA01066868877A3320294973
:1052E000088000240BE026483530005D01A9095DE7
:1052F000884202D04FF0010903E0601CC4B2062CC2
:10530000F1DB00BF1E48006BB0420ED11C4890F884
:105310003400B84209D11C48407D194991F82F103A
:10532000884202D1B9F1000F25D01548066380F8F4
:10533000347015480661076100240DE001A8015D85
:105340000F4835300155C4F105011048415C0C4847
:10535000401D0155601CC4B2062CEFDB01200C4936
:1053600008700948007D009007480369427D09A143
:105370000020F5F7C3FFFAF779FB00BF8DE70000C7
:1053800008520020143F0020805200200D3F0020D2
:10539000163F00206261636B757020636F6E6669F3
:1053A000673A25642C6861726456657273696F6E22
:1053B0003A25642C736F746656657273696F6E3A22
:1053C00025640A002DE9FE43804645464FF000095A
:1053D0000024FAF757FB012801D1BDE8FE834148BC
:1053E000007900B1F9E7002405E06868005D01A9D3
:1053F0000855601CC4B2062CF7DB6868807900068B
:105400006968C97940EA01406968097A40EA01207F
:105410006968497A40EA01066868877A324A162143
:105420001320F7F7E1FA002404E00220F7F734FA3A
:10543000601CC4B20A2CF8DB2B4A13211620F7F7A4
:10544000D3FA00240BE02748401D005D01A9095D47
:10545000884202D04FF0010903E0601CC4B2062C60
:10546000F1DB00BF1F48006BB0420ED11D4890F821
:105470003400B84209D11D48407D1A4991F82F10D7
:10548000884202D1B9F1000F28D01648066380F88F
:105490003470006B154908611248006B08610024E4
:1054A0000DE0C4F105011248415C0E48353001554C
:1054B00001A8015D0B48401D0155601CC4B2062CBB
:1054C000EFDB01200B4908700848007D0090074879
:1054D0000369427D08A10020F5F710FFFAF7C6FA2C
:1054E00000BF7AE70852002090D0030080520020CD
:1054F0000D3F0020163F00206261636B75702063D2
:105500006F6E6669673A25642C68617264566572CD
:1055100073696F6E3A25642C736F74665665727387
:10552000696F6E3A25640A0010B50446F1F79AFBDC
:1055300010BD10B50446F1F79FFB10BD0249096884
:105540000144014A116070476040002070B58AB084
:1055500004460D462E46202102A8F0F7AAFFF0B21D
:105560008DF80400300A8DF8050001208DF8080040
:105570000D4804900594A189ADF81A100221ADF8E8
:105580001E100021ADF81C1001A9089101208DF812
:10559000180001218DF81910228902A9A06909F0CB
:1055A0008FFF0AB070BD0000A19203000146887908
:1055B000012809D10879012806D1488842F602124B
:1055C000904201D1012070470020FCE701460248CB
:1055D00050F8210070470000208900200146014852
:1055E000405670475089002070B590B006460C4672
:1055F0001546A07818B901208DF80E0002E0A078B9
:105600008DF80E002088ADF80C0000200290607C20
:1056100002A910F055FFA07C0DF1090110F050FF18
:10562000E07B08B1012000E000209DF80A1060F343
:10563000C3018DF80A10207C08B1012000E0002091
:105640009DF80A1060F304118DF80A10207B08B150
:10565000012000E000209DF80A1060F300018DF8A1
:105660000A10207D08B1022000E001209DF80A10F8
:1056700060F342018DF80A101C2109A8F0F719FF08
:10568000607BC0F3001018B9607BC0F34010F8B124
:1056900000200090E07C0DF1010110F011FF00BF2F
:1056A0009DF8000020F00F00401C8DF800009DF8D0
:1056B000000020F0F00010308DF8000000BF9DF8D1
:1056C000020020F00600801C8DF80200CDF838D0D2
:1056D000607B8DF82400A07B8DF82500142104A8A0
:1056E000F0F7E7FE03A8049002A80590A088ADF8A3
:1056F0001C00A06820B1E088ADF81800A0680890F0
:10570000A069002849D000200190A0690088ADF868
:105710002C00A0694088ADF82E00A06940680A906E
:1057200001A80D90A169087B01A910F0C9FEA1692B
:10573000487B0DF1050110F0C3FEA069807A08B125
:10574000012000E000209DF8061060F3C3018DF8F1
:105750000610A069C07A08B1012000E000209DF881
:10576000061060F304118DF80610A069007A08B1E4
:10577000012000E000209DF8061060F300018DF884
:105780000610A069807B08B1022000E001209DF88E
:10579000061060F342018DF80610E06908B1E06977
:1057A0000C902B4604AA09A93046AADF10B070BDA0
:1057B00070B58AB004460E46202101A8F0F779FEA4
:1057C0000020099094F8C60200EB8001C1EB801024
:1057D00004EB400594F8C502B8B194F8C522521EF6
:1057E000D1B294F8C62202EB8203C3EB821204EB1F
:1057F000420501EBC10305F10A0202EB43000289F5
:10580000521C92B2ADF8242002E0E888ADF82400E2
:105810002889ADF8260003208DF80400099805902A
:10582000049405480390324601A90448006809F031
:1058300047FE0AB070BD000051700300E849002027
:1058400010B52DED048BB0EE408A9FED230AB0EE2B
:10585000409A9FED210AF0EE408A2048007848B136
:10586000B2EE040AC8EE000A1D48C0ED000A00208E
:105870001A490870B2EE040AC8EE000AF0EE609A07
:105880001748DFED180AB0EE690A03F052F8F0EE9F
:10589000408A9FED150AF4EEC08AF1EE10FA04D2A8
:1058A0009FED0D0AB0EE409A11E09FED100AF4EE64
:1058B000C08AF1EE10FA04DD9FED0D0AB0EE409AB9
:1058C00005E0B0EE680A06F0B3FFB0EE409AB0EE25
:1058D000490ABDEC048B10BD00000000FD3F002014
:1058E000F43F0020CDCC4C3D0000AF430000D2433C
:1058F0000000C842192000BF4FF0A0431A4600BF65
:10590000D2F81035C34003F00103194609B1012054
:1059100070470020FCE72DE9F04104460D464FF6A4
:10592000FF76304684420AD14FF48071284609F050
:10593000F4FB86B2B6F5807F10D126460EE0FF2C30
:105940000CDC2146284609F0D1FB80F001070FB19D
:10595000204601E04FF6FF70064600BF3046BDE826
:10596000F08110B50020F2F7EBF90120F2F7E8F929
:105970000220F2F7E5F90320F2F7E2F90420F2F74A
:10598000DFF90520F2F7DCF90620F2F7D9F9072054
:10599000F2F7D6F910BD000070B505460DB9094CF7
:1059A00001E0084C083409E0204607F010FB0646E9
:1059B00006B904E028467168884700BFF4E700BFD5
:1059C00070BD00001489002010B504462CB90120D8
:1059D000064948700020FFF7DFFF012C04D10120A9
:1059E00002498870FFF7D8FF10BD00000C89002025
:1059F0002DE9F047024613468C46D3E90245DCE91F
:105A00000267B6EB040877EB050002D30120BDE87E
:105A1000F0870020FBE701468878012805D191F83E
:105A20002000012801D100207047886A042802D094
:105A3000486A042801D10020F6E70120F4E72DE9A7
:105A4000FF4F03460C46002047E0225CFF2A3ED071
:105A5000C2F3C01922F080014DF82010B9F1000FF7
:105A60000DD05DF8201000BF4FF0A0452E46012755
:105A700007FA01F5C6F8085500BF00BF0DE05DF854
:105A8000201000BF4FF0A0452E46012707FA01F570
:105A9000C6F80C5500BF00BF00BF5DF820100125FF
:105AA0002E460027BC46B84600BF4FF0A04BDA4652
:105AB00045EA460B4BEA870B4BEA0C2B4BEA084EA8
:105AC0000AF5E06B4BF821E000BF00BF03E04FF0A8
:105AD000FF314DF82010411CC8B20428B5DB6D46DB
:105AE0001A68002107E055F8217002F5AC6646F807
:105AF00021704E1CF1B20429F5DB00BFBDE8FF8F19
:105B00000246002007E0536833F810308B4200D182
:105B10007047431C98B213888342F4DC00BFF7E758
:105B200033B58BB00546002000900C9878B1002466
:105B30000BE021460CA809F020FB28B1009A501C6C
:105B4000009001A820F81240641C142CF1D32C22E0
:105B500069462846F0F794FC0DB030BD10B50246FA
:105B60000B4600210DE0506830F811004FF6FF742D
:105B7000A04204D1506820F81130002010BD481C0C
:105B800081B210888842EEDC0420F7E701460888DD
:105B9000062808DB0888B0F5486F06DD08884FF650
:105BA000FF72904201D0072070474888062808DB22
:105BB0004888B0F5486F06DD48884FF6FF7290427E
:105BC00001D00720F0E708884FF6FF72904208D016
:105BD0004888904205D008884A88904201DD072015
:105BE000E2E70020E0E72DE9F04107460D461446C4
:105BF00098462088801D404502D90C20BDE8F081E0
:105C00003846FFF7C3FF064600BF304600B1F5E750
:105C100000BF0520218868542088401C2080122065
:105C2000218868542088401C208022885119388897
:105C300011F0FDFB218808442080228851197888C2
:105C400011F0F5FB2188084420800020D6E70000F1
:105C500010B5044600BF03A280212046F0F7DAFA0F
:105C600000BF10BD2E2E5C2E2E5C2E2E5C626C654D
:105C70005F6366675C736C6176652E63000000008D
:105C800030B587B01C216846F0F713FC0020009067
:105C90004FF4804001904FF4A030029001208DF825
:105CA0000C004FF6FF70ADF80E0001208DF81000CB
:105CB00000200590094806906846FDF7CBF9044698
:105CC00000BF254635B100BF05A293212846F0F755
:105CD000A1FA00BF00BF07B030BD0000515C030057
:105CE0002E2E5C2E2E5C2E2E5C626C655F636667CA
:105CF0005C736C6176652E6300000000F8B50546A4
:105D00000C46607A88B9207A10B91048476801E0DB
:105D10000E4887682A4639466068FCF71FFC06462D
:105D200016B1304610F0FCF80EE000202072074853
:105D3000406948B101208DF80000ADF802500348D9
:105D400041696846884700BFF8BD00000C86002006
:105D5000F0B585B004460D4617461E4614220B4981
:105D60006846F0F78DFBADF802408DF80850ADF8AD
:105D70000A708DF80C600022054801782046FDF776
:105D800047FA684602F0BAFC05B0F0BDEC820400A8
:105D9000404A002010B586B0044620880DF0A6F8D1
:105DA00000BB2088FDF7AEF930B92088012241F20E
:105DB000060102F034FA15E0208800220A49097829
:105DC000FDF726FA02208DF804002088ADF80600C1
:105DD00000208DF80C0000218DF80D1001A802F0B4
:105DE0008DFC00BF06B010BD404A002002460020D6
:105DF00003E0064B1B5C1354401C054B1B78984278
:105E0000F7DB034800780870704700002076002018
:105E10009A4700200246002003E0064B1B5C135407
:105E2000401C054B1B789842F7DB0348007808704C
:105E300070470000E475002099470020F0B5044643
:105E40000D460020002108E014F801C00646471C5A
:105E5000F8B20B4F07F806C0491CA942F4DB002139
:105E600008E012F801C00646471CF8B2044F07F8D4
:105E700006C0491C9942F4DB02490870F0BD0000DD
:105E8000E4750020994700202DE9F0410646DDE940
:105E9000064500200F88C7F307280746401CDFF897
:105EA0003CC10CF8078091F800800746401C0CF8B4
:105EB00007804F88C7F307280746401C0CF8078067
:105EC00091F802800746401C0CF807808F88C7F3C2
:105ED00007280746401C0CF8078091F80480074605
:105EE000401C0CF807801788C7F307280746401C9A
:105EF0000CF8078092F800800746401C0CF80780D9
:105F00005788C7F307280746401C0CF8078092F80B
:105F100002800746401C0CF807809788C7F30728C3
:105F20000746401C0CF8078092F804800746401C86
:105F30000CF807801F88C7F307280746401C0CF899
:105F4000078093F800800746401C0CF807805F88A4
:105F5000C7F307280746401C0CF8078093F8028017
:105F60000746401C0CF807809F88C7F307280746A0
:105F7000401C0CF8078093F804800746401C0CF87E
:105F800007802788C7F307280746401C0CF80780BE
:105F900094F800800746401C0CF807806788C7F318
:105FA00007280746401C0CF8078094F80280074633
:105FB000401C0CF80780A788C7F307280746401C39
:105FC0000CF8078094F804800746401C0CF8078002
:105FD000DFF80CC08CF80000BDE8F08120760020CE
:105FE0009A4700207FB506460C4600200290039099
:105FF000ADF80840ADF80A40009001906A4602A949
:10600000304690DF054605B100BF284604B070BD9C
:1060100010B5044621460248FDF79BFD10BD000067
:10602000807300207CB5002000900190094800900A
:10603000094801906846FDF729F9044600BF254646
:1060400035B100BF05A22F212846F0F7E3F800BFC5
:1060500000BF7CBD116003006C4700202E2E5C2E1B
:106060002E5C2E2E5C626C655F6366675C686F7386
:10607000742E63002DE9F04105460F460F4C0121B7
:10608000204609F0CBF8064600BF00BF00BF00BFA6
:10609000BFF35F8F00BF00BF00BF0EB9012000E05B
:1060A000002040B1284607F04BF908B1BDE8F08167
:1060B00002480AF08BFA00BFF8E70000044A00200B
:1060C00070B52DED0A8B04460D4694ED060AB1EE2F
:1060D000400A10EE101A0846F0F7FFFB41EC1B0BCC
:1060E000B0EE4B0AF0EE6B0AF7F7AEFDB0EE40AA49
:1060F000F0EE60AA51EC1A0BF0F71AFC09EE100A48
:1061000094ED060ADFED530AB4EEE00AF1EE10FA60
:1061100008DC94ED060ADFED500AB4EEE00AF1EE79
:1061200010FA2AD294ED040A10EE101A0846F0F77D
:10613000D4FB41EC1B0B94ED010AB1EE400A10EECA
:10614000101A0846F0F7C9FB41EC1C0BB0EE4B1AD5
:10615000F0EE6B1AB0EE4C0AF0EE6C0AF8F790F81D
:10616000B0EE40AAF0EE60AA51EC1A0BF0F7E0FB9B
:1061700008EE100ADFED398A4BE094ED000A10EECC
:10618000101A0846F0F7A9FB41EC1B0B94ED030A2B
:1061900010EE101A0846F0F7A0FB41EC1C0BB0EE15
:1061A0004B1AF0EE6B1AB0EE4C0AF0EE6C0AF8F7F0
:1061B00067F8B0EE40AAF0EE60AA51EC1A0BF0F7C7
:1061C000B7FB08EE100A94ED080A10EE101A084604
:1061D000F0F783FB41EC1B0B94ED070A10EE101A4D
:1061E0000846F0F77AFB41EC1C0BB0EE4B1AF0EED0
:1061F0006B1AB0EE4C0AF0EE6C0AF8F741F8B0EE0C
:1062000040AAF0EE60AA51EC1A0BF0F791FB08EEF1
:10621000900A9FED130A28EE000ABDEEC00A10EEA8
:10622000100A00B228809FED0E0A29EE000ABDEE8A
:10623000C00A10EE100A00B268809FED090A28EE2D
:10624000800ABDEEC00A10EE100A00B2A880BDECB4
:106250000A8B70BDEFFF7F3FEFFF7FBF00000000A4
:1062600000401C4602781206437842EA03428378D3
:1062700042EA0322C3781A43364B1A6002791206A7
:10628000437942EA0342837942EA0322C3791A43FB
:10629000304B5A60027A1206437A42EA0342837A0A
:1062A00042EA0322C37A1A432A4B9A60427B037B59
:1062B00042EA032212B2284B1A80C27B837B42EA55
:1062C000032212B2244B5A80427C037C42EA03220E
:1062D00012B2214B9A80C27C837C42EA03221F4B7C
:1062E0001A80427D037D42EA03221D4B1A80827D83
:1062F0001C4B1A80C27D1C4B1A70427E037E42EA00
:10630000032212B2194B1A80C27E837E42EA032214
:1063100012B2174B1A80427F037F42EA032212B265
:10632000134B5A80C27F837F42EA032212B2104B82
:106330009A8090F82020120690F8213042EA034219
:1063400090F8223042EA032290F823301A43094B96
:106350001A6070474C7D0020D0480020F64800208D
:10636000FA480020DC480020F2480020CC480020F9
:10637000D64800200049002002781206437842EAFD
:106380000342837842EA0322C3781A43364B1A60E9
:1063900002791206437942EA0342837942EA0322F0
:1063A000C3791A43304B5A60027A1206437A42EAA2
:1063B0000342837A42EA0322C37A1A432A4B9A6041
:1063C000427B037B42EA032212B2284B1A80C27B33
:1063D000837B42EA032212B2244B5A80427C037C24
:1063E00042EA032212B2214B9A80C27C837C42EAA9
:1063F00003221F4B1A80427D037D42EA03221D4B7C
:106400001A80827D1C4B1A80C27D1C4B1A70427E02
:10641000037E42EA032212B2194B1A80C27E837EA7
:1064200042EA032212B2174B1A80427F037F42EAEC
:10643000032212B2134B5A80C27F837F42EA0322A7
:1064400012B2104B9A8090F82020120690F821305A
:1064500042EA034290F8223042EA032290F82330C5
:106460001A43094B1A607047587D0020E24800200B
:10647000F4480020F8480020EE480020F1480020B1
:10648000DE480020E8480020FC48002070B50646A1
:106490000D4616B14FF4064070BD287920B1012891
:1064A00009D0022815D111E00220287128460EF0EB
:1064B000D3FA044610E0284602F01CFA044648F2DB
:1064C0000960844201D141F61D5405E041F61D5496
:1064D00002E048F20E6400BF00BF2046DCE7000087
:1064E0002DE9F04F89B004460F4691464FF0000B5E
:1064F00020216846EFF7DDFF94F8C60200EB80012B
:10650000C1EB801004EB400594F8C50200EBC0011C
:1065100005F10A0000EB410A94F8C502401C2979F4
:10652000884207D108AB00225146204606F0FBFC0A
:10653000834627E094F8C5621FE02879401EB042E8
:1065400002D14FF0000806E0701C00EBC00105F11D
:106550000A0000EB410808AB42465146204606F0CF
:10656000E2FC10B14FF0010B0AE0C24694F8C502FC
:10657000401C84F8C502701CC6B22879B042DCDC2D
:1065800000BF00BFBBF1000F05D101203870002013
:1065900009B0BDE8F08F0020387004208DF80000AD
:1065A000089804900394044802904A4669460348B8
:1065B000006808F085FFEBE751700300E849002010
:1065C0002DE9F0412DED068B84B006460F464FF0C5
:1065D0000008002005E036F9101001AA42F820104A
:1065E000401C0328F7DB0398002801DB014600E08C
:1065F00041429B4A11809B48007803280BDB9A4854
:1066000040689949086008468068486002209549BA
:1066100008704FF00108924801889248027800788B
:10662000401C904B1870904840F822108F4800781A
:10663000032809DB8E4840888D49088008468088F9
:106640004880022089490870784202B28748017860
:106650000078401C854B1870854820F81120B8F14F
:10666000010F72D1804880687F494968401A15D46B
:106670008048008828B97C48008900B27E4908809B
:1066800014E0794880687C49B1F9001088420DDD3A
:106690007548008900B27849088007E0754800888D
:1066A00020B97148008900B2744908806E4880683A
:1066B0007249B1F90010401AB0F57A7F15DD01205A
:1066C0006C490880684880686C49B1F90010401A2C
:1066D0006B49B1F90010884207DD634800896749BA
:1066E0000988401A00B2664908805F48806863499B
:1066F000B1F90010401AB0F57A7F2BDD6048B0F98F
:106700000000F0F794F841EC1A0B9FED5E0B53EC90
:10671000102BEFF7ABFF41EC180B53498968564A31
:10672000B2F90020501AF0F782F841EC190B53EC43
:10673000182BF0F7E5F814D24B4880684A494968AD
:10674000451A002D02DB284601E077E06842B0F5EB
:10675000C87F06DA0020474908804FF47A7048491C
:1067600008804A48007830BB0020494908804948E1
:10677000B0F90000B0F5967F05DA46480088401C65
:1067800000B2444908803B48008801280ED14148A6
:10679000B0F90000062809DB012401203B490870FC
:1067A00022463DA10020F4F7A9FD52E0002400207C
:1067B000364908704DE000240020364908803448EE
:1067C000B0F90000B0F5967F05DA31480088401C2A
:1067D00000B22F490880274B1B8873BB244BB3F9A9
:1067E0000030A3F5FA62002A01DB134600E05342B1
:1067F000B3F5967F19DC1E4BB3F90230A3F5FA61AD
:10680000002901DB0B4600E04B42B3F5967F0CDC20
:10681000174BB3F90430A3F5FA60002801DB0346F7
:1068200000E04342B3F5967F13DD194BB3F9003016
:10683000062B0EDB0020154908700AE000240A48E8
:10684000008900B20D4908800748008900B20A4952
:106850000880E0B204B0BDEC068BBDE8F08100001A
:1068600094490020D549002038850020D4490020D3
:10687000CE490020DA490020D8490020D64900201E
:10688000DC4900209A9999999999D93FCC490020DF
:10689000DE490020E0490020737465703D3D2564A9
:1068A0000A0000002DE9F04F2DED088B81B08146E4
:1068B0008A4617461C46129DB9F90400002801DBE0
:1068C000014600E0414200EE101AB8EEC0BABAF933
:1068D0000400002801DB014600E0414200EE101AEE
:1068E000F8EEC0BA3822FE49081FEFF7C9FD38227A
:1068F000FC49081FEFF7C4FD3822FB49081FEFF7DA
:10690000BFFD3822F949081FEFF7BAFD3822F849D0
:10691000081FEFF7B5FDF248001F80ED0EBAF148F1
:10692000001FC0ED0EBAB7F9000000EE100AB8EE75
:10693000C00ADFEDF00A80EE201AEB48001F80ED60
:106940000E1AB7F9020000EE100AB8EEC00ADFED29
:10695000E90A80EE201AE548001F80ED0E1AB7F90B
:10696000040000EE100AB8EEC00ADFEDE20A80EE85
:10697000201ADF48001F80ED0E1ADB48001F90ED43
:106980000E8AD0ED0E8AD948001F90ED0E9AD0EDF8
:106990000E9AD748001F90ED0EAAD0ED0EAA052042
:1069A00072E0D149091F01EB800191ED000AB4EEBC
:1069B000E80AF1EE10FA07D2CB49091F01EB80017A
:1069C00091ED000AF0EE408AC749091F01EB8001F2
:1069D00091ED000AB4EEC80AF1EE10FA07DDC249E3
:1069E000091F01EB800191ED000AB0EE408ABF491A
:1069F000091F01EB800191ED000AB4EEE90AF1EE06
:106A000010FA07D2B949091F01EB800191ED000A84
:106A1000F0EE409AB549091F01EB800191ED000AA3
:106A2000B4EEC90AF1EE10FA07DDB049091F01EB17
:106A3000800191ED000AB0EE409AAD49091F01EBCB
:106A4000800191ED000AB4EEEA0AF1EE10FA07D2E5
:106A5000A749091F01EB800191ED000AF0EE40AA61
:106A6000A349091F01EB800191ED000AB4EECA0AA7
:106A7000F1EE10FA07DD9E49091F01EB800191ED4F
:106A8000000AB0EE40AA401C0F288ADB9A4A9FED0C
:106A90009B0A0F219248001F06F0F4F80090984AD4
:106AA0009FED960A0F218E48001F06F087F880465A
:106AB000944A9FED920A0F218A48001F06F0E2F8DF
:106AC0008346914A9FED8D0A0F218648001F06F0EC
:106AD00075F80646012E05D1B8F1010F02D100204C
:106AE000009083467F48001F90ED0E0A8548D0ED48
:106AF000000A30EE600ADFED850AB4EEE00AF1EE3E
:106B000010FA23DD7648001F90ED0E0A7A48D0ED8A
:106B1000000A30EE600ADFED7E0AB4EEE00AF1EE24
:106B200010FA13DD6E48001F90ED0E0A7448D0ED88
:106B3000000A30EEC00AB0EEC00ADFED760AB4EE0D
:106B4000E00AF1EE10FA01D201200090009818B18D
:106B50000121714801600DE0B8F1000F03D0002061
:106B60006D49086006E06C480068012802D10220E7
:106B70006949086068480068002802DD14206749F8
:106B80000860BBF1000F03D00120654908600BE0ED
:106B90001EB100206249086006E0614800680128D3
:106BA00002D102205E4908605D480068002802DDCD
:106BB00014205C4908605A480068022805D1B8F1E1
:106BC000000F02D000205649086053480068022890
:106BD00003D116B1002050490860504800680028D1
:106BE00003DC5048006800281DDD38EE680ADFED40
:106BF0004E0AB4EEE00AF1EE10FA14D239EE690A48
:106C0000DFED490AB4EEE00AF1EE10FA0BD23AEEEB
:106C10006A0ADFED450AB4EEE00AF1EE10FA02D29C
:106C20000120288020803C480068002802DD0120E7
:106C3000208001E00020208039480068002802DD23
:106C40000120288001E000202880002095E02649CE
:106C5000091F01EB800191ED000AB4EEE80AF1EEA4
:106C600010FA07D22049091F01EB800191ED000ABB
:106C7000F0EE408A1C49091F01EB800191ED000AEA
:106C8000B4EEC80AF1EE10FA07DD1749091F01EB4F
:106C9000800191ED000AB0EE408A1449091F01EB12
:106CA000800191ED000AB4EEE90AF1EE10FA07D284
:106CB0000E49091F01EB800191ED000AF0EE409AA8
:106CC0000A49091F01EB800191ED000AB4EEC90ADF
:106CD000F1EE10FA2EDD0549091F01EB800125E0D8
:106CE000F88300203484002070840020AC840020CD
:106CF000E884002000000045844900200000FA4498
:106D00008C490020884900209049002000007A44E6
:106D10000000FA436F12833A5C4900207849002052
:106D2000604900207C490020CDCC4C3E91ED000A0A
:106D3000B0EE409A684901EB800191ED000AB4EE93
:106D4000EA0AF1EE10FA06D2634901EB800191EDF7
:106D5000000AF0EE40AA604901EB800191ED000AC3
:106D6000B4EECA0AF1EE10FA06DD5B4901EB8001D0
:106D700091ED000AB0EE40AA401C0A28FFF667AF6A
:106D800038EE680ADFED550AB4EEE00AF1EE10FACB
:106D90001AD239EE690ADFED510AB4EEE00AF1EEDB
:106DA00010FA11D23AEE6A0ADFED4C0AB4EEE00AAC
:106DB000F1EE10FA08D201211398018048480068CA
:106DC000401C4749086004E00021139801804448B2
:106DD000016043480068642806DD01202080288087
:106DE000404908604049086040480068012803D0D5
:106DF0003F480068012832D13E4890ED0D0AD0EDA1
:106E00000E0A30EE600AB0EEC00ADFED3B0AB4EEC7
:106E1000E00AF1EE10FA22D2384890ED0D0AD0EDDA
:106E20000E0A30EE600AB0EEC00ADFED330AB4EEAF
:106E3000E00AF1EE10FA12D2274890ED0D0AD0EDDB
:106E40000E0A30EE600AB0EEC00ADFED2B0AB4EE97
:106E5000E00AF1EE10FA02D20120208028802848B2
:106E60000068002804DD26480068401E24490860A8
:106E700024480068002804DD22480068401E21499B
:106E80000860208808B9288820B114201C490860AF
:106E90001C490860B4F9001014480160B5F90010ED
:106EA000134801600C4AD2ED0E1AB0EE611A134A73
:106EB000D2ED0E1AF0EE610A0E4AD2ED0E1AB0EEC5
:106EC000610AB5F90010B4F90000FDF799FD01B0B1
:106ED000BDEC088BBDE8F08FE48400208FC2F53C48
:106EE000804900205C490020604900207049002052
:106EF000744900206C840020CDCCCC3DA8840020B7
:106F0000784900207C49002070B5044620793D284E
:106F100002D141F23D0001E04FF48850054620883F
:106F20000022294606F07DF970BD000030B59FB003
:106F300004460D467C216846EFF7BBFAADF80250D7
:106F400003208DF8000001940448006818B16846D9
:106F50000249096888471FB030BD0000E44900209D
:106F60002DE9F04104460D46164694F8C60200EBA2
:106F70008001C1EB801004EB400840460DF0D0FECC
:106F80000746E7B3D4F8CC02062838D204F53470AB
:106F9000D4F8CC1200EBC110468004F53471D4F85B
:106FA000CC2201EBC211081D76224146EFF768FAA8
:106FB00045B1002104F53470D4F8CC2200EBC210A6
:106FC000017007E0022104F53470D4F8CC2200EB04
:106FD000C210017004F53470D4F8CC1200EBC1106B
:106FE000C767D4F8CC02401CC4F8CC020549D4F8D9
:106FF000CC020968884202D120460CF019FBBDE89A
:10700000F0810000EC4900202DE9F041A0B00446D9
:107010000D46164694F8C60200EB8001C1EB8010C5
:1070200004EB400840460DF07BFE074657B17C223A
:10703000064901A8EFF724FAADF80660029501A809
:10704000B84700BF20B0BDE8F08100004C810400CB
:107050002DE9F04105460C4616462746002087F8E4
:10706000C802324629463846FFF7CEFF3146384639
:10707000FFF75CFFBDE8F081F0B589B004460E462D
:107080004FF4BA612046EFF714FA202101A8EFF778
:1070900010FA31461E48006808F0E8F9054600BFBE
:1070A000284608B109B0F0BD00BFA4F8CA620020AC
:1070B000C4F8CC0284F8C70284F8C60284F8C5027A
:1070C00094F8C60200EB8001C1EB801004EB40078E
:1070D00094F8C6020F4901EB800000683860022076
:1070E0008DF804000120ADF814003968CDF81610B1
:1070F000049409480390324601A90548006808F045
:10710000DFF9054615B9012084F8C8022846C9E709
:10711000E849002044850020517003001CB5182167
:107120003048EFF7C6F900212E482C3880F84C1073
:1071300080F8491080F84D1080F84A1080F84E1001
:1071400080F84B1080F8461080F8481080F84710FF
:10715000002024492C3981F84400002121482C3892
:1071600080F8451020481F492C3948601F480860A6
:1071700000208862032103460122CDE90010114658
:10718000052008F075FF062009F019F8072009F01E
:1071900016F8082009F013F8092009F010F800216A
:1071A000062009F03DF90021072009F039F90021F6
:1071B000082009F035F90021092009F031F90021F2
:1071C000052009F02DF903200CF055FA01210520C6
:1071D00009F026F903200CF04EFAF4F7EFF90EF05F
:1071E00039FB1CBD606E002095360400B9360400E2
:1071F00038B50446134890F84900E8B1694611488B
:1072000006F0E8FD9DF8000000F0010088B10E488E
:1072100000210160818001460A4806F0C3F80A484F
:107220000088208008484088608007488088A080C7
:1072300005E04FF0FF3038BD4FF0FF30FBE7002096
:10724000F9E70000346E0020D840002001460548D0
:1072500002680A6042684A6002890A81807A8872FC
:1072600000207047786E002010B504462E4800219B
:10727000016081802D48016081802D4801608180FE
:107280002C48016081802C4890F84A0020B10622E9
:107290002549294806F0AFFA274890F8490020B15F
:1072A00006222249244806F0A6FA234890F84B000B
:1072B00020B106221E49204806F09DFA1E4890F88B
:1072C0004800012804D106221A491B4806F093FA07
:1072D0003CB315480088E0801348418821818188AB
:1072E00061811248008820801048408860800F48E3
:1072F0008088A0800E480088A0810D484188E181E7
:10730000818821820B48407800040A49097840EAC4
:1073100001200849C978084300EBC00101EB0010C7
:107320006061002010BD0000DE400020D840002039
:10733000E4400020EA400020346E00207CB50020AC
:1073400000900025002401A9144806F0A4FA9DF835
:10735000040008B36946114806F084F80F4890F815
:10736000490008B1E01C84B20C4890F84A0008B10A
:10737000E01C84B2094890F84B0008B1E01C84B2CC
:10738000064890F84800012801D1E01C84B2BDF8FD
:10739000000090FBF4F085B228467CBD346E0020DE
:1073A000052070471CB5F4F7E7F8002003210346D9
:1073B0000122CDE900101146052008F059FE0620F3
:1073C00008F0FDFE0021062009F02AF80021072020
:1073D00009F026F80021082009F022F800210920F0
:1073E00009F01EF80021052009F01AF800201CBD44
:1073F0007CB50121052009F013F8062501240020A1
:1074000000902346024601460190284608F030FECF
:1074100000BF18211548EFF74CF8002113482C380D
:1074200080F84C1080F8491080F84D1080F84A1010
:1074300080F84E1080F84B1080F8461080F8481005
:1074400080F84710002009492C3981F844000021B8
:1074500006482C3880F84510002004492C398862F1
:10746000F4F78AF8F4F7AAF800207CBD606E0020DB
:1074700038B50446194890F84C00A0422BD014B1FE
:10748000012C27D112E00021144806F0BAFD69460C
:10749000124806F08EFD9DF8000010B14FF0FF304D
:1074A00038BD00210D4880F84C1013E001210B4835
:1074B00006F0A7FD6946094806F07BFD9DF800002F
:1074C000012802D04FF0FF30EAE70121034880F89D
:1074D0004C1000BF00BF0020E2E70000346E002027
:1074E00038B50446244890F84900A04241D024B160
:1074F000012C29D0042C3BD112E000211E4806F0BB
:107500002EFD69461C4806F0E9FC9DF8000010B10C
:107510004FF0FF3038BD0021174880F8491027E0B0
:107520000421154806F01BFD6946134806F0D6FCF9
:107530009DF80000042802D04FF0FF30EAE7042154
:107540000D4880F8491013E001210B4806F007FDB3
:107550006946094806F0C2FC9DF80000012802D0E7
:107560004FF0FF30D6E70121034880F8491000BFF3
:1075700000BF0020CEE70000346E002038B504467E
:10758000194890F84400A0422BD014B1012C27D107
:1075900012E00021144806F06BFD6946124806F01F
:1075A00049FD9DF8000010B14FF0FF3038BD0020BC
:1075B0000D4981F8440013E001210B4806F058FD05
:1075C0006946094806F036FD9DF80000012802D002
:1075D0004FF0FF30EAE70120034981F8440000BF83
:1075E00000BF0020E2E70000346E00202DE9F043E8
:1075F00089B005460E4617469846DDF840900024AF
:107600005E4890F84600A8427AD015B1042D22D1E8
:1076100022E00021594806F0D5F808A9574806F09D
:10762000C1F89DF8200020B14FF0FF3009B0BDE84F
:10763000F0830021514805F071FF07A94F4805F07C
:107640002EFF9DF81C0010B14FF0FF30EEE7002137
:107650004A4880F846108DE00121484806F0B2F80B
:1076600008A9464806F09EF89DF82000012802D09F
:107670004FF0FF30DAE70621404806F07AF806A915
:107680003E4806F04BF89DF81800062802D04FF04F
:10769000FF30CBE7042E0FD10121384806F03FF927
:1076A00005A9364806F007F99DF81400012801D015
:1076B000701FBBE7E01C84B2042F0FD101212F48BB
:1076C00006F013F804A92D4805F0DBFF9DF8100023
:1076D000012801D0781FA9E7E01C84B2B8F1000F9F
:1076E00011D00121254805F066FF03A9234805F0C4
:1076F0002EFF9DF80C00012803D04FF0FF3095E7D6
:1077000039E0E01C84B2B9F1010F10D101211B480E
:1077100005F09EFF02A9194805F066FF9DF80800D4
:10772000012802D04FF0FF3080E7E01C84B22146F0
:10773000124806F08CF801A9104806F06BF8BDF865
:107740000400A04202D04FF0FF306FE704210B4845
:1077500005F0E4FE07A9094805F0A1FE9DF81C000C
:10776000042802D04FF0FF3060E70421034880F87E
:10777000461000BF00BF002058E70000346E002014
:1077800038B50446194890F84D00A0422BD014B1EA
:10779000062C27D112E00021144806F09DF9694615
:1077A000124806F06EF99DF8000010B14FF0FF305E
:1077B00038BD00210D4880F84D1013E006210B481C
:1077C00006F08AF96946094806F05BF99DF8000061
:1077D000062802D04FF0FF30EAE70621034880F880
:1077E0004D1000BF00BF0020E2E70000346E002013
:1077F00038B50446244890F84A00A04241D024B14C
:10780000012C29D0042C3BD112E000211E4806F0A7
:107810000EF969461C4806F0CCF89DF8000010B13E
:107820004FF0FF3038BD0021174880F84A1027E09C
:107830000421154806F0FBF86946134806F0B9F82C
:107840009DF80000042802D04FF0FF30EAE7042141
:107850000D4880F84A1013E001210B4806F0E7F8C4
:107860006946094806F0A5F89DF80000012802D0F5
:107870004FF0FF30D6E70121034880F84A1000BFDF
:1078800000BF0020CEE70000346E002038B504466B
:10789000194890F84500A0422BD014B1012C27D1F3
:1078A00012E00021144806F04DF96946124806F02E
:1078B0002CF99DF8000010B14FF0FF3038BD0021C9
:1078C0000D4880F8451013E001210B4806F03AF905
:1078D0006946094806F019F99DF80000012802D010
:1078E0004FF0FF30EAE70121034880F8451000BF60
:1078F00000BF0020E2E70000346E0020F8B5054626
:107900000F461646002E01DD062E02DB4FF0FF303B
:10791000F8BD454890F84B00A84278D0062E7DD29D
:10792000DFE806F07C03102730444DB106200090BC
:1079300001236A462921382010F092F9044600E01C
:1079400000246BE09DB1FF20009001236A462921AD
:1079500038200CF0ABFF0446601C18B19DF8000005
:10796000062802D04FF0FF3402E0002400E000249B
:1079700054E0009501236A460A21382010F070F97E
:1079800004464BE0FF20009001236A460A2138207C
:107990000CF08CFF0446601C18B19DF80000A84252
:1079A00002D04FF0FF3400E0002437E087B301211C
:1079B0001D4806F0B4F91D491B4806F0C9F9042119
:1079C000194806F0F1F8FF20009001236A460321D0
:1079D000154806F002F90021134806F0E5F89DF875
:1079E0000000012802D04FF0FF3091E700210E483F
:1079F00006F046F901210C4805F0C2FF01210A48B2
:107A000006F025F90024084880F84B5005E006E010
:107A1000FFE70024044880F84B5000BF01E000203D
:107A200076E7204674E70000346E0020D440002042
:107A300038B50446194890F84700A0422BD014B13D
:107A4000012C27D112E00021144806F0FEF9694606
:107A5000124806F0DCF99DF8000010B14FF0FF303D
:107A600038BD00210D4880F8471013E001210B4874
:107A700006F0EBF96946094806F0C9F99DF80000DF
:107A8000012802D04FF0FF30EAE70121034880F8D7
:107A9000471000BF00BF0020E2E70000346E002066
:107AA00038B50446184890F84800A04229D0A4B13F
:107AB000012C25D10121144806F0E0F9694612484D
:107AC00006F094F99DF80000012801D0A01E38BDF1
:107AD00001210D4880F8481012E000210A4806F004
:107AE000CDF96946084806F081F99DF8000010B10B
:107AF0004FF0FF30EBE70021034880F8481000BF4B
:107B000000BF0020E3E70000346E00201CB5002019
:107B1000032103460122CDE9001011460B2008F095
:107B2000BBFA0C2008F057FB0D2008F054FB002195
:107B30000C2008F08AFC00210D2008F086FC0021B2
:107B40000B2008F082FC052008F026F801210B200C
:107B500008F07BFC052008F01FF8F1F79AFC0C48B0
:107B60000021016041608160C1600A4808494860A5
:107B70000948086000210648C17300200449887341
:107B80000CF032FC08B100201CBD4FF0FF30FBE7C9
:107B9000846E002003950200C79602000146024849
:107BA000C089088000207047846E00207CB50446A0
:107BB00001208DF80000134806236A46012146681B
:107BC0003820B047054615B94FF0FF307CBDBCB139
:107BD0009DF800009DF8011040EA012000B22080CD
:107BE0009DF802009DF8031040EA012000B2608079
:107BF0009DF804009DF8051040EA012000B2A08025
